:020000040800F2
:10000000000008202D0C0108396700083B67000834
:100010003D6700083F6700084167000800000000D6
:10002000000000000000000000000000436700081E
:10003000456700080000000047670008496700089E
:100040007D0C01087D0C01087D0C01087D0C010868
:100050007D0C01087D0C01087D0C01087D0C010858
:100060007D0C01087D0C01087D0C01087D0C010848
:100070007D0C01087D0C01087D0C01087D0C010838
:100080007D0C01087D0C0108516700087D0C0108FA
:100090007D0C01087D0C01087D0C01087D0C010818
:1000A0007D0C0108696700086B6700087D0C01087A
:1000B0006D6700087D0C01087D0C01087D0C0108AE
:1000C0007D0C01087D0C01087D0C01087D0C0108E8
:1000D0007D0C0108716700087D0C01087D0C01088A
:1000E0007D0C01087D0C01087D0C01087D0C0108C8
:1000F000256800087D0C01087D0C01087D0C0108B5
:100100007D0C01087D0C0108296800087D0C0108A0
:100110007D0C01087D0C0108496800086968000829
:100120007D0C01087D0C01087D0C01087D0C010887
:100130007D0C01087D0C01087D0C01087D0C010877
:100140007D0C01087D0C01087D0C01087D0C010867
:100150007D0C01087D0C0108896800087D0C0108F0
:100160007D0C01087D0C01087D0C01087D0C010847
:100170007D0C01087D0C01087D0C010800000000C9
:100180007D0C01087D0C01087D0C01087D0C010827
:100190007D0C01087D0C01087D0C01087D0C010817
:1001A0007D0C01087D0C01087D0C01087D0C010807
:1001B0007D0C01087D0C01087D0C01087D0C0108F7
:1001C0007D0C01087D0C0108000000007D0C010879
:1001D0007D0C01087D0C01087D0C01087D0C0108D7
:1001E0007D0C01087D0C01087D0C01087D0C0108C7
:0801F0007D0C01087D0C0108E3
:100200000348044B834202D0034B03B118477047A5
:10021000D8010020D8010020000000000548064B4E
:100220001B1AD90F01EBA301491002D0034B03B1F4
:1002300018477047D8010020D801002000000000B6
:1002400010B5064C237843B9FFF7DAFF044B13B11E
:100250000448AFF300800123237010BDD8010020B3
:1002600000000000800C010808B5044B1BB10449D4
:100270000448AFF30080BDE80840CFE7000000006D
:10028000DC010020800C010811F0FF01034600F0A2
:10029000030239D08ABB026810B501EB012E0EEBC8
:1002A0000E4E8EEA0204A2F1013323EA0203A4F106
:1002B000013222EA0402134313F0803F0FD150F8B9
:1002C000044F84EA0E0CA4F10133ACF1013223EAAD
:1002D000040322EA0C02134313F0803FEFD00378AB
:1002E00023B936E010F8013F002B32D09942F9D102
:1002F00010BD8A4228D09A0729D01A7818460133AF
:10030000002AF6D110467047CAB90268A2F101333B
:1003100023EA020313F0803F08D150F8042FA2F122
:10032000013323EA020313F0803FF6D003785BB178
:1003300010F8013F002BFBD17047990705D01846F4
:1003400013F8012B002AF8D170471846DDE718464C
:10035000A1E7184610BD00BF2DE9F04F2DED0A8B27
:1003600097B0894600219246129100220021CDE9E2
:1003700004128046494611910F4611F8012B2D2A8F
:100380005ED801A050F822F063050008410400087F
:100390004104000841040008410400084104000829
:1003A00041040008410400084104000877030008E4
:1003B0007703000877030008770300087703000835
:1003C00041040008410400084104000841040008F9
:1003D00041040008410400084104000841040008E9
:1003E00041040008410400084104000841040008D9
:1003F00041040008410400084104000841040008C9
:100400004104000841040008770300084104000883
:1004100041040008410400084104000841040008A8
:100420004104000841040008410400084104000898
:1004300041040008D10A000841040008E50A000848
:1004400000210791302A00F09A80002308932F2A78
:10045000144640F2DD84002338461E461D4613E054
:100460000130082D1190C8BF03EB83030478C6BF89
:1004700002EB4302A2F13003A1F130062F2C05F16B
:100480000105224640F3CC8006EB8601392C02EBB5
:100490004101E5DDB6490993012201F017FE099BF0
:1004A00000287DD111990A46013111915478002D0F
:1004B00040F05185302C40F0FE840A46104601324F
:1004C00011921478302CF9D0C1F101010844A4F143
:1004D0003102082A39D8119F411CA4F130020A9137
:1004E0000125BE464FF0000C06EB860602EB4606E1
:1004F00000200EF1010211929EF80140A4F130019A
:10050000092900F2BD82DDF844E001300A460029E5
:10051000EFD00128D8BF05F1010B40F3508400EB68
:10052000050B0BF1FF34099703E07E00AC4200F0AD
:100530004584082D06EB860705F10105F5DD102D34
:10054000DCBF03EB83035B00F0E7652C40F0CD825A
:1005500000220121CDE909129446089A024340F095
:100560009D829FED818BBAF1000F01D0CAF80090F7
:10057000B0EE480B17B0BDEC0A8BBDE8F08F7A786F
:1005800002F0DF02582A00F0DC83013711973A7835
:10059000302AFAD0002A00F06B820123089356E734
:1005A0000020CDE90900AC46652C48D0452C46D04A
:1005B0004FF0000B002D40F08F80089B034340F06C
:1005C0005782099B002BCCD1692C00F0498400F3A1
:1005D0004284492C00F044844E2CC2D1654911A8B4
:1005E00001F0D4FF0028BCD0119B1B78282B00F011
:1005F0005185614802F0CCF8B0EE408BBAF1000FA3
:1006000002D0119BCAF80030079B002BB0D0B1EE8E
:10061000488BB0EE480B17B0BDEC0A8BBDE8F08FED
:1006200053490993012201F051FD099B0028B7D1DC
:10063000119A0A90511C11915478AC465EE7002D36
:100640008BD0DDF8449009F10102119299F8014034
:100650002B2C00F020822D2C00F0158200220B9212
:10066000A4F1300BBBF1090F00F20582302C119A76
:100670000AD1013211921478302CFAD0A4F1310150
:10068000082995D8A4F1300B511C119154782F2CC6
:1006900040F3CF838E460C9208E0013111919EF811
:1006A00001402F2CA2F1300B06DD8E460BEB8B02A6
:1006B000392C04EB4202F0DD0C9A891A082940F328
:1006C000B88344F61F6B0B9A002A3FF473AFCBF14B
:1006D000000B002D3FF471AF07EE906A0A9AB8EE56
:1006E000677BABEB0202BCF1000F08BFAC46102DDC
:1006F00009922A46A8BF1022092D8DED047B0EDD3C
:1007000006EE903A1D4B03EBC20313ED125B0F2D67
:10071000B8EE666BA7EE056B8DED046B30DC099BC4
:10072000002B00F0E882099B40F33782162B40F340
:1007300086830999C5F125038B4221DB0F4BC5F157
:100740000F054A1B03EBC50503EBC20395ED008BB8
:1007500093ED007B9DED046B28EE068B28EE078B56
:100760004CE700BFAFF30080000000000000000075
:100770004814010858140108BC140108000F0108AE
:10078000AB1A099A1344002B40F3B58113F00F0103
:100790000AD0C74A02EBC1029DED046B92ED007BCB
:1007A00027EE067B8DED047B33F00F0240D0B2F5CF
:1007B0009A7F00F36B83102A4FEA221340F3BB8425
:1007C000BC4C9DED047B00202246014613F0010F36
:1007D00001F101014FEA630304D092ED006B0120A7
:1007E00027EE067B012B02F10802EFD108B18DED57
:1007F000047B059BA3F15473059304EBC1049DEDA9
:10080000046B94ED007BAC4B27EE067B17EE902A31
:10081000AA4913408B428DED047B00F23783A8492F
:100820008B4240F2E083A74C4FF0FF33CDE9043414
:100830000023089300962B4662463946404602F054
:100840008DF88146002800F021830A9BCDF83CA05A
:10085000A3EB0B0B099B002BB4BF5A4600224FF0B1
:10086000000B23EAE3739FED8E9B0A920B935C4689
:10087000BFE0991A1F29A5EB010500F301820122AF
:1008800002FA01F30C9300230D932F44089B554467
:10089000AA4552461F44A8BF2A46BA42A8BF3A46B4
:1008A000002A03DDAD1ABF1AAAEB020A0A9B002B2D
:1008B00000F38C81002D00F3A281099B002B00F333
:1008C000D581002F00F3C581BAF1000F08DD214664
:1008D0005246404602F02AFA0446002800F0C2813F
:1008E00012993246404602F0B7FA8346002800F0DB
:1008F000B9810023C568C360214602F08BFA002845
:10090000C0F29483059F00F02F832146584602F0E1
:100910004FFCB0EE007BB4EEC70BF1EE10FA00F224
:100920004C81002D40F0BC81049B002B40F03382B1
:10093000C7F31303002B40F0E181B7EE007BB4EE68
:10094000C70BF1EE10FA00F10A83B6EE00BB20EE01
:100950000BBBB1EE4BAB5848DFF870C107EA0001A2
:10096000614553EC1A2B00F0A0810898E0B1B1F179
:10097000D46F19D8B4EEC9BBF1EE10FA11D8BCEEA1
:10098000CBBB1BEE103A012B38BF01230BEE103A04
:10099000B8EE4BBB002D40F08B82B1EE4B7B53EC9D
:1009A000172B03F1D660431AB0EE480B43EC1A2B19
:1009B0000C9102F00DFBAAEE008B8DED048B18EE6E
:1009C000907A0C99089B23B93B4B3B40994200F02D
:1009D0009A811299404601F04FFF3146404601F09E
:1009E0004BFF2146404601F047FF5946404601F083
:1009F00043FFD9F80410404601F0FEFE06460028E9
:100A000000F03081D9F810200232920009F10C0177
:100A10000C3001F08DFA9DED048B14AA13A9404609
:100A2000B0EE480B02F064FB1290002800F0F0805A
:100A30000121404602F03EF80446002800F01281F1
:100A4000139A002AC0F200810A9B0B9F02EB030A53
:100A5000089B149DD21A2A441B4B013A9A42C5F1B5
:100A60003605FFF606AF01230022CDE90C320CE774
:100A70009FED0D8BC2E5CDF844904FF0000B99E54A
:100A80000122099290E501220B9209F102021192D2
:100A900099F80240E4E500220B92F6E70025D0E544
:100AA0000000C0FFFFFFDF41000000000000000069
:100AB000000F0108F00F01080000F07F0000A07C8B
:100AC0000000907CFFFFEF7F02FCFFFF0000E07F53
:100AD00000220792791C11917A78002A3FF441ADE7
:100AE0000F46AFE401220792F4E7452C3FF430AD06
:100AF0000123099361E53FF49BAE5B4213F00F01C4
:100B00000AD0BD4A02EBC1029DED046B92ED007B61
:100B100086EE077B8DED047B1B113FF489AE1F2B06
:100B200035DC13F0100218BF6A229DED047B089299
:100B3000B24A0021D80704D592ED006B012127EEBF
:100B4000067B5B1002F10802F4D109B18DED047B44
:100B5000089BA3B1DDE90401C1F30A52C2F16B03A2
:100B6000002B0ADD1F2B40F3F0820020342B049071
:100B700040F32B834FF05C7305936A2308939DED3C
:100B8000047BB5EE407BF1EE10FA7FF453AE2223E6
:100B90009FED8F8BC8F8003030E51633FFF6F0ADCF
:100BA0000A9BA3EB0B0B944B03EBCB0393ED007B66
:100BB0009DED046B86EE078B20E5B6EE00BB20EEC4
:100BC0000BBB002D69D1B1EE4BABC4E621461A46F2
:100BD000404602F03BF80446002843D00146129AF2
:100BE000404601F07DFF00283CD00E90129940460F
:100BF00001F042FE0E9A1292002D7FF75EAE12991E
:100C00002A46404602F092F8129000287FF455AE32
:100C1000DDF83CA09FED708B2223C8F80030014620
:100C2000404601F029FE3146404601F025FE2146AE
:100C3000404601F021FE4946404601F01DFE59465E
:100C4000404601F019FED9E40B9BDDF828A09F1A5D
:100C5000FEE631463A46404602F068F8064600286D
:100C60007FF432AEDDF83CA01298D3E731460B9A00
:100C7000404601F0EBFF064600287FF422AEF1E784
:100C8000C2F17F4202F57F0202F57B420121E2328E
:100C900001FA02F3CDE90C13F7E5B0EE4BAB5AE6DF
:100CA000B7EE00ABB0EE4ABB55E6A7F1547305931F
:100CB0009DED04CBB0EE4C0B0C9102F089F950483D
:100CC000A0EE0ACB1CEE907A4E4B0C99384098421D
:100CD0008DED04CB6ED918EE902A03F154739A422D
:100CE00003D118EE103A0133BCD0474B4FF0FF321E
:100CF000CDE904236DE69DED048B7FE4BFEE00ABF0
:100D0000B7EE00BB27E651EC1B0B04F087FB04F0A9
:100D10003FFB049B41EC170B1D43C7F313073D43F7
:100D20003BEE477B27D19FED2E6BB4EEC67BF1EEF9
:100D300010FA7FF54EAE9DED048BDDF83CA01298C5
:100D40006DE70293079B019312AB00932F4A13ABFD
:100D500011A9404600F084FB10F00F0504463FF453
:100D600087AE062D40F0AA80013700239FED188B37
:100D70001197079342E49FED1C6BB4EEC67BF1EE36
:100D800010FAD8D49FED1A6BB4EEC67BF1EE10FAD0
:100D90007FF71FAECFE7049B012BAFD1002FADD162
:100DA000DDF83CA0129B184622239FED098BC8F862
:100DB000003034E707F15477059703E6099F0A9C52
:100DC000082D04440A9468DC5D46FFF78DBB00BF24
:100DD0000000000000000000000000000000F07FA4
:100DE0009535A094FFFFCF3F9535A094FFFFDF3FDF
:100DF00035E5AF350000E03F000F0108C00C0108E9
:100E00000000F07FFFFF9F7CFFFFEF7F980C010841
:100E1000AF490122384601F059F9002800F09280CC
:100E200000231E4618460A931D4609939C46FFF769
:100E3000BDBB44F61F629345A8BF934643E4A54B50
:100E4000099A03EBC20393ED008B9DED047B28EE22
:100E5000078BFFF7D3BB6E2C3FF4C0ABFFF781BB12
:100E60009D4911A801F092FB00283FF47AAB119B39
:100E70009A49013B11A8119301F088FB10B9119B0D
:100E8000013311939FED8E8BFFF7B8BB22239FEDAB
:100E90008C8BC8F80030FFF7B1BBBBF1100FDCBF83
:100EA00003EB830301EB43035D460020FFF721BB07
:100EB000B0EE4B7B73E50020FFF709BB129A3AB105
:100EC000352114A802F0BAF91299404601F0D4FC79
:100ED000013D139B042D00F2AA81DFE805F0032DEC
:100EE0002A1F0300149A049203F23342159B23F441
:100EF000801343EA02530593E40502D543F000430F
:100F00000593774A1A409DED048B002A7FF476AB57
:100F100000F03AFF22230360FFF770BB4FF0FF326F
:100F20006FF00043CDE90423E3057FF5E4AE059BB4
:100F3000E4E76B4B0593F7E7DDE91412159BCDE968
:100F40000412D9E711990A460131119154780646E5
:100F50000346FFF7AFBAAC460A90FFF7CFBABEEE32
:100F600000ABB6EE00BBF6E4DDE90CC3DDF83CA057
:100F70005C49C7F31302002D39D08A4200F0ED809E
:100F80005BBB049B1CEA030F29D0B0EE480B02F0B8
:100F90001FF8089B002B00F03181C7F30A53C3F1FF
:100FA0006B03002B40F32E81190501F17F530022C2
:100FB00003F5401343EC172BA0EE078B9FED427B0C
:100FC000474B28EE078B18EE902A1340002B7FF436
:100FD000B6AE2223C8F80030B1E63B42D5D1089B1B
:100FE000002BEBD1ABE602F15473059320E4002A09
:100FF0007CD1DDE904010246002840F0A080089B76
:10100000002B40F0EA80059B23F000473F0D3F0591
:10101000A7F580176FEA17536FEA035305934FF054
:10102000FF3304939DED048B1298F8E5DDE904127B
:101030000D43DDF83CA0D2D1C2F31303002BCED177
:1010400022F000473F0D3F05B7F1D66F3D46C6D9A8
:10105000DBF814301BB9DBF81030012BBFDD59462B
:101060000122404601F062FE2146834601F0D2FE95
:101070000028B4DD089B002BCAD0A5F580156FEAC7
:1010800015536FEA035305934FF0FF3304939DED1F
:10109000048B93E7144911A814AA01F093FA0528C8
:1010A0007FF4A7AA159B43F0FF4343F4E0030593A5
:1010B000149B04939DED048BFFF7A0BAAFF300805F
:1010C000000000000000F07F000000000000503928
:1010D00048140108000F01084C14010850140108BD
:1010E0000000F07FFFFF0F00AC0C0108002B4DD17A
:1010F000049B1CEA030F3FF472AFB0EE480B01F003
:1011000067FF089B002B48D0C7F30A53C3F16B035A
:10111000002B7ADD1B0503F17F51002001F5401102
:1011200041EC170BA0EE478BB5EE408BF1EE10FAB9
:101130007FF444AF36E6444C0021FFF75ABB2BBB8B
:1011400012EA0C0F3FF44BAFD7E74FF0FF3202FA31
:1011500003F3049A1A4004920FE5089A0499CAB15D
:101160003A4A3A40B2F1D46F14D8120DC2F16B0270
:101170004FF0FF3000FA02F2914219D0002B7FF4B9
:101180002CAF11EA0C0F3FF42AAFFEE63B423FF4CE
:1011900026AFB2E74FF0FF32EEE7129B38EE408BFE
:1011A000B5EE408BF1EE10FA18467FF438ADFAE553
:1011B000274B9F4232D0254B3B4003F580130593CC
:1011C000002304939DED048B09E7C2F14B024FF01D
:1011D000FF3393400B400593CFE41C4D3D40B5F1E8
:1011E000D66F3FF64AAFB5F15C7F3FF6E7AE2223FC
:1011F0009FED118B1298C8F8003010E5129838EE68
:10120000008B0CE538EE008BD8E638EE408BB5EE5F
:10121000408BF1EE10FA7FF4D1AEC3E50131CAD1B3
:1012200022239FED078B1298C8F80030F7E40023C3
:1012300062E600BFAFF30080000000000000000085
:10124000000000000000F07FF00F01080000F07FB8
:10125000FFFFEF7F014BFFF77FB800BF500000207A
:1012600010B4054C8446134620685DF8044B0A46CA
:101270006146FFF771B800BF0000002010B4054CB4
:10128000054B84460A4620685DF8044B6146FFF72B
:1012900063B800BF000000205000002010B51C4CB7
:1012A0008446134620680A466146FFF755F8B4EEB7
:1012B000400BF1EE10FAB0EE407B17D6B7EEC00B44
:1012C000DFED146AB0EEC06AB4EE666AF1EE10FAB1
:1012D0000BDDB0EEC77B9FED0C6BB4EE467BF1EE01
:1012E00010FA02DC236822221A6010BD17EE903A31
:1012F000002B094804DA01F053FAB1EE400A10BDA0
:10130000BDE8104001F04CBAFFFFFFFFFFFFEF7F89
:1013100000000020FFFF7F7FBC14010810B5224CA5
:10132000224B84460A4620686146FFF715F8B4EE62
:10133000400BF1EE10FAB0EE407B23D6B7EEC00BB7
:10134000DFED1B6AB0EEC06AB4EE666AF1EE10FA29
:101350000CDDB0EEC75B9FED126BB4EE465BF1EEB9
:1013600010FA03DC236822221A6010BD10EE103A36
:1013700013F0FF4FF9D10F4B17EE902A1340002BBB
:10138000F0D110BD17EE903A002B0B4804DA01F0B3
:1013900007FAB1EE400A10BDBDE8104001F000BAF6
:1013A000FFFFFFFFFFFFEF7F000000205000002045
:1013B000FFFF7F7F0000F07FBC1401082DE9F041A2
:1013C0000469B4EB611F05DC002303610023436162
:1013D000BDE8F08100F114054E1111F01F0C05EB72
:1013E000840E05EB860321D055F8261004339E4564
:1013F00021FA0CF1CCF120082DD92F461A6802FAF7
:1014000008F20A4347F8042B53F8041B9E4521FABF
:101410000CF1F3D8A31B9B00053B9B08013305EBA4
:10142000830445F8231079B104340DE09E4588BF4C
:1014300000F11002C8D953F8041B42F8041F9E455E
:10144000F9D8A41B05EB8404631B9B10AC42036119
:10145000BCD0BDE8F08141610029B5D02C46E3E75E
:101460002DE9F04F0F6885B0CDE90020BA780393DD
:10147000302A894640F0EC81FB1C1A78302A1C4641
:1014800003F10103F9D0E71B023FDFF8008318F8EE
:101490000230002B00F0EE80237818F803304FF074
:1014A000000A5546002B00F06D81264616F8013FD4
:1014B00018F80330002BF9D1B3490122304600F06F
:1014C00005FE834600284CD03278002D00F0A18123
:1014D000AB1B4FEA830B02F0DF02502A35464CD09B
:1014E000C9F80060BAF1000F74D12A1B013A072A2B
:1014F000514604DD5210072A01F10101FADC01987E
:1015000001F07AF98246002800F05F8200F11406AB
:10151000A542029666D90027B9460DE0202F1AD0C1
:101520003A4604372B7818F8033003F00F03934042
:1015300049EA0309A54258D015F8013D2E2BEDD1FB
:10154000A542EBD390490122284600F0BFFD0028B8
:10155000F0D0202FE4D1002246F8049B04279146C6
:10156000E0E7002D00F06581327802F0DF02AB1B6E
:10157000502A4FEA830B3546B2D16A782B2A00F005
:1015800046812D2A40F0D3800120AA7818F8021055
:101590004A1E182A05F1020600F2D380727818F864
:1015A0000220103901365AB90CE001EB810116F81E
:1015B000013F02EB4102A2F1100118F803200AB129
:1015C000192AF2DD00B149428B44C9F80060BAF132
:1015D000000F8AD0002F0CBF06250025284605B035
:1015E000BDE8F08F029E4FF0000946F8049B029B75
:1015F000F61AB610CAF81060484601F009FA009BC6
:1016000076011C68361AA64274DCC0F204810027F9
:10161000009B9A685A45C0F23B81009B5A685A4524
:101620004BDDA2EB0B0B5C4500F38D80DB68022BDE
:1016300000F0DD80032B00F04A81012B40F0DB80BD
:101640005C4540F0D880012C08D0611E504601F066
:1016500023FE002800F0CF80009B5A6803990A609F
:10166000029A0123CAF8103013600E9B6225C3F85A
:1016700000A0B3E744490122204600F027FD82463E
:10168000002840F08580637818F80320651C002A44
:1016900000F08080302B2C4640F0248114F8013F6C
:1016A000302BFBD018F80330B3FA83FA01274FEA46
:1016B0005A1A002B7FF4F9AE64E0012587B1009B34
:1016C000DA68022A6ED0032A70D0012A06D1B9073F
:1016D00004D5029B1A681743FA076AD445F010052F
:1016E0000E9BC3F800A0039B2846C3F800B005B0CA
:1016F000BDE8F08F361B3146504601F0CDFD074660
:1017000078B1711E4A11029B012753F8220001F0A3
:101710001F0207FA02F2024203D0B94200F3C98065
:10172000022731465046FFF749FEB34470E718F8E8
:1017300002104A1E182A05F101064FF000007FF63C
:101740002DAF2E46CCE60BF1FF36002F40F0A980DE
:10175000002E40F0A8807311029A06F01F0652F87E
:1017600023200123B34013425946504618BF47F087
:101770000207FFF723FE009BA4EB0B040225D3F81E
:1017800004B09BE7264697E648140108E80C0108D8
:101790002378254603F0DF03502B00F09380C9F82F
:1017A000005017E70F9BC3F101030F930F9B002B12
:1017B00094D0DAF81070029A4FEA8709904602EB4B
:1017C0008706002003E0964242F8040C43D9944671
:1017D00052F8041B4B1CF6D00131022DCCF800103E
:1017E00079D014F01F0440F0A580212578E70F9BE5
:1017F000002B3FF433AF0198514601F03DF85025DE
:101800000E9A00232846136005B0BDE8F08F002033
:10181000BBE6AB465FE6A61B51460198324601F097
:1018200085FA00F11403ABEB060B82460293002706
:10183000EEE6727818F80210751C2E4600293FF467
:101840004AAE16F8012F18F80230002BF9D13FE606
:10185000BC1C002719E6DAF80820974244DA0AEBA4
:1018600087017A1C0120022DCAF81020DDF80880BB
:10187000486130D0002A6ADC0022CAF81020002219
:10188000CAF81420009B9A680BF1010B5A45ACDA98
:101890000198514600F0F0FF0E9A0023A325136033
:1018A0009CE6012757E73146504601F0F5FC074614
:1018B00051E7B11E504601F0EFFC00283FF430AF75
:1018C00003272EE74FF0000B4FF0010A55E60F9B60
:1018D000002B90D0C2E6009B1A68013AA24260D069
:1018E0002225FDE60127E0E5DAF804100198013130
:1018F00000F082FF064600286DD0DAF81020023290
:1019000092000AF10C010C3000F012FB51460198D4
:1019100000F0B2FF3269012006EB8201022D024481
:10192000326106F114084861B246D4D09742BFF63E
:1019300058AF9FE7C144C4F1200459F8040C01F0EA
:1019400067F8A042BFF651AFDAF8102092E708EB33
:1019500082040AF11800DAF8142084424FEA520295
:101960002BD94546036842EAC37245F8042B50F868
:10197000042B84424FEA5202F4D8A4EB0A0119392D
:101980008908013148F8212008EB810102B10431B6
:10199000A1EB080292104145CAF810207FF472AF03
:1019A0006DE7621104F01F0458F822100122A240D2
:1019B0000A4214BF2125222592E6C8F800200AB168
:1019C0004146E4E7CAF8102059E7064B064852465C
:1019D000E42100F0EBFE034B03483246842100F083
:1019E000E5FE00BF5C140108701401082DE9F04702
:1019F000074649480E46354616F801EB10F80EC06A
:101A00001CF0080CF7D1BEF12D0F5AD0BEF12B0FF0
:101A100003BF96F800E06446AE1C64464BB9BEF1C5
:101A2000300F5CD00A23DFF8F4804FF0050A9946A6
:101A30000AE0102B4AD04FF0FF38B8FBF3F803FB55
:101A400008FA6FEA0A0A99460025284605E02CD0D4
:101A500009FB00C0012516F801EBAEF1300CBCF11A
:101A6000090F06D9AEF1410CBCF1190F0BD8AEF13C
:101A7000370C634510DDB5F1FF3FECD04045E6D9AA
:101A80004FF0FF35E7E7AEF1610CBCF1190F03D859
:101A9000AEF1570C6345EEDC6B1C0BD004B1404239
:101AA0000AB165B91160BDE8F087D445D0DD4FF0CB
:101AB000FF35D0E722233B602846002AF3D0711E71
:101AC000F0E796F800E00124AE1CA7E7BEF1300F66
:101AD00011D04FF00F0A6FF070489946B4E7337891
:101AE00003F0DF03582B0BD008234FF0070A6FF0E9
:101AF00060489946A8E7307800F0DF005828E8D120
:101B00004FF0100996F801E04FF00F0A02366FF01F
:101B100070484B4698E700BFE90D0108999999195B
:101B200064E700BF10B4044C8446134620685DF897
:101B3000044B0A46614659E70000002010B4044CEB
:101B40008446134620685DF8044B0A4661464DE71B
:101B50000000002070B50F4B0F4DAB42A3EB050604
:101B600007D0B610002455F8043B01349847A6422C
:101B7000F9D80FF085F8094D094B5E1BAB424FEACF
:101B8000A60606D0002455F8043B01349847A64227
:101B9000F9D870BD30180108301801083018010854
:101BA00034180108000000000000000000000000E0
:101BB0000000000000000000000000000000000025
:101BC00030B490F800F020F007016FF0000C10F036
:101BD000070491F820F040F048804FF000046FF0C7
:101BE0000700D1E9002391F840F000F1080082FAE3
:101BF0004CF2A4FA8CF283FA4CF3A2FA8CF34BBBAE
:101C0000D1E9022382FA4CF200F10800A4FA8CF226
:101C100083FA4CF3A2FA8CF3E3B9D1E9042382FAF4
:101C20004CF200F10800A4FA8CF283FA4CF3A2FA09
:101C30008CF37BB9D1E9062301F1200182FA4CF241
:101C400000F10800A4FA8CF283FA4CF3A2FA8CF3A8
:101C5000002BC6D0002A04BF04301A4612BAB2FACA
:101C600082F200EBD20030BC7047D1E9002304F0CF
:101C70000305C4F100004FEAC50514F0040F91F804
:101C800040F00CFA05F562EA05021CBF63EA0503A1
:101C900062464FF00004AAE710B4114C84461CF8C9
:101CA000013B11F8010BE25C02F00302012A225C05
:101CB00002F0030208BF2033012A06D01B1A0AD102
:101CC0000028ECD15DF8044B70472030181AE6D09C
:101CD0005DF8044B704718465DF8044B704700BF31
:101CE000E90D0108830730B547D0541E002A3ED0C5
:101CF000CAB2034601E0013C39D303F8012B9D072A
:101D0000F9D1032C2CD9CDB205EB05250F2C05EB11
:101D1000054535D9A4F1100222F00F0C03F1100E85
:101D2000E6444FEA121C1A46C2E90055C2E90255C0
:101D300010327245F8D10CF1010214F00C0F03EBD4
:101D4000021204F00F0C13D0ACF1040323F00303D0
:101D50000433134442F8045B9342FBD10CF00304B8
:101D60002CB1C9B21C4403F8011BA342FBD130BD06
:101D700064461346002CF4D1F9E703461446C0E745
:101D80001A46A446E0E700BF014B1868704700BF41
:101D900000000020242B2DE9F84F43D8012B41D01F
:101DA000804649481F468E4675461EF801BB10F80E
:101DB0000B4014F00804F7D1BBF12D0F6FD0BBF12D
:101DC0002B0F08BF9EF800B06FF0004908BF05F167
:101DD000020E73BBBBF1300F4BD00A273B460025E8
:101DE000B9FBF7F6284607FB169A05E03AD007FB41
:101DF00000C001251EF801BBABF1300CBCF1090F8E
:101E000006D9ABF1410CBCF1190F19D8ABF1370C65
:101E100063451EDDB5F1FF3FECD08642E6D24FF0C0
:101E2000FF35E7E7FFF7B0FF162303600020BDE8AA
:101E3000F88F102BD3D1BBF1300F23D01F46CEE744
:101E4000ABF1610CBCF1190F03D8ABF1570C634532
:101E5000E0DC6B1C2BD054B9002AE8D085BB1160A4
:101E6000BDE8F88FE245C2DA4FF0FF35C2E74042E5
:101E7000F2E79EF8003003F0DF03582B08D0082764
:101E80003B46ACE79EF8000000F0DF005828D5D1B3
:101E900010279EF801B03B460EF1020E9FE79EF818
:101EA00000B04FF0004905F1020E012491E7222312
:101EB000C8F8003032B10EF1FF3148461160CFE76B
:101EC0008146F8E74846B2E7E90D010862E700BF3E
:101ED00010B4044C8446134620685DF8044B0A464F
:101EE000614657E70000002010B4044C84461346B6
:101EF00020685DF8044B0A4661464BE7000000206D
:101F000010B4034CD4F8E040A4465DF8044B60479D
:101F10005000002049B1FF2A02D80A700120704702
:101F20008A2303604FF0FF3070470846704700BFB8
:101F3000844641EA000313F003036DD1403A41D3D4
:101F400051F8043B40F8043B51F8043B40F8043B93
:101F500051F8043B40F8043B51F8043B40F8043B83
:101F600051F8043B40F8043B51F8043B40F8043B73
:101F700051F8043B40F8043B51F8043B40F8043B63
:101F800051F8043B40F8043B51F8043B40F8043B53
:101F900051F8043B40F8043B51F8043B40F8043B43
:101FA00051F8043B40F8043B51F8043B40F8043B33
:101FB00051F8043B40F8043B51F8043B40F8043B23
:101FC000403ABDD2303211D351F8043B40F8043BC3
:101FD00051F8043B40F8043B51F8043B40F8043B03
:101FE00051F8043B40F8043B103AEDD20C3205D3D3
:101FF00051F8043B40F8043B043AF9D2043208D0CB
:10200000D2071CBF11F8013B00F8013B01D30B883C
:1020100003806046704700BF082A13D38B078DD01A
:1020200010F003038AD0C3F10403D21ADB071CBFEC
:1020300011F8013B00F8013B80D331F8023B20F856
:10204000023B7BE7043AD9D3013A11F8013B00F88F
:10205000013BF9D20B7803704B7843708B78837017
:102060006046704740EA01039B0710B501D1032A7F
:1020700017D8844601F1FF3E07E01EF8011F03F860
:10208000011B541E29B19C4622466346002AF4D106
:1020900010BD9444002CFBD003F8011B6345FBD119
:1020A00010BD8E468446DEF80040A4F1013323EAD9
:1020B000040313F0803F71460EF1040EDAD1043AA6
:1020C000032A4CF8044BEED87146D3E7002A3ED0E1
:1020D00030B584460446084380070B462ED1032AB8
:1020E00007D82BE0043A25D01EF0803F22D1032AE6
:1020F00022D92068194653F8045BA0F1013EA8429A
:10210000A4462EEA000E04F10404EBD09CF8000073
:102110000C7884421DD1E64668B11EF8010F11F813
:10212000014FA2EB0E03A04203F1FF3311D11CEBD0
:102130000303F1D1002030BDA44619469CF80000ED
:102140000C78A04205D1012AF4D0E646E4E7104617
:102150007047001B30BD00BF000000000000000001
:1021600002780B78012A28BF9A4240F0D8806DE9A6
:10217000044540EA0104CDE902676FF0000C4FEA24
:1021800044721AB380EA010414F0070F6BD100F017
:10219000070420F0070004F0030521F007014FEACF
:1021A000C505F0E8042314F0040FF1E804670CFA05
:1021B00005F462EA040266EA04060BD063EA04034B
:1021C000624667EA0407664604E000BFF0E80423BD
:1021D000F1E8046782FA4CF582EA0604A4FA8CF46A
:1021E0006CBB83FA4CF583EA0705A5FA8CF595B923
:1021F00050E9022351E9026782FA4CF582EA0604AB
:10220000A4FA8CF483FA4CF583EA0705A5FA8CF559
:102210002543DBD09CB92DBAB5FA85F424F0070428
:1022200027FA04F1DDE9026723FA04F303F0FF0063
:1022300001F0FF01FDE80445A0EB0100704724BA5E
:10224000B4FA84F424F0070426FA04F1DDE9026705
:1022500022FA04F202F0FF0001F0FF01FDE804455C
:10226000A0EB0100704714F0030F3CD110F0030401
:1022700028D150F8082B51F8083B82FA4CF582EA35
:102280000305A5FA8CF55DB950F8042C51F8043C0F
:1022900082FA4CF582EA0305A5FA8CF5002DE8D008
:1022A0002DBAB5FA85F424F0070423FA04F122FAD2
:1022B00004F202F0FF0001F0FF01FDE80445A0EB8D
:1022C000010070474FEAC40420F0030050F8082BC7
:1022D00021F0030151F8083B0CFA04F462EA04020D
:1022E00063EA0403C9E710F003041DD0A1EB040165
:1022F00020F00300E40750F8042B06D012D28B78AC
:102300005FFAA2F4E41A06D12BB1CB785FFAB2F4EB
:10231000E41A00D133B920465DF8104B7047A2EBA8
:102320000300704701F1040150F8042BCC0721F0A1
:10233000030151F8043B48D824D222F07F4482FAAA
:102340004CF594EA1325A5FA8CF50AD165B951F834
:10235000043B84EA0204B4EB036F0ED150F8042B63
:10236000EBE74FEA132355E035F07F454DD1087870
:10237000FDE80445C0F1000070474FEA126203F027
:10238000FF0347E002EA1C4482FA4CF594EA134545
:10239000A5FA8CF50AD165B951F8043B84EA020428
:1023A000B4EB034F0CD150F8042BEBE74FEA134387
:1023B00030E015EA1C4528D10B884FEA124229E08B
:1023C0004FEA124203EA1C4324E002F0FF0482FABF
:1023D0004CF594EA1365A5FA8CF50AD165B951F864
:1023E000043B84EA0204B4EB032F09D150F8042B18
:1023F000EBE74FEA13630DE015F0FF0F05D10B6813
:102400004FEA122223F07F4304E04FF00000FDE882
:102410000445704712BA1BBA82FA4CF482EA0304EC
:10242000A4FA8CF5B5FA85F402FA04F203FA04F37F
:102430004FEA1260FDE80445A0EB1360704700BF4F
:1024400030B404787CB10D7885B10A462B4602E0A1
:1024500012F8013F1BB1A342FAD130BC704710F80B
:10246000014F002CF1D1204630BC704710F8014FCD
:10247000002CFBD1F7E700BF08B410B5002A9DB0CF
:10248000044636DB4FF40273ADF814304FF000030E
:102490001B930291069120AB17D0013A4FF6FF71C2
:1024A00004920792ADF816101F9A019302A901F049
:1024B00005F8421C01DA8B232360029B00221A706C
:1024C0001DB0BDE8104001B070474FF6FF71049297
:1024D0000792ADF816101F9A019302A900F0EEFFC3
:1024E000431C01DA8B2323601DB0BDE8104001B00E
:1024F00070478B2303604FF0FF30F5E70CB410B545
:10250000214B00291C689CB038DB4FF000034FF4CE
:1025100002721B93ADF81420029006901FAB18D0E6
:1025200001394FF6FF7204910791ADF8162002A908
:102530001E9A0193204600F0C1FF421C01DA8B2352
:102540002360029B00221A701CB0BDE8104002B04C
:1025500070474FF6FF7204910791ADF8162002A95B
:102560001E9A0193204600F0A9FF431C01DA8B2339
:1025700023601CB0BDE8104002B070478B2323607D
:102580004FF0FF30F5E700BF0000002010B40468F2
:10259000013409E014F8013BA3F1410CBCF1190F1F
:1025A00098BF2033934208D111F8012B002AF1D1B2
:1025B000046001205DF8044B704700205DF8044B77
:1025C000704700BF09682DE9F04F4B1102EB830300
:1025D00011F01F0B07460CBF1846181D3C680CBFB6
:1025E0001D1F1D46002340F8043C617885B001346E
:1025F000002900F0A8809E469A461E460B460146DA
:102600001046DFF8889101975A46A846AC468346A3
:1026100010E0202B00F28F80564508DDE04502D9FE
:10262000BEF1070F5FDDE34554D34FF0080E14F8F9
:10263000013FB3B119F80370002FEAD00EF1010E7B
:10264000BEF1080F06F101063ADCDCF800301B0190
:1026500007F00F071F43CCF8007014F8013F002B60
:10266000E8D15B46084693461A46002E6BD0C44517
:1026700002D2BEF1070F73DD62454DD2111F6346D2
:1026800053F8044B41F8044FAB42F9D9A5EB0C03C6
:1026900023F00303691C04330CF1010C8C4588BF43
:1026A00004231344002143F8041BAB42FBD950F828
:1026B000043C002B4DD1AA4249D055F8043DF8E71F
:1026C000E345B4D200234CF8043C4FF0010EACF1CA
:1026D000040CBDE70023ACF104084CF8043CB246FE
:1026E000C4469E46A3E7CEF108008000CDE9022C47
:1026F000DCF800306746C0F1200E8446786800FAA6
:102700000EF21A4320FA0CF33A6047F8043FB8453A
:10271000F4D8DDE9022C86E750F8043CBBF1000F49
:10272000C7D0CBF1200B4FF0FF3121FA0BF10B405A
:1027300040F8043CBDE70846194629295B46019F3D
:1027400093461A4609D0042005B0BDE8F08F012356
:102750002B60052005B0BDE8F08F01343C6084E7B4
:10276000CEF10803DCF800109B00C3F1200E664692
:102770000C46776807FA0EF1214327FA03F431601B
:1027800046F8044FB045F4D876E700BFE80C0108DE
:102790009FED010B704700BF000000000000F87FB4
:1027A0009FED010A704700BF0000C07F00B50B4CD1
:1027B00025681446EE681A4685B003460D464CB1AE
:1027C00007490095CDE901143046064901F0C6FBE2
:1027D00001F0C2F804490C46F3E700BF00000020F6
:1027E000B0140108C0140108BC14010808B5134650
:1027F0000022FFF7DBFF00BF70B5C66905460C4637
:102800005EB1F368A3B153F82400E8B1026843F85D
:1028100024200023C0E9033370BD102001F080FBA9
:102820000646E861E8B10023C0E90033C0E902339D
:1028300021220421284601F06BF9EB69F060DB6886
:10284000002BE0D1002070BD012101FA04F6721DB9
:102850009200284601F05CF90028F3D0C0E9014657
:10286000D7E7034B034832466B21FFF79FFF00BFBA
:10287000F01401080815010870B5C66905460C4634
:102880004EB13CB1EB696268DB6853F822102160FD
:1028900043F8224070BD102001F042FB0246E8617F
:1028A00020B1C0E90066C0E90266EAE7024B0348CE
:1028B0008F21FFF77BFF00BFF01401080815010806
:1028C0002DE9F0410D6907460E461C4601F1140E34
:1028D0000020DEF800108BB202FB03434FEA134CDA
:1028E000090C02FB01CC01309BB203EB0C43854287
:1028F0004EF8043B4FEA1C44EBDC3CB1B368AB42FE
:1029000007DD06EB850301355C6135613046BDE8C6
:10291000F081716838460131FFF76EFF804690B153
:102920003269023206F10C0192000C30FFF700FB15
:10293000314638464646FFF79FFF06EB85030135D3
:102940005C613561E2E7034B03484246BA21FFF779
:102950002DFF00BF5C140108081501082DE9F8439C
:102960001746284A1E4608330C46092E82FB0312DE
:102970004FEAE3730546C3EB62033ADD4FF0010C07
:1029800000214FEA4C0C634501F10101F9DC2846B6
:10299000FFF732FF014670B3089B4361092F4FF0E8
:1029A0000103036112DC0A340927BE420BDDF61B6A
:1029B000264414F8013B0A22303B2846FFF780FFEB
:1029C000B4420146F5D10846BDE8F88304F1090890
:1029D00004EB0709444614F8013B0A22303B284621
:1029E000FFF76EFF4C450146F5D1A7F108044444BA
:1029F000DBE70021CBE70A46034B0448D321FFF76E
:102A0000D5FE00BF398EE3385C14010808150108B3
:102A1000B0F5803F034636BF030400201020B3F119
:102A2000807F3CBF1B020830B3F1805F3CBF1B01BD
:102A30000430B3F1804F03D3002B06DB0130704725
:102A40009B0003D45B0003D4202070470230704702
:102A500003307047036813F00702014607D0DA0716
:102A60001FD4980721D55B080B600120704798B2EE
:102A7000A0B11046DAB20AB908301B0A1A0704BF1F
:102A80001B0904309A0704BF9B080230DA0703D4FD
:102A90005B0800F1010006D00B6070471B0C102092
:102AA000E8E700207047202070479B080B60022059
:102AB000704700BF10B50C460121FFF79DFE02468E
:102AC00018B10123C0E9043410BD034B034840F2A0
:102AD0004511FFF76BFE00BF5C14010808150108E3
:102AE0002DE9F04FD1F810801569A84585B00E4644
:102AF000924605DB2A46534645468A4690461E4680
:102B0000DAF80830DAF8041005EB0804A342B8BF7D
:102B10000131FFF771FE8446002800F08B8000F140
:102B2000140707EB840E774505D23B46002243F895
:102B3000042B9E45FBD8143606EB88080AF11409CD
:102B4000464509EB850566D2A5EB0A03153B23F044
:102B500003030AF1150A043355452CBF9B464FF079
:102B6000040BCDF808E00394AE46E24605E0090CFC
:102B70002AD1B04507F104074AD956F8041B8DB293
:102B8000002DF4D0CC463C46002301965CF8040BA3
:102B9000216886B28AB2000C05FB0622090C1A4491
:102BA00005FB001101EB124192B242EA0142E645F7
:102BB00044F8042B4FEA1143E8D8019E47F80B3044
:102BC00056F8041C090CD4D03B68002248461D4628
:102BD0003C469446028801FB02C202EB15429BB2BE
:102BE00043EA024344F8043B50F8043B25684FEAAB
:102BF000134CABB201FB0C3303EB124370454FEAAD
:102C0000134CE7D3B04547F80B3007F10407B4D8AD
:102C1000DDE902E4D446002C02DC05E0013C03D0EF
:102C20005EF8043D002BF9D06046CCF8104005B0AA
:102C3000BDE8F08F034B044862464FF4B171FFF7D3
:102C4000B5FD00BF5C140108081501082DE9F0432B
:102C500012F0030383B0144607462DD10E46A4108C
:102C60001CD0FA698AB39568002D39D0E3074FF07C
:102C7000000906D4641011D0286898B10546E3070E
:102C8000F8D531462A463846FFF72AFF31468046B6
:102C90003846FFF7F1FD64104646EDD1304603B0EB
:102CA000BDE8F0832A4629463846FFF719FF286019
:102CB000C0F800900546E2E7013B184A52F823208D
:102CC0000023FFF7FDFD0646C9E7102001F028F9B3
:102CD0000246F861E0B10023C0E90033C0E90233E5
:102CE000012138460192FFF787FD019A054640B160
:102CF000012340F27121C0E9043100239060036098
:102D0000B4E7074B07482A4640F24511FFF74EFD4E
:102D1000054B044840F2B311FFF748FDF00E0108DF
:102D20005C14010808150108F01401082DE9F047AA
:102D30000D4691462B69496803EB6218AB6808F1B0
:102D400001049C4207464FEA621A04DD5B009C4284
:102D500001F10101FADC3846FFF74EFD0646002876
:102D60004DD0BAF1000F00F114000EDD0AF105029A
:102D70004FEA820C034606EB8202002143F8041B53
:102D80009342FBD1ACF114031844296905F11403F3
:102D900019F01F0903EB810129D0C9F1200E8446E7
:102DA0004FF0000A1A6802FA09F242EA0A024CF8E5
:102DB000042B53F8042B994222FA0EFAF2D84B1B3B
:102DC000153B23F00303043305F11502914238BF8C
:102DD000042340F803A0BAF1000F00D1444638465E
:102DE00034612946FFF748FD3046BDE8F0870438D6
:102DF00053F8042B40F8042F9942F9D8EEE7034B1F
:102E0000034832464FF4EF71FFF7D0FC5C14010821
:102E1000081501080B6984460069C01A16D10CF127
:102E2000140C14310CEB830210B401EB830301E0AA
:102E3000944508D252F8044D53F8041D8C42F7D043
:102E400005D24FF0FF305DF8044B7047704701200A
:102E50005DF8044B704700BF2DE9F04F15460A6935
:102E60002B69D21A002A83B0884640F0878001F18E
:102E7000140605F1140101EB830106EB830301E065
:102E80009E427ED253F8044D51F8042D9442F7D05F
:102E900075D32B460024454698466968FFF7ACFC7D
:102EA0008146002800F089802E69C460D8F810009F
:102EB00005F1140B08F1140E09F1140A05F11002C2
:102EC0000EEB80000BEB860157464FF0000CCDF85F
:102ED00004B05EF8044B52F8045F1FFA84FBABB2F7
:102EE000A3EB0B03240C6344C4EB154404EB234411
:102EF0009BB243EA0443704547F8043B4FEA244C35
:102F0000E7D8A0EB080208F115084045A2F1150228
:102F100034BF0020012092080028DDF804B002F13F
:102F200001044FEA840408BF04240BEB0405A94202
:102F3000544433D92746284650F8043B1CFA83FEF4
:102F40001A0C634402EB2E429BB243EA02438142D5
:102F500047F8043B4FEA224CEED80139491B21F0D7
:102F600003010C4423B954F8043D013E002BFAD070
:102F70004846C9F8106003B0BDE8F08F89DA012433
:102F80008BE70021FFF738FC814678B1012200234E
:102F9000C0E90423484603B0BDE8F08F00284FEA9B
:102FA000820208BF00220AEB0204DBE7064B074857
:102FB0004A4640F23721FFF7F9FB034B03484A46E4
:102FC00040F24521FFF7F2FB5C14010808150108E7
:102FD00082B08DED000B164B019A1340A3F1507394
:102FE000002B06DD00221946104641EC100B02B002
:102FF00070475B42B3F1A07F4FEA235209DA4FF4E6
:103000000023134100221946104641EC100B02B078
:103010007047A2F114031E2BDABF4FF00042DA40D2
:10302000012200231946104641EC100B02B07047F4
:103030000000F07FF8B5046900F1140606EB840483
:10304000271F54F8045C2846FFF7E2FCC0F1200378
:103050000A280B6033DDBE42A0F10B0119D254F8EF
:10306000080C21B3C1F120078D4020FA07F2154367
:103070008840A4F1080145F07F538E4243F4401389
:1030800019D254F80C1CF9400843024643EC102BAB
:10309000F8BD0B280AD005FA01F141F07F5300205A
:1030A00043F44013024643EC102BF8BD002045F0DA
:1030B0007F5343F44013024643EC102BF8BDC0F19C
:1030C0000B0C25FA0CF1BE4241F07F5338BF54F887
:1030D000081C00F1150034BF21FA0CF1002105FA9B
:1030E00000F0084343F44013024643EC102BF8BDB4
:1030F0002DE9F0430E4683B0012159EC108B1546A3
:10310000FFF77AFB0446002846D0C9F30A57C9F3F3
:1031100013030FB143F480130193B8F1000313D1EB
:1031200001A8FFF797FC019B636101222030226117
:103130000FB3A7F233470744C0F13500376028606A
:10314000204603B0BDE8F08368460093FFF782FC99
:10315000019BF8B10099C0F1200203FA02F2C340CA
:103160000A430193002B62610CBF01220222A3617A
:103170002261002FDDD104EB8203A0F232403060E7
:103180001869FFF745FCC0EB42102860204603B0E9
:10319000BDE8F083009AE5E7034B0448224640F27D
:1031A0000F31FFF703FB00BF5C140108081501088D
:1031B000F0B583B00E4669460746FFF73BFF01A90D
:1031C000304655EC104BB0EE407BFFF733FF3369D0
:1031D0003A69D21ADDE900315B1A03EB4213002B86
:1031E00009DD17EE902A02EB035545EC174B87EEED
:1031F000000B03B0F0BD10EE902A51EC100BC3EBA6
:10320000033302EB035141EC100B87EE000B03B0CC
:10321000F0BD00BF172808DDB7EE000BB2EE047B4F
:10322000013820EE070BFBD17047034B03EBC003C3
:1032300093ED040B704700BFF00E010801394911EE
:1032400001F1010C116902F1140303EB81018B42BE
:1032500000EB8C0C16D210B5A0F1040E53F8044B01
:103260004EF8044F9942F9D88B1A153B23F003030B
:1032700004331844844504D9002340F8043B8445B2
:10328000FBD810BD844505D9002340F8043B844594
:10329000FBD87047704700BF03694A11934200F1A1
:1032A000140009DA00EB830302E053F8042DAAB9F5
:1032B0008342FAD80020704700EB8203F8DD11F05A
:1032C0001F01F5D010B450F8224024FA01F28A40D0
:1032D000944209D001205DF8044B704701207047EB
:1032E00053F8042D002AF5D18342F9D800205DF867
:1032F000044B70472DE9F0478F681D46AF420B68BD
:103300000C46164636D8B1F90CC01CF4906F0ED19D
:103310003D46184631462A4600F010FDA368DF1BE3
:103320002368A7602B4400202360BDE8F0874A692A
:10333000096902EB42025F1A02EBD2726B1C521057
:103340003B44934292BF914699461A461CF4806FC3
:10335000804611D0114600F013FC824600B321696B
:103360003A46FEF7E5FDA38923F4906343F080031A
:10337000A38105E02F46CCE700F004FE824658B159
:103380000AEB0703A9EB0707A760C4F810A0C4F86D
:10339000149023602F46BCE72169404600F070FC82
:1033A000A3890C2243F04003C8F800204FF0FF30FF
:1033B000A381BAE72DE9F04F9368176883B092466E
:1033C000002B74D04FF0000B8B680A6881460C46C6
:1033D0005D4645E0B4F90C3013F4906F2CD0D4E97D
:1033E0000401161A01EB410202EBD272711C521059
:1033F0002944914292BF904688460A465B0539D5DA
:103400001146484600F0BCFB019000283DD03246F2
:103410002169FEF78DFDA289019B22F4906242F0A2
:103420008002A2819819A8EB0606A660C4F8148051
:1034300023612060A8462E463246594600F07EFCA5
:10344000DAF80810A3682268A3EB08033244491B8A
:10345000A3602260CAF8081049B3D7E900B508375D
:1034600098461046002DF8D09D421E46B2D2A8467E
:103470002E46E1E70146484600F084FD0346002859
:10348000D0D12169484600F0FBFBA3890C2243F010
:103490004003C9F800204FF0FF30A3810022002331
:1034A000CAF80820CAF8043003B0BDE8F08F002045
:1034B0000023CAF8043003B0BDE8F08F2DE9F04FC7
:1034C0001C468B891D069DB088468146934603D5D0
:1034D0000B69002B00F0F1800023099343F22003D5
:1034E000ADF829309BF800307D4D03940126002B68
:1034F00073D0DA4603E01AF8013F002B75D0252B74
:10350000F9D1BAEB0B0473D19AF80020002A64D0E9
:1035100000234FF0FF32CDE905230AF1010A04939D
:1035200007938DF853301A9305E0049A06FA03F3D3
:103530001A430492A2465446052214F8011B284659
:1035400000F09EFCA346431B0028EED1049BD80646
:1035500044BF20228DF8532019079AF8001044BF69
:103560002B228DF853202A2950D1039A1168043256
:10357000002903927CDB07919AF801102E295BD079
:10358000584C0322204600F07BFC38B1049B001B02
:103590004022824013430BF1010B04931BF8011BE3
:1035A00051488DF82810062200F06AFC002865D0EA
:1035B0004E4B002B55D003AA00924D4B424604A916
:1035C0004846AFF3008007467A1C06D0099B3B446F
:1035D00009939BF80030002B8BD1B8F80C305B06B8
:1035E0007AD409981DB0BDE8F08FBAEB0B04F4D083
:1035F00023465A4641464846FFF77CFE0130ECD050
:10360000099B9AF80020234409937FE7A1F1300237
:10361000092A88BFD346B1D8079B00E0013421783E
:1036200003EB830302EB4303A1F13002092AF5D92E
:103630002E290793A346A3D19BF801102A2927D14D
:10364000039B9BF802101A6805920433002A0BF1C1
:1036500002000393B8BF4FF0FF338346B8BF059312
:103660008EE7039B073323F0070308330393ADE78B
:10367000494243F00203079104937DE703AA0092B5
:103680001B4B424604A9484600F040FD07469BE715
:10369000A1F130020023092A05930BF1010B3FF63B
:1036A0006FAF1BF8011F03EB830302EB4303A1F190
:1036B0003002092AF5D9059362E7402100F060FA4B
:1036C000C8F80000C8F8100018B14023C8F814303A
:1036D00002E70C23C9F800304FF0FF3082E700BF4B
:1036E00038150108401501084415010800000000C4
:1036F000F532000810B4034CD4F8E440A4465DF859
:10370000044B60475000002082B049B15AB16BB100
:1037100013780B601278101E18BF012002B070479A
:1037200001A9002AF3D1104602B070476FF00100E2
:10373000F4E700BF00207047024A0349034800F045
:103740007DBB00BFBC0100208D3A000804000020B2
:103750000C4B4168994210B5044601D000F096F92F
:10376000A168094B994202D0204600F08FF9E16828
:10377000064B994204D02046BDE8104000F086B9BF
:1037800010BD00BFF40100205C020020C402002034
:10379000002070472DE9F8432A4C2B49DFF8BC90F4
:1037A000DFF8BC80294FC4F8381100250423082213
:1037B000294604F15C00264EE360C4E90055C4E9E3
:1037C0000455A5606566A561FEF78CFA214B636719
:1037D0000822294604F1C400C4E90849C4E90A875B
:1037E000C4E91A55C4E91E552567C4F8CC50C4F87D
:1037F00080502663FEF776FA174BC4F8DC30294672
:1038000004F16803082204F59670C4F88830C4E90E
:103810002398C4E92576C4E93455C4E93855C4F879
:10382000D850C4F83451C4F8E850FEF75BFA04F1FC
:10383000D003C4E93D98C4E93F76C4F8F030BDE850
:10384000F88300BFF401002039370008D947000889
:10385000FD4700080900010012000200714700083E
:1038600099470008F8B5254BD3F838310646002BA8
:103870003CD0234FD7E90134013B04D51DE05A1C4D
:1038800004F1680419D0B4F90C50013B002DF6D1B5
:103890001C4BE360C4E90155C4E904556566256025
:1038A000A5610822294604F15C00FEF71BFAC4E971
:1038B0000D55C4E912552046F8BD3D680DB12F469F
:1038C000D8E74FF4D671304600F05AF9044680B17B
:1038D0000423C0E900530C302946A0604FF4D07295
:1038E0002546FEF7FFF93C602F46C3E7FFF752FF7E
:1038F000BFE70C2338603360DDE700BFF401002030
:10390000BC0100200100FFFF036A03B17047044BB4
:10391000044AD3F838310262002BF7D13AE700BFEE
:10392000F401002051370008704700BF704700BF06
:10393000024A0349002000F081BA00BFBC01002008
:1039400035370008024A0349002000F077BA00BF6B
:10395000BC0100209137000808B5062001F06EF97F
:1039600001200CF029FE00BFB1F90C302DE9F04127
:103970001E070C4680463DD44A68002A56DDE56A9B
:10398000002D34D00022D8F80060C8F8002013F4CD
:103990008052216A57D101234046A847451C024660
:1039A00066D0B4F90C30E56A216A580705D563681A
:1039B000D21A636B0BB1236CD21A00234046A8477E
:1039C000431C42D00023636023692360A389DF0482
:1039D00000D56065616BC8F8006041B104F1440333
:1039E000994202D0404600F04BF900236363002067
:1039F000BDE8F0810E69002EF9D09B070D6808BF65
:103A00004B690E6018BF0023AD1B8B600BE02B468B
:103A10003246216AA76A4046B847B0F1000CA5EBD0
:103A20000C05664406DD002DF1DCE0E70A6C002A97
:103A3000A5DCDCE7B4F90C3043F04003A3814FF080
:103A4000FF30BDE8F081626DAFE7D8F80010B4F93F
:103A50000C301D29F0D80C4ACA40D507ECD5226994
:103A6000226000226260DA04B4D50029B1D0B1E747
:103A7000D8F80030002B94D01D2B01D0162BD9D1B3
:103A8000C8F80060B3E700BF010040200B69B3B184
:103A900010B5044682B008B1036A5BB1B1F90C30CD
:103AA00013B9002002B010BD204602B0BDE810409E
:103AB000FFF75ABF0191FFF727FF0199EEE70020BA
:103AC000704700BFB8B138B50D4A036915680446A0
:103AD0002BB10DB12B6A53B1B4F90C300BB90020E6
:103AE00038BD21462846BDE83840FFF73DBF28468F
:103AF000FFF70AFFF0E7034A0349044800F09EB9C4
:103B000000000020BC0100208D3A000804000020C5
:103B100070B5A1FB025454B9294600F031F80646AD
:103B200018B12A462146FEF7DDF8304670BD0C225A
:103B300002600026F9E700BF70B5104E33680546F5
:103B40000C46B3B12146284600F000FE431C0CD0C1
:103B5000C41C24F00304A04205D0211A284600F01A
:103B6000F5FD013001D0204670BD4FF0FF342046F6
:103B700070BD194600F0EAFD3060E3E73003002035
:103B80002DE9F843CD1C25F0030508350C2D38BF71
:103B90000C25002D064618DBA94216D8DFF8DC807C
:103BA00000F0F6FBD8F80420A2B1144603E06368E5
:103BB00022467BB11C4623685B1BF8D40B2B1FD815
:103BC0009442636854D053600CE00C2333600020AF
:103BD000BDE8F88329463046FFF7AEFF431C044694
:103BE00019D00560304600F0D5FB04F10B00231D11
:103BF00020F00700C21A1CBF1B1AA350BDE8F883AF
:103C000061199442256014BF5160C8F804106351D3
:103C100063684B60E6E7D8F804701FB33C467F68E2
:103C2000002FFBD123683946304604EB030900F02E
:103C30008DFD814516D12368ED1A29463046FFF7E0
:103C40007BFF01300ED02368D8F804202B4423607A
:103C5000536883B1A34203D01A465B689C42FBD1F0
:103C60000023B0E70C233360304600F093FBAEE74F
:103C7000C8F80430B6E7C8F80470B3E73003002092
:103C8000002950D038B551F8043C0C1F002BB8BFA8
:103C9000E418054600F07CFB274A13682BB1A342C9
:103CA0000CD92168601883422CD0636028461460C8
:103CB000BDE8384000F06EBBA3420FD81A465B68DF
:103CC000002BF9D111685018844217D02CD36360AF
:103CD00054602846BDE8384000F05CBB11685018BD
:103CE000A04214D020D8216860188342EFD1186810
:103CF0005B680844C4E900035460EAE723680B44A6
:103D00001360E6E718685B6808442060CDE7206828
:103D10000144501883421160DBD1D3E9000401440F
:103D2000C2E90014D5E770470C232B602846BDE894
:103D3000384000F02FBB00BF3403002088420ED96A
:103D40008B1883420BD900EB020C002A6ED062461E
:103D500013F801CD02F801CD9942F9D170470F2A2D
:103D60000FD8034602F1FF3C002A5FD00CF1010C92
:103D7000013B8C4411F8012B03F8012F6145F9D167
:103D8000704740EA01039B0751D1A2F1100370B5BF
:103D900001F1200C23F00F0501F1100E00F11004C9
:103DA000AC441B095EF8105C44F8105C5EF80C5CD7
:103DB00044F80C5C5EF8085C44F8085C5EF8045C4F
:103DC00044F8045C0EF1100EE64504F11004E9D14C
:103DD000013312F00C0F01EB031102F00F0400EBA2
:103DE000031328D0043C24F003064FEA940C1E442D
:103DF0001C1F8E465EF8045B44F8045FB442F9D1A0
:103E00000CF1010402F0030203EB840301EB8401D3
:103E100002F1FF3C4AB10CF1010C013B8C4411F85A
:103E2000012B03F8012F6145F9D170BD704702F1F4
:103E3000FF3C03469AE72246EAE700BF2DE9F84334
:103E40000746884616464FF00009D6E90154013D61
:103E500010D4A389012B08D9B4F90E3001332146BF
:103E6000384602D0C04749EA0009013D6B1C04F105
:103E70006804EED13668002EE7D14846BDE8F883E5
:103E800001F0FF01102A2BDB10F0070F08D010F80B
:103E9000013B013A8B422DD010F0070F42B3F6D10F
:103EA000F0B441EA012141EA014122F007047FF028
:103EB00000070023F0E80256083C85EA010586EA7F
:103EC000010685FA47F5A3FA87F586FA47F6A5FABB
:103ED00087F68EB9EED1F0BC01F0FF0102F00702C7
:103EE00032B110F8013B013A83EA010313B1F8D172
:103EF0000020704701387047002D06BF3546033853
:103F0000073815F0010F07D1013015F4807F02BF8B
:103F1000013015F4C03F0130F0BC0138704700BFDC
:103F2000024B01461868FFF72BBE00BF00000020BF
:103F3000024B01461868FFF7A3BE00BF0000002037
:103F40000CB400B583B004AB53F8042B019300F01C
:103F500069FA03B05DF804EB02B070470EB410B517
:103F600083B005AB064C53F8042B0193014620683F
:103F700000F058FA03B0BDE8104003B0704700BF2E
:103F8000000000202DE9F041144641B30AB3064673
:103F90000D4600F037FC8442074602D8B4EB500FC0
:103FA00013D821463046FFF7EBFD804650B1BC42A6
:103FB0002246294628BF3A46FDF7BAFF2946304631
:103FC000FFF75EFE4046BDE8F081A8464046BDE8EA
:103FD000F081A046FFF754FE4046BDE8F081BDE801
:103FE000F0411146FFF7CCBD2DE9F84F92461F4630
:103FF0000A698B68DDF828909A42B8BF1A46CAF859
:10400000002091F843300C46064613B10132CAF83D
:104010000020226891065FD5DAF800300233CAF832
:104020000030226812F0060F11461DD1E168994256
:10403000D8BF114618DD4FF0000804F1190B05E058
:10404000E568DAF80030ED1A45450CDD01235A46E3
:1040500039463046C847013008F10108F0D14FF029
:10406000FF30BDE8F88F216894F84330003B18BF5B
:1040700001238A060AD5E1185A1C302081F8430032
:10408000224494F8451082F84310023304F14302AD
:1040900039463046C8470130E1D02368DAF800508D
:1040A000216903F00603042BD4E902201BD08A42C5
:1040B00020DD4FF00008521A90441A34002501E028
:1040C000454517DA0123224639463046C8470130B4
:1040D00005F10105F4D1C2E712F0060F0DD0003B47
:1040E00018BF0123D2E7401B8A4220EAE078E2DCD5
:1040F0000028E2DC0020BDE8F88FE168DAF8003043
:104100009942D8BF114696DCAEE700BF2DE9F047D3
:10411000174684B00A7E0C9D0C460646984601F16F
:10412000430C002A35D0A2F15803D9B2202969D80E
:10413000202B67D8DFE813F0E60066006600660013
:104140006600660066006600660066006600AC00F9
:10415000700066006600660066007000660066001B
:104160006600660021008300C60066006600B60097
:104170006600830066006600EC002B6822686169B7
:10418000181D286010061B6802D4520600F1E0805A
:1041900019600023E1462361CDF800803B4603AA65
:1041A00021463046FFF720FF013020D023694A46E0
:1041B00039463046C047013019D02368E068DDF841
:1041C0000C909B0718D5484516DD002504F1190A07
:1041D00004E0E068A0EB0903AB420DDD0123524689
:1041E00039463046C047013005F10105F1D14FF0A5
:1041F000FF3004B0BDE8F0874845B8BF484604B07A
:10420000BDE8F08784F84220012004F14209002330
:10421000206184F84330BFE72A682368111D18061F
:10422000296002D4590600F19580106801460028E3
:104230006268C0F2938054484FF00A0E15E020687F
:104240002B6810F0800F53F8041B02D1400648BFC2
:1042500089B26F2A4C482B6014BF4FF00A0E4FF002
:10426000080E0023626884F84330002AA26051DB04
:10427000236823F00403236000294BD1002A7BD15B
:10428000E146BEF1080F56D0ACEB0903236183E78A
:104290002B681A6804332B6004F1420984F8422029
:1042A0000120B4E72B686268191D2960D3F80090DB
:1042B00000214846FFF7E4FD002863D0A0EB090089
:1042C0006060A4E7236843F02003236078222F482E
:1042D00084F845202A6813F0800F52F8041B03D19C
:1042E00013F0400F18BF89B22A60DA0744BF43F0C9
:1042F0002003236019B9236823F0200323604FF0C3
:10430000100EAEE7582384F845301F482368E1E7D4
:104310002368DBE77546E146B1FBF5F305FB131AAD
:104320000A46AA4210F80A1009F8011D1946F3D2EC
:10433000BEF1080FA8D12368DD07A5D562682369FF
:104340009A42A1DC302309F8013C09F1FF399BE7CF
:1043500019801EE7B2F90010084668E72D20002AF0
:10436000A26084F8430002DB23F0040323600A25E3
:1043700005484942AE46CEE7037884F8423004F15E
:1043800042097EE7606842E74C15010860150108A4
:10439000704700BF704700BF9368013B002B9360DC
:1043A00011DA10B49469A34209DB0A2907D0136813
:1043B000581C1060197008465DF8044B70475DF892
:1043C000044B00F073B91368581C1060197008464C
:1043D000704700BF9BB1F8B5134406460F46541E04
:1043E0005D1E01E0AC4208D014F8011F3A46304689
:1043F000FFF7D2FF431CF5D1F8BD0020F8BD002027
:10440000704700BF936810B514461BB918460023C7
:10441000636010BD00F0FEF90023A3600023636019
:1044200010BD00BF2DE9F04FA1B08B4691461C4650
:10443000049018B1036A002B00F01C81BBF80C300B
:10444000180740F19580DBF81030002B00F09080C9
:104450000023CA460D9343F22003ADF839309AF891
:104460000030864E07940127002B79D0D14604E016
:1044700019F8013F002B00F08580252BF8D1B9EB0E
:104480000A0840F0828099F80030002B68D00023A1
:104490004FF0FF32CDE9092309F1010908930B938D
:1044A0008DF863301E9305E0089A07FA03F31A4368
:1044B0000892A1464C46052214F8011B3046FFF72E
:1044C000DFFCA246831B0028EED1089BD90644BF1F
:1044D00020228DF8632099F800101A0744BF2B2280
:1044E0008DF863202A2966D1079A116804320029C1
:1044F0000792C0F29A800B9199F801102E2970D082
:104500005F4C03222046FFF7BBFC38B1089B001B21
:104510004022824013430AF1010A08931AF8011B52
:1045200058488DF838100622FFF7AAFC002800F042
:104530008280554B002B69D007AA0092534B0498F8
:104540005A4608A9AFF300800390039B013307D0BC
:104550000D9B039A13440D939AF80030002B85D1DC
:10456000BBF80C305B060AD40D9821B0BDE8F08F83
:104570000498594600F010FC00283FF469AF4FF052
:10458000FF30F2E7B9EB0A08EAD00AF1FF35CDF8BF
:104590001490A946049D01E0A0453ED94C465A46D8
:1045A00019F8011F2846FFF7F7FE02340130A4EB8B
:1045B0000A04F1D1D4E7A1F13002092A88BFCA4622
:1045C0009CD80B9B00E00134217803EB830302EBC2
:1045D0004303A1F13002092AF5D92E290B93A246F3
:1045E0008ED19AF801102A292FD1079B9AF8021030
:1045F0001A6809920433002A0AF102000793B8BF2F
:104600004FF0FF338246B8BF099379E7079B073322
:1046100023F00703083307939AE70D99DDF8149008
:10462000414499F800300D912FE7494243F00203CD
:104630000B91089360E707AA0092144B04985A461E
:1046400008A9FFF763FD03907FE7A1F13002002383
:10465000092A09930AF1010A3FF652AF1AF8011F1D
:1046600003EB830302EB4303A1F13002092AF5D9DE
:10467000099345E7FFF748F9E0E600BF3815010860
:10468000401501084415010800000000D54300084A
:1046900010B4054C8446134620685DF8044B0A4666
:1046A0006146FFF7BFBE00BF00000020F8B50D4611
:1046B0001446064610B1036A002B37D0A389A269BD
:1046C000A2601A0719D52369BBB122686169D31AA0
:1046D000EDB299422F4620DD0133A1680139A16076
:1046E000511C2160157062699A420DD0A389DB07C5
:1046F00001D50A2D08D03846F8BD2146304600F0D5
:104700004BFB38B92369E0E721463046FFF7BEF995
:104710000028F0D04FF0FF37EDE721463046FFF795
:10472000B5F90028F6D122680123D6E7FFF7ECF8A7
:10473000C4E700BF10B4044C03460A4620685DF885
:10474000044B1946FFF7B2BF0000002038B5074DF3
:104750000022044608462A600BF000FF431C00D0EC
:1047600038BD2B68002BFBD0236038BD38030020F8
:1047700010B50C46B1F90E1000F070FB002803DBF9
:10478000636D0344636510BDA38923F48053A38143
:1047900010BD00BF002070472DE9F0410C46B1F973
:1047A0000C101F46CB05054616460BD421F480514C
:1047B000A1813B46B4F90E1032462846BDE8F041CF
:1047C00000F002BCB4F90E100223002200F0E6FB58
:1047D000B4F90C10EAE700BF10B50C46B1F90E10A1
:1047E00000F0DCFBB4F90C30421C0EBF23F4805304
:1047F00043F480536065A38110BD00BFB1F90E1072
:1048000000F0B8BA51F8043C181F002BBCBF0B587D
:10481000C01870479368002B00F0F8802DE9F04F26
:10482000B1F90CC01CF0080F83B0904681460C46CD
:1048300031D00B697BB31CF00207D8F8006038D088
:104840000027D4F828B0216ADFF8C4A23D465545B8
:104850002B463A4628BF53464846C5B1D84700289C
:1048600040F3CA80D8F808301B1A07442D1AC8F83C
:104870000830002B00F0B68055452B46D4F828B000
:10488000216A28BF53463A464846002DE6D1D6E96C
:1048900000750836DBE72146484600F07DFA00281F
:1048A00040F0AF80B4F90CC0D8F800601CF00207EB
:1048B000C6D11CF0010A63D12368A1685746184687
:1048C0008B46002F58D01CF4007F00F0B580B94211
:1048D0000A4600F2E1801CF4906F2FD021696269D2
:1048E0005D1A02EB420202EBD2726B1C52103B4487
:1048F000934292BF93469B461A461CF4806F00F089
:10490000EA8011464846FFF73BF9002800F0F9809D
:104910002A4621690090FDF70BFBA289009B22F437
:10492000906242F08002A2815819ABEB0505C4F8F1
:1049300014B02361A5602060BB463A465146009200
:10494000FFF7FCF9A1682368009AA1EB0B011A4458
:104950003D46A16022600027D8F808305B1BAA44BE
:10496000C8F80830002B3DD02368A168B4F90CC00A
:1049700018468B46002FA6D1D6E900A708369EE739
:104980003846BB463D460097002D41D0002846D012
:10499000009A2068A168D4E90473AA4228BF2A4675
:1049A000B84204D901EB030A524500F385809342D3
:1049B00075DC216AA76A5A464846B847B0F1000A32
:1049C0001ADD009BB3EB0A0300930FD00120D8F847
:1049D0000830A3EB0A03D344A5EB0A05C8F8083056
:1049E000002BD1D1002003B0BDE8F08F214648460E
:1049F000FFF74CF80028EAD0B4F90C3043F040033C
:104A0000A3814FF0FF3003B0BDE8F08F0020704766
:104A1000756833460836002DFAD0D3F800B02A4620
:104A20000A215846FFF72CFA002867D00130A0EB86
:104A30000B0300931A46ACE722699A4214D36269C9
:104A4000BA4211D86FF00043BB4228BF3B46A56A6B
:104A500093FBF2F3216A02FB03F348465246A84750
:104A6000051EC9DD7F1B77E7B94228BF39460D46D1
:104A700018460A465146FFF761F9A1682368491BA9
:104A80002B44A16023600029ECD121464846FEF763
:104A9000FDFF0028E6D0AFE7BB463A464EE7594651
:104AA0000192FFF74BF9019AA3689B1AA360236850
:104AB00013442360924684E759465246FFF73EF975
:104AC00023685344236021464846FEF7DFFF002851
:104AD0003FF477AF90E74846FFF754FA03460028C3
:104AE0007FF422AF21694846FFF7CAF8B4F90C30C9
:104AF0000C22C9F8002023F080037FE76A1C009293
:104B000047E70C22B4F90C30C9F8002076E700BF63
:104B100000FCFF7F38B5C46B0CB1002038BD80218C
:104B20000546FFF72DF80246E86330B1031F7C32DB
:104B300043F8044F9342FBD1EFE74FF0FF3038BD0D
:104B400030B51F2983B0054608D8C36B0C4653B156
:104B500053F8240043F8242003B030BD162303602B
:104B60004FF0FF30F8E780210192FFF709F8019A32
:104B7000E86303460028F3D0011F00F17C05002004
:104B800041F8040FA942FBD1E2E700BF1F2938B565
:104B900005461ED8C26B0C466AB152F8213053B19B
:104BA000012B06D0591C10D0002142F824102046B9
:104BB0009847002038BD284600F044FA22460146B6
:104BC0002846BDE8384000F027BA162303600120CC
:104BD00038BD162303604FF0FF3038BD1F292AD897
:104BE00038B5C36B0C460546A3B153F8242003EB3C
:104BF00084034AB1511C0BD0012A07D0002520465E
:104C00001D609047284638BD012038BD032038BDBF
:104C1000022038BD8021FEF7B3FF0346E86338B1B8
:104C2000021F00217C3042F8041F8242FBD1DCE7E6
:104C30004FF0FF3038BD4FF0FF30704738B5134BA1
:104C40001F281D681DD8EA6B044662B152F8203057
:104C50004BB1012B05D0591C0FD0002142F8201078
:104C60009847002038BD284600F0ECF9224601465E
:104C70002846BDE8384000F0CFB916232B6001204C
:104C800038BD16232B604FF0FF3038BD00000020E8
:104C9000114B1F2870B51E6808D8F36B04460D46EB
:104CA0004BB153F8240043F8245070BD16233360F1
:104CB0004FF0FF3070BD80213046FEF761FF0346A4
:104CC000F0630028F4D0021F00217C3042F8041F5A
:104CD0008242FBD1E5E700BF0000002038B50B4B56
:104CE0001D68EC6B0CB1002038BD80212846FEF712
:104CF00047FFE86338B1031F00F17C0243F8044F1B
:104D00009342FBD1EFE74FF0FF3038BD00000020A9
:104D100038B5174B1F281D6826D80446E86BA0B18C
:104D200050F8243000EB84004BB15A1C0BD0012BFF
:104D300007D00025056020469847284638BD012049
:104D400038BD032038BD022038BD80212846FEF73B
:104D500017FFE86340B1031F00F17C01002243F814
:104D6000042F8B42FBD1DBE74FF0FF3038BD00BF93
:104D70000000002038B5074D0022044608462A608E
:104D80000BF03EFC431C00D038BD2B68002BFBD041
:104D9000236038BD3803002038B52F4B1B6805460B
:104DA0000C4613B11A6A002A4BD0B4F90C3018071C
:104DB0001CD5226922B313F0010107D061690020DC
:104DC0004942A060A1613AB1002038BD980758BFA0
:104DD0006169A160002AF7D1190658BF1046F4D5C1
:104DE00043F04003A3814FF0FF3038BDD9062CD5E6
:104DF0005A0712D4226943F00803A381002ADAD1AA
:104E000003F42071B1F5007FD5D02146284600F08B
:104E10003BF8B4F90C302269CDE7616B51B104F174
:104E20004402914204D02846FEF72AFFB4F90C3020
:104E30000022626322690021C4E9002123F02403D7
:104E4000D9E71846FEF760FDAFE7092243F04003BB
:104E50002A60A381C7E700BF0000002038B50C46D8
:104E6000084D8446114620461A4600232B606446AE
:104E70000BF0A8FB431C00D038BD2B68002BFBD0E7
:104E8000236038BD3803002070B5B1F90C300C46F2
:104E9000990796B007D504F147030122C4E904320B
:104EA000236016B070BDB4F90E100029054629DB49
:104EB0006A4600F0C9F8002822DB4FF480612846DA
:104EC000019EFEF75DFE88B3A389206043F0800356
:104ED00006F47046A381B6F5005F4FF48063C4E921
:104EE0000403DED1B4F90E10284600F083F8002840
:104EF000D7D0A38923F0030343F00103A381D0E7B4
:104F0000B4F90C3013F0800F14BF40264FF48066C4
:104F100031462846FEF734FE40B1A389206043F0B5
:104F20008003C4E90406A38116B070BDB4F90C3047
:104F30009A05B6D423F0030304F1470243F00203B9
:104F40000121C4E90421A3812260AAE770B50C46BF
:104F5000B1F90E10002996B015461E460FDB6A46C1
:104F600000F072F800280ADB019B03F47043A3F5FC
:104F70000053B3FA83F34FF480625B0908E0A2891F
:104F800012F0800F4FF0000314BF40224FF48062F4
:104F9000002033602A6016B070BD00BF38B50C46E3
:104FA000084D8446114620461A4600232B6064466D
:104FB0000BF030FB431C00D038BD2B68002BFBD01E
:104FC000236038BD3803002038B50C46084D8446B0
:104FD000114620461A4600232B6064460BF002FB64
:104FE000431C00D038BD2B68002BFBD0236038BD9C
:104FF0003803002038B5074D0022044608462A60D1
:105000000BF006FB431C00D038BD2B68002BFBD0F7
:10501000236038BD3803002070B50C46084D0346A8
:105020000026204611461C462E600BF0BDFA431C9C
:1050300000D070BD2B68002BFBD0236070BD00BF7B
:10504000380300200BF0AEBA70B50C46084D03468D
:105050000026204611461C462E600BF0D4FA431C55
:1050600000D070BD2B68002BFBD0236070BD00BF4B
:105070003803002081F0004102E000BF83F00043CC
:1050800030B54FEA41044FEA430594EA050F08BFE3
:1050900090EA020F1FBF54EA000C55EA020C7FEAA7
:1050A000645C7FEA655C00F0E2804FEA5454D4EB24
:1050B0005555B8BF6D420CDD2C4480EA020281EAEE
:1050C000030382EA000083EA010180EA020281EA26
:1050D0000303362D88BF30BD11F0004F4FEA013178
:1050E0004FF4801C4CEA113102D0404261EB410187
:1050F00013F0004F4FEA03334CEA133302D052420D
:1051000063EB430394EA050F00F0A780A4F10104C8
:10511000D5F1200E0DDB02FA0EFC22FA05F2801802
:1051200041F1000103FA0EF2801843FA05F35941E8
:105130000EE0A5F120050EF1200E012A03FA0EFC67
:1051400028BF4CF0020C43FA05F3C01851EBE37191
:1051500001F0004507D54FF0000EDCF1000C7EEBAE
:1051600000006EEB0101B1F5801F1BD3B1F5001FEC
:105170000CD349085FEA30004FEA3C0C04F101040B
:105180004FEA445212F5800F80F09A80BCF1004F34
:1051900008BF5FEA500C50F1000041EB045141EAB6
:1051A000050130BD5FEA4C0C404141EB0101013C7F
:1051B00028BFB1F5801FE9D291F0000F04BF01466E
:1051C0000020B1FA81F308BF2033A3F10B03B3F140
:1051D00020020CDA0C3208DD02F1140CC2F10C02D0
:1051E00001FA0CF021FA02F10CE002F11402D8BF2E
:1051F000C2F1200C01FA02F120FA0CFCDCBF41EAFA
:105200000C019040E41AA2BF01EB0451294330BDC8
:105210006FEA04041F3C1CDA0C340EDC04F11404A5
:10522000C4F1200220FA04F001FA02F340EA03007C
:1052300021FA04F345EA030130BDC4F10C04C4F1C2
:10524000200220FA02F001FA04F340EA03002946A2
:1052500030BD21FA04F0294630BD94F0000F83F4EC
:10526000801306BF81F480110134013D4EE77FEACF
:10527000645C18BF7FEA655C29D094EA050F08BF1B
:1052800090EA020F05D054EA000C04BF19461046FC
:1052900030BD91EA030F1EBF0021002030BD5FEA40
:1052A000545C05D14000494128BF41F0004130BD68
:1052B00014F580043CBF01F5801130BD01F00045BC
:1052C00045F0FE4141F470014FF0000030BD7FEA2F
:1052D000645C1ABF194610467FEA655C1CBF0B462A
:1052E000024650EA013406BF52EA033591EA030F41
:1052F00041F4002130BD00BF90F0000F04BF002139
:10530000704730B54FF4806404F132044FF000056B
:105310004FF0000150E700BF90F0000F04BF0021E4
:10532000704730B54FF4806404F1320410F000454A
:1053300048BF40424FF000013EE700BF42004FEA45
:10534000E2014FEA31014FEA02701FBF12F07F43C2
:1053500093F07F4F81F06051704732F07F4208BF79
:10536000704793F07F4F04BF41F40021704730B580
:105370004FF4607401F0004521F000411CE700BFCC
:1053800050EA010208BF704730B54FF000050AE04F
:1053900050EA010208BF704730B511F0004502D550
:1053A000404261EB41014FF4806404F132045FEA52
:1053B000915C3FF4D8AE4FF003025FEADC0C18BFFB
:1053C00003325FEADC0C18BF033202EBDC02C2F1ED
:1053D000200300FA03FC20FA02F001FA03FE40EA7F
:1053E0000E0021FA02F11444BDE600BF53B94AB9D8
:1053F000002908BF00281CBF4FF0FF314FF0FF30DD
:1054000000F0A4B9ADF1080C6DE904CE00F040F84D
:10541000DDF804E0DDE9022304B0704708B5024678
:105420000B4643EC172BB5EEC07BF1EE10FA03D41C
:10543000BDE8084000F00CB8B1EE477B51EC170B0B
:1054400000F006F8404261EB410108BD0000000099
:105450009FED0B6B41EC170B9FED0B5B27EE066B83
:10546000BCEEC66BB8EE464BA4EE457BFCEEC77BAC
:1054700016EE101A17EE900A704700BFAFF30080C7
:10548000000000000000F03D000000000000F041BE
:105490002DE9F047089D0E4604460F46002B4AD1E1
:1054A00094468C45B2FA82F260D942B1C2F120032F
:1054B000974020FA03F30CFA02FC1F4394404FEA92
:1054C0001C4E1FFA8CF6B7FBFEF1230C0EFB117776
:1054D00043EA074301FB06F098420AD91CEB030399
:1054E00001F1FF3780F01581984240F212810239B4
:1054F00063441B1AA4B2B3FBFEF00EFB103344EA64
:10550000034400FB06F6A6420AD91CEB040400F192
:10551000FF3380F00081A64240F2FD8064440238EF
:1055200040EA0140A41B00211DB1D4400023C5E97D
:105530000043BDE8F0878B4205D90DB1C5E90001F4
:1055400000210846F5E7B3FA83F1002946D1B342BA
:1055500002D3824200F2F580841A66EB0302012036
:105560001746002DE5D0C5E90047E2E7002A40F0E4
:105570009380A1EB0C034FEA1C471FFA8CFE01211C
:10558000B3FBF7F607FB1630230C43EA00430EFB90
:1055900006F0984208D91CEB030306F1FF3802D24B
:1055A000984200F2D08046461B1AA4B2B3FBF7F033
:1055B00007FB103344EA03440EFB00FEA64508D95E
:1055C0001CEB040400F1FF3302D2A64500F2B680C2
:1055D0001846A4EB0E0440EA0640A5E7C1F12007F7
:1055E0008B4022FA07FC4CEA030C06FA01FE20FA73
:1055F00007F426FA07F344EA0E0400FA01F84FEA2A
:105600001C404FEA1449B3FBF0FE1FFA8CF600FB76
:105610001E3349EA03430EFB06F9994502FA01F2EB
:105620000BD91CEB03030EF1FF3A80F085809945FE
:1056300040F28280AEF1020E6344A3EB0909A4B2EA
:10564000B9FBF0F300FB139944EA094403FB06F6A7
:10565000A64208D91CEB040403F1FF3068D2A6422D
:1056600066D9023B644443EA0E40A41BA0FB02E659
:10567000B4427346B14652D34FD05DB1B8EB03028A
:1056800064EB090404FA07F722FA01F31F43CC4044
:10569000C5E9007400214CE7C2F1200120FA01F3B2
:1056A0000CFA02FC26FA01F1964033434FEA1C47FC
:1056B0001FFA8CFEB1FBF7F007FB1016190C41EA3C
:1056C000064100FB0EF68E4204FA02F408D91CEBE8
:1056D000010100F1FF382DD28E422BD902386144EE
:1056E000891B9BB2B1FBF7F607FB161143EA014396
:1056F00006FB0EF1994208D91CEB030306F1FF38B3
:1057000014D2994212D9023E63445B1A46EA004120
:1057100036E73946EDE6184602E7F045ADD2BEEB76
:10572000020366EB0C060138B146A6E74646ECE7F5
:10573000034698E74046D3E7D6467EE764440238FE
:1057400047E708460DE7023E63442DE7704700BF78
:1057500000B500F00700C0F1070CBCF1040F28BF32
:105760004FF0040C031D062B0FD9C31E4FF0FF3E54
:105770000EFA0CF021EA000199400EFA03FE22EA2B
:105780000E0241EA02005DF804FB0023EEE7000090
:10579000064B074A1A6000225A609A60DA604FF49A
:1057A000006119615A6114229A6170471004002047
:1057B000002C014000B583B00D4B1A6B42F48002FF
:1057C0001A631B6B03F480030193019B094BD86898
:1057D00000221146C0F30220FFF7BAFF0001C0B259
:1057E000054B83F8460340229A6003B05DF804FB42
:1057F0000038024000ED00E000E100E02DE9F04F4C
:105800008FB0002409940A940B940C940D94984B37
:105810001A6B42F020021A631A6B02F02002019206
:10582000019A1A6B42F080021A631A6B02F080022E
:105830000292029A1A6B42F004021A631A6B02F087
:1058400004020392039A1A6B42F001021A631A6B64
:1058500002F001020492049A1A6B42F002021A63E7
:105860001A6B02F002020592059A1A6B42F01002BE
:105870001A631A6B02F010020692069A1A6B42F033
:1058800008021A631A6B02F008020792079A1A6B51
:1058900042F040021A631B6B03F040030893089B1D
:1058A000DFF8DC8122464FF4C861404606F0FBFD7C
:1058B000DFF8D0912246B821484606F0F4FD0122D7
:1058C0004021484606F0EFFDDFF8BCA122464B21FF
:1058D000504606F0E8FD674E01224FF480713046D5
:1058E00006F0E1FD22464FF44061304606F0DBFD54
:1058F00001220C21304606F0D6FD01224FF48041F2
:10590000304606F0D0FDDFF884B122464FF44F61F7
:10591000584606F0C8FD584F01224FF480513846D2
:1059200006F0C1FD01224FF48051584606F0BBFD40
:1059300022464FF4C171384606F0B5FD01224FF4FE
:105940000061384606F0AFFD01224FF400513846A1
:1059500006F0A9FD22464FF47E41484806F0A3FD1B
:10596000182309930A9401250B9509A9404606F0CE
:1059700091FC4FF4C86309930A950B940C9409A900
:10598000404606F087FCF02309930A950B940C948B
:1059900009A9484606F07EFC082309930A950B9452
:1059A00003230C9309A9484606F074FC4B23099382
:1059B0000A950B940C9409A9504606F06BFC4FF421
:1059C000F04309930A940B9409A9404606F062FC3F
:1059D0004FF4506309930A950B940C9409A930462F
:1059E00006F058FC0C23099311230A930B940C9492
:1059F00009A9304606F04EFC4FF4804309930A95FE
:105A00000B9403230C9309A9304606F043FC41F69E
:105A1000F04309930A950B940C9409A9584606F093
:105A200039FC43F6821309930A950B940C9409A947
:105A3000384606F02FFC4FF4807309930A940B94B8
:105A400009A9504606F026FC09950A940B9409A969
:105A5000384606F01FFC4FF47E4309930A950B94D9
:105A60000C9409A9054806F015FC0FB0BDE8F08FAD
:105A70000038024000100240000C024000180240B2
:105A800000140240000802400000024000040240EE
:105A90002DE9F04192B02822002108A8FCF722F954
:105AA00000240294039404940594069407942A4BCA
:105AB0005A6C42F400525A645A6C02F40052019239
:105AC000019A1A6B42F010021A631B6B03F0100369
:105AD0000093009B4FF480530293022503954FF0EF
:105AE0000308CDF81080052707971C4E02A9304601
:105AF00007F045F84FF4005302930395CDF810805A
:105B000005940694079702A9304607F038F84FF439
:105B1000806308934FF4827309934FF470630A9380
:105B20000B950C944FF400730D9318230E930F9460
:105B30001094072311930A4C08A9204608F03CF85A
:105B4000636823F010036360636823F008036360F5
:105B500012B0BDE8F08100BF0038024000100240E2
:105B6000003401402DE9F04192B02822002108A81C
:105B7000FCF7B8F800240294039404940594069466
:105B800007942F4B1A6C42F480421A641A6C02F488
:105B900080420192019A1A6B42F002021A631B6B57
:105BA00003F002030093009B4FF4005302934FF065
:105BB0000208CDF80C800327049705260796214D8F
:105BC00002A9284606F0DBFF4FF480430293CDF88C
:105BD0000C80049705940694079602A9284606F0BF
:105BE000CEFF4FF400430293CDF80C800497059448
:105BF0000694079602A9284606F0C1FF08944FF4C0
:105C0000827309934FF470630A930B940C944FF4CE
:105C100000730D9310230E930F9410940723119388
:105C2000094C08A9204607F0C7FF636823F010035A
:105C30006360636823F00803636012B0BDE8F0811D
:105C40000038024000040240003800402DE9F041D5
:105C500092B02822002108A8FCF744F800240294FE
:105C600003940494059406940794294B5A6C42F4C7
:105C700080125A645A6C02F480120192019A1A6BD3
:105C800042F020021A631B6B03F020030093009B79
:105C900080230293022503954FF00308CDF810806E
:105CA000052707971B4E02A9304606F068FF4FF400
:105CB000807302930395CDF810800594069407979E
:105CC00002A9304606F05BFF4FF4806308934FF45F
:105CD000827309934FF470630A930B950C944FF4FD
:105CE00000730D9318230E930F94109407231193B0
:105CF000094C08A9204607F05FFF636823F01003F2
:105D00006360636823F00803636012B0BDE8F0814C
:105D10000038024000140240005001402DE9F041DB
:105D200092B02822002108A8FBF7DCFF002402948F
:105D300003940494059406940794294B5A6C42F4F6
:105D400000125A645A6C02F400120192019A1A6B02
:105D500042F001021A631B6B03F001030093009BE6
:105D600020230293022503954FF00308CDF81080FD
:105D7000082707971B4E0DEB0701304606F0FFFE84
:105D8000802302930395CDF810800594069407971D
:105D90000DEB0701304606F0F2FE08944FF48273D3
:105DA00009934FF470630A930B9501230C934FF4FE
:105DB00000730D9318230E930F94109407231193DF
:105DC000094C08A9204607F0F7FE636823F010038A
:105DD0006360636823F00803636012B0BDE8F0817C
:105DE00000380240000002400054014010B586B067
:105DF0000024019402940394049405941D4B1A6C9E
:105E000042F001021A641B6C03F001030093009B33
:105E1000194BD86822462146C0F30220FFF798FCB0
:105E20000001C0B2154B83F81C034FF080521A607A
:105E30004FF47A73ADF804300294114B0393049439
:105E400001A94FF0804008F06DFB4FF080431A68C5
:105E500022F080021A6099680A4A0A409A605A68D9
:105E600022F070025A609A6822F080029A6006B0AE
:105E700010BD00BF0038024000ED00E000E100E08E
:105E800040D10C00F8BFFEFF10B586B0002401948D
:105E900002940394049405941B4B1A6C42F008027C
:105EA0001A641B6C03F008030093009B174BD8681F
:105EB00022462146C0F30220FFF74AFC0001C0B28F
:105EC000134B83F832034FF480225A602D23ADF830
:105ED000043002947C23039304940E4C01A92046C1
:105EE00008F020FB236823F080032360A2680A4B9C
:105EF0001340A360636823F070036360A36823F01A
:105F00008003A36006B010BD0038024000ED00E041
:105F100000E100E0000C0040F8BFFEFF10B586B0C5
:105F20000024019402940394049405941A4B1A6C6F
:105F300042F020021A641B6C03F020030093009BC4
:105F4000164BD86822462146C0F30220FFF700FC1A
:105F50000001C0B2124B83F837034FF400025A60BD
:105F600040F29733ADF804300294632303930D4C51
:105F700001A9204608F0D6FA236823F080032360A5
:105F8000636823F0700343F010036360A36823F099
:105F90008003A36006B010BD0038024000ED00E0B1
:105FA00000E100E00014004010B586B00024019428
:105FB00002940394049405941A4B1A6C42F0100254
:105FC0001A641B6C03F010030093009B164BD868F7
:105FD00022462146C0F30220FFF7BAFB0001C0B2FF
:105FE000124B83F836034FF480025A604BF2AF3302
:105FF000ADF804300294132303930D4C01A92046FD
:1060000008F090FA236823F080032360636823F08C
:10601000700343F010036360A36823F08003A36060
:1060200006B010BD0038024000ED00E000E100E0E5
:106030000010004072B6FEE700B585B00023009363
:106040000193029303932B482B4A02604FF4403292
:106050004260836001220261836180F82030C36264
:1060600026498162C3600521C16180F830304261F8
:1060700004F0E2FF002831D10923009301230193AA
:106080000723029369461B4805F0BEF940BB08236D
:106090000093022301936946164805F0B5F908BB41
:1060A00002230093032301936946124805F0ACF9DB
:1060B000D0B90A2300930423019369460D4805F0E3
:1060C000A3F998B90B230093052301936946094866
:1060D00005F09AF960B905B05DF804FBFFF7AAFF77
:1060E000FFF7A8FFFFF7A6FFFFF7A4FFFFF7A2FF48
:1060F000FFF7A0FFDC040020002001400100000F9A
:1061000000B585B0002300930193029303931448D4
:10611000144A02604FF4403242608360036183613D
:1061200080F82030C362104A8262C3600122C261DB
:1061300080F83030426104F07FFF68B90F2300938C
:1061400001230193072302936946054805F05CF992
:1061500020B905B05DF804FBFFF76CFFFFF76AFF9D
:1061600094040020002201400100000F2DE9F041BD
:10617000B4B000212D912E912F9130913191329117
:1061800033912791289129912A912B912C9190223A
:1061900003A8FBF7A7FD4023039303A805F07AFDAE
:1061A000002840F09E80504B5A6C42F010025A6416
:1061B0005A6C02F010020292029A1A6B42F001022B
:1061C0001A631B6B03F001030193019B4FF40073EF
:1061D00027934FF00208CDF8A080032729970024C9
:1061E0002A942B9407262C96404D27A9284606F082
:1061F000C6FC4FF480632793CDF8A08029972A949A
:106200002B942C9627A9284606F0B9FC384BD3F8D6
:10621000B82022F0F05242F00062C3F8B820D3F860
:10622000B82022F0C00242F04002C3F8B820D3F8F0
:10623000B82042F44032C3F8B820D3F8B82022F492
:106240009072C3F8B820D3F8B82022F40072C3F8D3
:10625000B820D3F8B82042F48062C3F8B820D3F84D
:10626000B82022F4C052C3F8B820D3F8B82022F4E2
:10627000C042C3F8B820D3F8CC2022F00402C3F8FF
:10628000CC201C4BD86822462146C0F30220FFF7E1
:106290005FFA0001C0B2184B83F8250320225A6030
:1062A0004FF4E1332D932E942F9430940C2331939B
:1062B0003294339404F1804404F588342DA92046A7
:1062C00008F0D0F9636823F490436360A36823F077
:1062D0002A03A360236843F00103236034B0BDE8C0
:1062E000F081FFF7A7FE00BF003802400000024027
:1062F0000064024000ED00E000E100E008B50B485A
:106300000B4B03604FF4E133436000238360C360B1
:1063100003610C2242618361C361036243620AF03C
:1063200054FC00B908BDFFF785FE00BF3C03002008
:10633000007C004010B596B000241294139414947D
:1063400015940B940C940D940E940F941094119436
:106350002C2221466846FBF7C5FC2548254B0360E7
:10636000446084600823C36004614461846107F071
:1063700013FE002832D14FF48053129312A91C4807
:1063800007F04CFF00282BD1194807F035FE48BB19
:1063900060230B9304230C9300220D920F920BA900
:1063A000134807F091FEF8B900230093019302937C
:1063B000039304934FF400520592069307934FF012
:1063C0000072089209930A936946094808F062F836
:1063D00060B9074800F0DEFB16B010BDFFF72AFEDB
:1063E000FFF728FEFFF726FEFFF724FEFFF722FE49
:1063F000C40300200000014000B595B03422002104
:1064000007A8FBF76FFC0023029303930493059303
:106410000693244B1A6C42F080521A641B6C03F0F2
:1064200080530093009B204B1A6842F440421A604C
:106430001B6803F440430193019B012307934FF42E
:106440008033089302230D934FF480020E92192299
:106450000F924FF4B8721092119308221292139374
:1064600007A805F0C5F8B0B906F02CF8A8B90F23B5
:10647000029302230393002304934FF4A053059344
:106480004FF480530693062102A805F027FB30B98C
:1064900015B05DF804FBFFF7CDFDFFF7CBFDFFF76F
:1064A000C9FD00BF003802400070004008B506F08A
:1064B000E3F8FFF7A1FFFFF7A1F9FFF77BF9FFF77B
:1064C000E7FA00F01DF9FFF791FCFFF7DDFCFFF79D
:1064D000B3FDFFF715FEFFF745FBFFF7B7FBFFF72F
:1064E0001DFCFFF743FEFFF753F9FFF717FDFFF71A
:1064F0005BFDFFF703FFFFF71DFF01F03BFD01F020
:1065000097FDFCE700B583B0009313460A460146A9
:10651000034806F03FFF00B1012003B05DF804FB23
:106520001004002000B583B0009313460A460146CC
:10653000034807F053F800B1012003B05DF804FBF5
:106540001004002008B5034807F025FB043818BFE5
:10655000012008BD1004002008B50146014807F0DD
:1065600008FB08BD1004002000B583B001238DF89E
:10657000073000F0D5F810B900238DF807309DF8EA
:10658000070003B05DF804FB10B5FFF7EDFF134BF8
:106590001870012212490A7012490A70124A002129
:1065A00011601B78DBB2012B03D002200F4B187057
:1065B00010BD0F4C002323617623A361204607F012
:1065C000BDFA074B1870A26B074B1A6010B9054B48
:1065D00000221A70054B1870EAE700BF280500205A
:1065E000C9010020C801002024050020CA010020A4
:1065F0001004002008B5074B01221A70FFF7A2FF14
:1066000020B9044A137803F0FE031370014B187885
:1066100008BD00BFCD01002010B50446094B012282
:106620001A70FFF7B1FF30B1064A1378DBB20649A2
:106630000B70107810BD2046FFF7DCFF014B18707F
:10664000F2E700BFCD010020CC01002008B5FFF724
:10665000D1FF024B1870187808BD00BFCB01002095
:1066600008B5084611461A464FF0FF33FFF74AFFB8
:1066700030B9FFF767FF03460028FAD1184608BD76
:106680000123FBE708B5084611461A464FF0FF33D1
:10669000FFF748FF30B9FFF755FF03460028FAD14E
:1066A000184608BD0123FBE730B589B0134B1878B5
:1066B00010F001041BD1154603291CD8DFE801F0B6
:1066C00002040A100C4613E06846FFF745FF069BDC
:1066D0002B600DE06846FFF73FFF079B2B8007E02C
:1066E0006846FFF739FF079B5B0A2B6000E0032435
:1066F000204609B030BD0424FAE700BFCD010020D8
:1067000008B50349034809F023FF034B187008BD7F
:106710006015002018100108641500200020704743
:1067200008B50121034805F0B7FE08B9012008BDEE
:106730000020FCE7000C0240FEE7FEE7FEE7FEE774
:10674000FEE770477047704708B505F0A1FF08BD28
:1067500008B5034804F0BDFD024804F0BAFD08BDC9
:10676000DC0400209404002070477047704700004C
:1067700008B52B4BDB6913F0010F2AD00123284AFF
:106780001362274AD26912F0020F03D0244B02226F
:106790001A620123224AD26912F0040F03D0204B5F
:1067A00004221A6201231E4AD26912F0080F12D184
:1067B000A3B91B4BDB6913F0200F19D0184B1B68D2
:1067C00013F0200F14D0164B586AC0B201F06AFCC7
:1067D0000DE00023D5E7124B08221A62104BDB694B
:1067E00013F0200F01D00E4B5B6A01F09BFC08BD3B
:1067F0000B4BDB6913F0400FF9D0094B1B6813F00A
:10680000400FF4D0064B40221A62054A52E8003F7E
:1068100023F0400342E800310029F6D1E7E700BF4A
:10682000001001407047000008B5064B1B6913F0CB
:10683000010F05D0034B6FF001021A6101F08CFCCF
:1068400008BD00BF000C004008B5064B1B6913F0E3
:10685000010F05D0034B6FF001021A6101F06AFCD1
:1068600008BD00BF0010004008B5064B1B6913F0BF
:10687000010F05D0034B6FF001021A6101F064FCB7
:1068800008BD00BF0014004008B50B4B5B6813F057
:10689000006F09D1084B5B6813F0007F03D0064BF3
:1068A0004FF00072DA6008BD034B4FF00062DA600F
:1068B00001F056FCF7E700BF0064024082B00A4BCB
:1068C0001A6C42F080521A641A6C02F080520092E4
:1068D000009A5A6C42F480425A645B6C03F4804321
:1068E0000193019B02B070470038024030B58DB073
:1068F00000230793089309930A930B930368384A7C
:10690000934204D0374A934246D00DB030BD364B47
:106910005A6C42F480725A645A6C02F4807201928A
:10692000019A1A6B42F004021A631A6B02F0040215
:106930000292029A1A6B42F001021A631A6B02F079
:1069400001020392039A1A6B42F002021A631B6B54
:1069500003F002030493049B03240794089407A9FB
:10696000224805F097FC0423079308940025099515
:1069700007A91F4805F08EFC07940894099507A9FC
:106980001C4805F087FC2A462946122005F01CFE0B
:10699000122005F029FEB8E7134B5A6C42F48062CE
:1069A0005A645A6C02F480620592059A1A6B42F09E
:1069B00020021A631B6B03F020030693069B20231F
:1069C00007930323089307A90B4805F063FC0022F3
:1069D0001146122005F0F8FD122005F005FE94E79F
:1069E000002001400022014000380240000802401F
:1069F000000002400004024000140240F0B5ADB0B7
:106A0000044600212791289129912A912B919022C7
:106A100003A8FBF767F92268224B9A4201D02DB0F8
:106A2000F0BD4FF42003039303A805F033F90028C9
:106A300035D11D4B5A6C42F400625A645A6C02F410
:106A400000620092009A1A6B42F004021A631A6BF9
:106A500002F004020192019A1A6B42F008021A63D2
:106A60001B6B03F008030293029B4FF4F853279328
:106A7000022728970026299603252A950C242B9473
:106A800027A90A4805F006FC04232793289729968E
:106A90002A952B9427A9064805F0FCFBBFE7FFF7D2
:106AA000C9FAC6E7002C0140003802400008024045
:106AB000000C024000B587B00368304A93421ED0F4
:106AC0002F4A934228D02F4A934230D02E4A9342E5
:106AD00040D02E4A93421CD12D4B5A6C42F4802256
:106AE0005A645B6C03F480230593059B00221146D6
:106AF0001A2005F069FD1A2005F076FD09E0244B07
:106B00001A6C42F004021A641B6C03F00403019334
:106B1000019B07B05DF804FB1D4B5A6C42F001026B
:106B20005A645B6C03F001030293029BF1E7184B7C
:106B30005A6C42F002025A645B6C03F00203039346
:106B4000039B002211462C2005F03EFD2C2005F071
:106B50004BFDDEE70E4B5A6C42F400325A645B6C1C
:106B600003F400330493049B00221146192005F01E
:106B70002BFD192005F038FDCBE700BF00080040D1
:106B80000000014000040140004401400048014071
:106B90000038024000B589B00023039304930593A5
:106BA000069307930368274A934208D0264A9342E4
:106BB0001AD0264A93422FD009B05DF804FB244B2B
:106BC0001A6B42F002021A631B6B03F0020300937C
:106BD000009B4FF48073039302230493079303A94C
:106BE0001C4805F057FBE7E7194B1A6B42F01002FF
:106BF0001A631B6B03F010030193019B4FF40073A6
:106C0000039302230493032306930123079303A909
:106C1000114805F03FFBCFE70D4B1A6B42F0020223
:106C20001A631B6B03F002030293029B4FF4007381
:106C30000393022304930323079303A9054805F054
:106C400029FBB9E70008004000000140004801406E
:106C500000380240000402400010024010B5ACB001
:106C6000044600212791289129912A912B91902265
:106C700003A8FBF737F82268174B9A4201D02CB0D3
:106C800010BD4FF40053039303A805F003F800BBB5
:106C9000124B1A6C42F000421A641A6C02F0004265
:106CA0000192019A1A6B42F010021A631B6B03F0F7
:106CB00010030293029B03232793022228920022AF
:106CC00029922A9308232B9327A9054805F0E2FA75
:106CD000D5E7FFF7AFF9DBE7007C00400038024062
:106CE0000010024018B101280ED0002070470D4B53
:106CF00093F8B33023B10B4B93F8B53013B9704709
:106D00000020704701207047064B93F8B4302BB138
:106D1000044B93F8B6301BB9002070470020704731
:106D20000120704768150020B0F57A7F05DB4DF62D
:106D3000E053984204DC80B270474FF47A70704799
:106D40004DF6E050704702460B46002918BF002858
:106D50000CBF012000201AD01168196092889A8017
:106D60005A78012A14D81A786AB15A88323A92B2FB
:106D700040F29E718A420BD89A88B2F5805F07D89C
:106D80000120187070475A809A80012070470020B7
:106D900070470000E0B110B50446037843B14FF4EA
:106DA0007A52002300206188FEF720FB024600E0B3
:106DB000002272B6074B2068C3F82801A188A3F807
:106DC0002C110021C3F83011C3F8342162B610BD74
:106DD000704700BF6815002072B6074B93F83C312E
:106DE000DBB2FF2B06D0044A92F83C310133DBB210
:106DF00082F83C3162B670476815002072B6064BC7
:106E000093F83C3133B1044A92F83C31013BDBB298
:106E100082F83C3162B6704768150020014BD87685
:106E2000704700BF68150020028802F00101364B50
:106E300083F8AC10C2F3400183F8AD10C2F38001B7
:106E400083F8AE10C2F3C00183F8AF10C2F3001193
:106E500083F8B010C2F3401183F8B110C2F380116F
:106E600083F8B210C2F3C01183F8B310C2F300214B
:106E700083F8B410C2F3402183F8B510C2F3802127
:106E800083F8B610C2F3003183F8B710C2F3403272
:106E900083F8B8204288A3F8D0208288A3F8E020A5
:106EA0004289A3F8BA20828907EE902AF8EE677A21
:106EB0009FED167A67EE877AC3ED357AC28907EEC1
:106EC000902AF8EE677A67EE877AC3ED367A028AFF
:106ED00007EE902AF8EE677A67EE877AC3ED397A83
:106EE000428A07EE902AF8EE677A67EE877AC3ED5A
:106EF0003A7A828AA3F8BC20C28AA3F8DC20028BEB
:106F0000A3F8EC20704700BF681500200000803B0C
:106F1000002918BF002816D000B584468E460023ED
:106F20000DE0991C5A001CF811000EF813003CF8F3
:106F300011100132090A0EF802100133DBB20A2BDC
:106F4000EFD95DF804FB704708B5064800210160E1
:106F500041608160C160018220223230FAF7C2FEB6
:106F600008BD00BF26160020054B00221A609A803B
:106F70009A60DA6047F6FF71198259821A75704774
:106F80009016002008B5034A537E1843507603F04C
:106F900079FF08BD6815002008B50C280CD8DFE87B
:106FA00000F00A07070B07070B0B0B0B0B0707007B
:106FB0000420FFF7E7FF08BD0120FFF7E3FFFAE732
:106FC00008B5044B012283F83C20587E03F05AFF99
:106FD00008BD00BF6815002008B510B1034642790E
:106FE0002AB90420FFF7CEFFFFF7EAFF08BD0089AA
:106FF000D98801F00101C0F30B0001F087FEFFF713
:10700000DFFFF3E710B5044C204601F0E0F854F838
:10701000402C44F8382C10BDA815002008B5084BAA
:1070200093F846302BB1064A136892689B1A642B7A
:1070300000D808BDFFF7E6FF0220FFF7A3FFF8E73F
:107040006815002010B5074C4FF4C6720021204689
:10705000FAF748FE002084F88E01A4F88C0103F0B2
:10706000DBFE10BDA816002070B50646164D0024A4
:107070006C76AC7685F83C402C766C612C612C7378
:10708000C5F81041C5F81441C5F81841C5F81C41B0
:10709000C5F82041C5F82441FFF766FFFFF7D2FF8E
:1070A000204603F0EFFE05F18E0002F06FFC05F1C3
:1070B000400001F08CF885F8684001F079FB16B1CA
:1070C0002C606C60AC6070BD6815002008B5034B87
:1070D00083F83A0003F0C6FE08BD00BF6815002023
:1070E00008B5044B93F83A2083F83B20FFF7EEFFF6
:1070F00008BD00BF6815002008B5054B1B7E03B115
:1071000008BD01F06DF9024B01221A76F8E700BFC5
:10711000681500202DE9F04782B0394B00229A769D
:1071200008B142793AB90420FFF72CFFFFF748FF76
:1071300002B0BDE8F087C5880689448905F00108DA
:10714000C5F34007C5F38009FFF746FEB9F1000F0C
:1071500023D015F0080F05D104F00F09344641F68D
:10716000FF7601E04FF0010900963B464A46214672
:10717000404602F01EF905464B462246414602F0C3
:107180005DFA30B9FFF73AFE1D4B9D76FFF718FF09
:10719000CEE78020FFF7F6FEF4E75FFA86F9C6F344
:1071A000032A26430ED0B9F1000F05D0B9F13F0FE5
:1071B00004D94FF03F0901E04FF0010944B94FF6FF
:1071C000FF7405E04FF6FF744FF0020A4FF001091B
:1071D00007B10227009453464A464146384602F01A
:1071E000A5F805460194CDF800A04B463A46414625
:1071F00002F0B8F90028C5D08020FFF7C3FEC1E730
:107200006815002010B510B1044643793BB902F06F
:1072100061F90420FFF7B6FEFFF7D2FE10BDFFF7BD
:10722000DBFDE18804F1080002F018F920B1FFF756
:10723000E5FDFFF7C5FEF1E702F04CF98020FFF70E
:10724000A1FEF4E730B5ADF2344D00230B938DF879
:10725000133000286BD0037823B9002420460DF2A8
:10726000344D30BD0BAB009340F2FF330CAA00212C
:1072700002F0C2FC00285CD10B9B0CAC0025E5544D
:1072800000E00134237883B1002203A92046FAF7F5
:107290002BFE039BA342F4D0B5F5805F03D20135EA
:1072A000ADB21C46EEE70024D8E7012D06D92846EA
:1072B00002F0B4F810B100240CAD07E00024CDE7D3
:1072C000013503E002F006F9C8E7039D2B78BBB156
:1072D000002203A92846FAF707FE039BAB42EFD032
:1072E00005AB23F814000134A4B20C2CEDD12146D7
:1072F000184602F0B3F804460028E3D00024E4E77F
:107300002CB1214605A802F0A9F8044648B10DF1B8
:10731000130002F0EBF89DF813302BB19DF81340E9
:107320009CE702F0D7F899E702F0D4F8F6E70024DA
:1073300094E7002492E700283ED030B583B004469D
:107340000378012B1DD0022B2CD0002B36D1807856
:1073500000B10220E38800932379E278617801F09C
:10736000E5FF6178A27802B102222379E5880195D0
:107370000093E37802F0F6F8B0FA80F0400903B029
:1073800030BD838900938378827A0189407802F046
:1073900010F8A37A2289617802F050F9B0FA80F0EF
:1073A0004009ECE743781BB10E30FFF74BFFE6E7EF
:1073B00001F054FF0120E2E7012070470020DEE7E2
:1073C00070B582B000238DF80730254A937608B156
:1073D000427932B90420FFF7D5FDFFF7F1FD02B085
:1073E00070BDC48805894689FFF7F6FC022C0ED0D3
:1073F000032C21D0012C2CD11EB9284602F00EF806
:10740000F0B902F067F88020FFF7BCFD18E03543C3
:1074100005D002F05FF88020FFF7B4FD10E00DF119
:10742000070002F063F80E4B98769DF807303BB9E1
:107430008020FFF7A7FD03E0354306D102F04AF8AC
:10744000FFF7DCFCFFF7BCFDC9E78020FFF79AFDE2
:10745000F4E702F03FF88020FFF794FDF0E700BF6B
:107460006815002070B50646264C04F1AC0CD4F823
:10747000BE00D4F8C210D4F8C620D4F8CA30ACE8A4
:107480000F00B4F8CE30ACF8003004F1D00504F1B0
:10749000F0030FCB85E80F0004F1E00504F58073DD
:1074A0000FCB85E80F000020FFF710FE002584F8C1
:1074B0003B5003F0EDFB02F00DF801F0CFFE2A4641
:1074C0002946284601F082FC01F004F829462846A6
:1074D00001F01CFC0C4B1B6813F0400F04D00A4A4F
:1074E000136823F040031360084B1B6813F0400F30
:1074F00004D0064A136823F0400313603046FFF7B8
:10750000B3FD70BD681500200038004000540140F4
:1075100038B508B142792AB90420FFF733FDFFF7E7
:107520004FFD38BDC5880489C4F30D044389C3F3F6
:107530000D0344EA8334FFF74FFC2246C5F34001B4
:1075400005F0010001F042FCFFF758FCFFF738FDA1
:10755000E7E7C0B110B50446D0F87C2190F8791166
:1075600090F8780101F032FC94F88011B4F88201AF
:1075700001F0CCFB94F88A3103B910BD94F88B016B
:1075800001F09AFCF9E7704738B504460D46FFF75D
:1075900023FC2946204601F069F9FFF72FFC38BD8E
:1075A00010B5414C94F8AD10003918BF01210120ED
:1075B00001F05EF894F8AE10003918BF01210220E6
:1075C00001F056F894F8AF10003918BF01210120DE
:1075D00001F062F894F8B010003918BF01210220C0
:1075E00001F05AF894F8B110003918BF01210120B8
:1075F00001F06AF894F8B210003918BF0121022096
:1076000001F062F894F8B7302BB9284AC4F8D420B6
:10761000274AC4F8D820244B93F8B83033B9224B0A
:10762000224AC3F8E420224AC3F8E8201E4B93F80C
:10763000B5301BB11C4B93F8B33083B90021012046
:1076400001F05AF8184B93F8B6301BB1164B93F86B
:10765000B430B3B90021022001F04EF810BD47F656
:10766000FF74114BA3F8384121460320FFF78CFF2C
:1076700021460320FFF788FF0121084601F03CF86E
:10768000E0E747F6FF74084BA3F83A41214604208F
:10769000FFF77AFF21460420FFF776FF0121022041
:1076A00001F02AF8DAE700BF681500200000204149
:1076B0000AD7233CF0B583B0002876D00F460546A4
:1076C0002AB190F8D130002B4DD1002600E00026E1
:1076D0000020FFF7C7FE364C4FF4C672294604F56A
:1076E000A070FAF725FCA4F8CC72012384F8CE32FE
:1076F00004F1AC0C05F1D40EBEE80F00ACE80F00AD
:10770000DEF80030ACF8003004F1D00C05F1E803ED
:107710000FCB8CE80F00E03405F1F8030FCB84E8C1
:107720000F0000238DF800308DF80130ADF80230E5
:10773000ADF80430694605F5C270FFF704FBA0B14F
:107740006846FFF727FB05F58470FFF7F4FD044654
:1077500078B12846FFF7FDFE284603F05DFB76B9B9
:10776000204603B0F0BD0126B2E70120FFF70AFC76
:10777000E6E7FFF777FE8020FFF704FCF0E70D4A0D
:10778000136843F04003136002F58E32136843F030
:1077900040031360FFF704FF0120FFF797FC044B41
:1077A000012283F83B203446DAE70024D8E700BF03
:1077B000681500200038004030B5EBB00023ADF86C
:1077C0001A3000F02FFF18B1002420466BB030BDF6
:1077D00004460120FFF722FB02F09EF9054680B126
:1077E0006946284802F03BFA002818BF042817D041
:1077F00005280ED10120FFF7C5FB0420FFF70EFB83
:10780000E3E70120FFF7BEFB0220FFF707FB2C4652
:10781000DBE70120FFF7B6FB0320FFF7FFFAD4E711
:10782000031FDBB2012BE5D90DF11A0107A802F005
:107830000DFF044688B19DF8EE40ACB10122BDF8C1
:107840001A1007A8FFF736FF044688B19DF8ED30FF
:10785000ABB10920FFF7E2FAB7E70120FFF792FB8F
:107860000520FFF7DBFAB0E70620FFF7D7FAACE711
:107870008020FFF787FB0720FFF7D0FAA5E7082055
:10788000E8E700BF2C10010810B510B10446437999
:107890002BB90420FFF776FBFFF792FB10BD0E4AD1
:1078A000136843F04003136002F58E32136843F00F
:1078B00040031360FFF7C6FBA01DFFF7B5FAFFF703
:1078C0006FFE0120FFF702FC044B012283F83B20EE
:1078D000FFF776FBE2E700BF0038004068150020A4
:1078E00030B585B070B3427962B3C288032A30D80C
:1078F00002F001018DF80810C2F340028DF8092052
:107900000289ADF80A204389ADF80C30694602A817
:10791000FFF719FA18B31A4B93F8285193F8294135
:107920006846FFF737FA55B19DF800301BB19DF856
:107930000130A34203D02046FFF7D4F9A8B9FFF7DE
:107940003FFB04E00420FFF71DFBFFF739FB05B008
:1079500030BD0420FFF716FBFFF732FBF7E70420EA
:10796000FFF710FBFFF72CFBF1E704F19C02E01C92
:10797000034B33F81210C0B2FFF706FEDFE700BF7B
:107980006815002010B50446012814D80846FFF7F2
:10799000CBF90146084B04F19C0223F8120093F83E
:1079A000283123B1044B93F82931A34203D0033487
:1079B000E0B2FFF7E9FD10BD6815002038B52B4B8C
:1079C00093F82831002B46D0284B93F83A30012BFE
:1079D00041D1264B93F83C31002B3DD1234B93F8FA
:1079E00029412046FFF77EF9A8B3204D04F19C03FE
:1079F00035F81300FFF798F9A0F57A739BB24DF6AE
:107A0000E052121A92B2934228BF1346B5F82C21C5
:107A10009A4200D31A46154DD5F83031DB0E144981
:107A200031F9133002FB03F3124A82FB03121A44AA
:107A3000DB17C3EBA2330334E4B21844FFF774F945
:107A40000146204600F012FFD5F83031D5F8342138
:107A50001344C5F8303138BD044BD3F83021D3F886
:107A600034110A44C3F83021F5E700BF681500203F
:107A7000741501080300018030B585B08646002AE0
:107A800018BF00280CBF0120002037D00C46154637
:107A9000102B34D94B1E9BB20F2B30D800230093F0
:107AA00001930293039312E01A1D3EF812104FEA5D
:107AB000430C04AA02EB430202F8101C090A0CF161
:107AC00011020DEB020C0CF8101C0133DBB2072B7A
:107AD000EAD9E3B20F2B08D803F110026A4412F876
:107AE000102C62B90133DBB2F4E72246694628461E
:107AF000FAF71EFA00232B55012000E0002005B004
:107B000030BD000010B586B01E4B00229A7690B1B1
:107B1000044643797BB1C388022B1BD0032B26D0AC
:107B2000012B2AD1112301AA81890630FFF7A4FF76
:107B300048B9022412E003F0ABF80420FFF722FA60
:107B4000FFF73EFA11E06289218901A802F0C2FF25
:107B5000044602E003F044F8044614B12046FFF75F
:107B60001BFA084B9C76FFF72BFA06B010BD03F00A
:107B70008FF802F0A9FF0446EFE703F089F801242B
:107B8000ECE700BF6815002008B588B142797AB1EA
:107B9000B0F806C002894389CCF340010CF0010023
:107BA0001CEA010F0AD17AB1402A0ED940220CE01A
:107BB0000420FFF7E7F9FFF703FA12E00420FFF7CC
:107BC000E1F9FFF7FDF90CE001222BB1B3F5FA7FE3
:107BD00003D94FF4FA7300E0022301F061F9FFF7D3
:107BE000EFF908BD30B587B01A4B00229A76E8B19C
:107BF0004279DAB1C5880489162C20D80022009277
:107C00000192029203920492ADF814206946063064
:107C1000FFF77EF922466946284602F0A3FF044694
:107C2000A8B90C4B9C76FFF7CBF906E003F030F8CF
:107C30000420FFF7A7F9FFF7C3F907B030BD03F041
:107C400027F80420FFF79EF9FFF7BAF9F5E7FFF7E9
:107C5000A3F9E6E76815002000283BD008B50378B3
:107C6000013B0C2B0AD8DFE803F0070A10141A1D99
:107C70002023262C2F322900FFF706FE08BD002006
:107C8000FFF7F0FBFFF79CF9F8E70220FFF728FA6F
:107C9000F4E7114BDA7E9A76FFF792F9EEE7FFF7F9
:107CA00031FFEBE7FFF736FAE8E7FFF731FCE5E7EE
:107CB000FFF76AFFE2E7FFF78FF9DFE7FFF710FE54
:107CC000DCE7FFF77DFBD9E7FFF79CFAD6E7FFF784
:107CD00089FFD3E7704700BF68150020184B93F861
:107CE00068305BB372B6164B93F868300BB962B666
:107CF000704730B58BB0124D05F16A0C01AC8A3576
:107D0000A646DCF80000DCF80410DCF80820DCF8FB
:107D10000C30AEE80F000CF1100C7446AC45EFD1FE
:107D2000DCF80000CEF80000054B002283F8682044
:107D300062B601A8FFF790FF0BB030BD704700BFDF
:107D400068150020184B1B7B33B103F0FF02164B64
:107D500000211973012A00D0704700B5E5B0B3F8CF
:107D6000CC22ADF8022093F8CE325BB101A90DF11F
:107D7000020002F07DFC58B90120FFF703F965B05D
:107D80005DF804FB0DF1020101A802F05FFCF2E7CF
:107D90000122BDF8021001A8FFF78CFC0028EED1EB
:107DA0008020FFF7EFF8EAE7681500202DE9F04F93
:107DB00089B006460D46012000F02CFE4B4CA4F87D
:107DC0001801012000F026FEA4F81801022000F09E
:107DD00021FEA4F82401022000F01CFEA4F82401D6
:107DE000032000F017FE032000F014FEA4F8100199
:107DF000042000F00FFE042000F00CFEA4F81C018B
:107E0000002E4AD1002D65D1002000F015FF012081
:107E100000F012FF0546012000F00EFF064601208B
:107E200000F00AFF0746012000F006FF804601200F
:107E300000F002FF8146022000F0FEFE032000F069
:107E4000FBFE042000F0F8FE042000F0F5FE824660
:107E5000052000F0F1FE254C04F18E0BB4F8BC10A7
:107E6000584601F09FFD2368CDF81CA0CDF818906E
:107E7000CDF81480049703960295B4F81C21019262
:107E8000B4F810210092B4F82421B4F8181158461F
:107E900001F08BFD09B0BDE8F08F636804F11406B2
:107EA0000096012204F5887104F1D00001F0C2FDB2
:107EB00001460020FFF766FD63680096022204F584
:107EC0008E7104F1E00001F0B5FD01460120FFF7DD
:107ED00059FD97E7054CB4F8DC100120FFF754FB7F
:107EE000B4F8EC100220FFF74FFB8DE76815002077
:107EF000084B5A681B699A4200D8704710B5054C68
:107F00006368236101210846FFF750FF012384F8CD
:107F10003B3010BD6815002038B5134B93F83C304A
:107F2000012B13D0022B1DD1104C204601F05CFD1B
:107F3000A4F172052946204601F060FD1E21284665
:107F400000F052FC002304F8523C0BE0084C0221E4
:107F5000204600F033FC2046002300F819398376D0
:107F600080F83C3038BD00BF68150020F6150020B1
:107F70008115002010B54FF4347200212648F9F71E
:107F8000B1FEFEF7E1FF0120FFF76EF800F04AFBBB
:107F900000283DD00020FFF799F800241E4B83F8FD
:107FA0003B402046FEF73AFF00F0D2FB00F07AFE9D
:107FB00002F080FD2146204600F0A8FE00F08AFA7B
:107FC0002146164806F0BAF9154BDA6842F001026C
:107FD000DA601A6842F001021A6003F58063DA6819
:107FE00042F00102DA601A6842F001021A6003F5F9
:107FF0008063DA6842F00102DA601A6842F0010236
:108000001A60FFF779F801F0EDF8FFF7D5FB10BD26
:1080100002F0D8FEBEE700BF68150020C4030020B0
:10802000000C004008B1014A107370476815002029
:1080300010B5FFF761F81A4B93F83A30012B11D0C5
:10804000174C206802F02CFFFFF7ECFFFFF746FE0D
:10805000FFF778FE94F83A30032B1CD8DFE803F0E2
:1080600007050C15FFF744FFEAE7FFF741FFFFF7AD
:1080700053FFFEF7D3FF10BD094B022283F83C20CB
:1080800093F83B00FFF722F8F1E7FEF799FF002095
:10809000FFF71CF8EBE70320FFF718F8E7E700BF4E
:1080A0006815002030B58BB001461B4B93F8463065
:1080B00013B9194B1A689A6001AA184800F08BF896
:1080C000022803D0012807D00BB030BDFEF79AFF7D
:1080D0000220FEF757FFF7E70F4B93F86830B3B96C
:1080E0000DF1040E0E4C09ADF446BCE80F00206003
:1080F0006160A260E360E6461034AC45F4D1DCF880
:1081000000002060044B012283F86820DCE7022095
:10811000FEF738FFD8E700BF68150020A81500203B
:10812000D215002008B5FEF76DFF0220FEF72AFFEA
:1081300008BD000008B5034A13680133136000F05E
:10814000FFFA08BD68150020024A536801335360E6
:10815000704700BF6815002008B5FFF72FFC08BD69
:1081600008B500F07DFB08BD00230C2B0DD803EBF8
:108170004302074931F81220824201D00133F4E76B
:1081800003EB430301EB430070470020704700BF3F
:10819000B4150108002918BF00280ED000B5844688
:1081A0008E460088012304E03CF813205040013340
:1081B0009BB27345F8D35DF804FB0020704728B1EB
:1081C00008B528220021F9F78DFD08BD704708B5D4
:1081D000FFF7F5FF08BD70B5002A18BF002800F0B2
:1081E00085800446164685798DB1012D14D003682B
:1081F000002B37D09A78954238D24219D171013587
:10820000EDB285719B789D4234D200256FE0C1713B
:108210008180012383716AE00172808840EA012035
:10822000A080FFF7A1FF206030B10223A371837803
:10823000022B06D000255AE02046FFF7C8FF022592
:1082400055E0242200213046F9F74CFD23685B7984
:10825000337023681B887380012373712046FFF7F6
:10826000B6FF44E0FFF7B3FF022540E0FFF7AFFFA2
:1082700002253CE0242200213046F9F733FD236833
:108280005B79337023681B8873802368DB783371D4
:1082900000220EE0511CC9B24B00DBB2E018C079DD
:1082A00001332344DB7940EA032306EB4202D38007
:1082B0000A462368D9789142ECD893F90410002932
:1082C00011DBCDB22946B01DFFF764FF06EB450177
:1082D000CB88984214BF0020012070712046FFF720
:1082E00076FF012503E001237371F7E70025284697
:1082F00070BD000008B503F0ADFC034B9B6813F4A0
:10830000E05F00D0400008BD0038024030B58FB0BB
:10831000002309930A930B930C930D9302930393F9
:1083200004930593069307930893FFF7E3FF264C06
:10833000A4FB0034E40D254B984200D80124244BC3
:108340001A6B42F002021A631A6B02F002020092E8
:10835000009A1A6C42F004021A641B6C03F00403C6
:108360000193019B4FF48073099302230A93002524
:108370000B950C950D9309A9164803F08BFF164831
:10838000164B0360013C4460856040F2E733C360F4
:108390000561856105F030FE08B10FB030BD602386
:1083A00002934FF4967303930495069508220DEB00
:1083B0000201094805F088FE0028EED10821064890
:1083C00005F0BCFFE9E700BF6BCA5F6BFF2C310112
:1083D0000038024000040240381800200008004025
:1083E000124A52E8003F43F4807342E8003100290A
:1083F000F6D10E4A52E8003F43F0200342E8003134
:108400000029F6D1094A02F1080353E8003F43F07E
:108410000103083242E800310029F3D1044B002265
:1084200083F8252320225A60704700BF00100140C6
:1084300000E100E0F0B589B00024039404940594B1
:1084400006940794204B1A6B42F040021A631A6B91
:1084500002F040020192019A1A6B42F008021A637C
:108460001B6B03F008030293029B184D22464FF446
:108470007641284604F017F8154F224680213846E9
:1084800004F011F84FF47643039301260496059403
:10849000069403A9284603F0FDFE80230393049667
:1084A0000594069403A9384603F0F4FE4FF40063E4
:1084B00003930494059603A9284603F0EBFEFFF707
:1084C00025FF09B0F0BD00BF00380240001802408F
:1084D000000C02402DE9F0413C4E002208213046BC
:1084E00003F0E1FF00228021304603F0DCFF384F2B
:1084F00000224FF48071384603F0D5FF002210218E
:10850000304603F0D0FF334C00224FF48061204608
:1085100003F0C9FF304D00220821284603F0C3FFB5
:1085200000220121284603F0BEFF00220221284636
:1085300003F0B9FF00224FF40061204603F0B3FFBF
:1085400000222021304603F0AEFF06F5006601222E
:108550004FF48061304603F0A6FFDFF880800122EF
:108560004021404603F09FFF01224FF480413046F6
:1085700003F099FF01224FF40071404603F093FF8E
:1085800001224FF48041204603F08DFF012240215B
:10859000284603F088FF01224FF48051384603F04B
:1085A00082FF01224FF48071304603F07CFF0122EC
:1085B0004FF48051204603F076FF01224FF4005122
:1085C000384603F070FFBDE8F08100BF00080240AC
:1085D000000C02400004024000000240001402406F
:1085E0000F4B1B6813F0400F04D00D4A136823F0A3
:1085F000400313600A4B1A6822F00202104318600D
:108600001A6822F00102114319601B6813F0400F31
:1086100004D1034A136843F040031360704700BF5E
:108620000038004008B54FF48071044803F034FF6F
:10863000012814BF0020012008BD00BF0000024037
:1086400008B50121034803F027FFB0FA80F0400984
:1086500008BD00BF000C024008B54FF4006103489C
:1086600003F01AFFB0FA80F0400908BD001802407C
:1086700008B5012802D0022806D008BD0A46082104
:10868000044803F010FFF8E70A468021014803F090
:108690000AFFF2E70008024008B5012802D00228CC
:1086A00007D008BD0A464FF48071054803F0FBFE71
:1086B000F7E70A461021034803F0F5FEF1E700BF93
:1086C000000C02400008024008B5012802D0022830
:1086D00007D008BD0A464FF48061054803F0E3FE69
:1086E000F7E70A460821034803F0DDFEF1E700BF83
:1086F000000402400000024010B50C46012802D0E0
:1087000002280CD010BD0A464FF40061094803F05E
:10871000CAFE22460121084803F0C5FEF2E70A46D8
:108720002021064803F0BFFE22460221024803F042
:10873000BAFEE7E7000402400000024000080240E1
:1087400008B50221014803F0B4FE08BD000C024048
:10875000144BD3F8B82022F00102C3F8B8204FF030
:108760000062DA604FF00072DA600F4A02F108032B
:1087700053E8003F43F08003083242E8003100290B
:10878000F3D1084BD3F8B82042F01002C3F8B82058
:10879000D3F8B82042F00402C3F8B820034B0022FB
:1087A0001A707047006402400010014084180020D5
:1087B000014B00221A707047841800208C4600225A
:1087C0000CE033B9074BDB6913F08003F9D00123C8
:1087D000F7E7815C034B9962013292B26245F1D3B3
:1087E000704700BF001001401A4B1B78002BFBD1D3
:1087F000194BD3F8B82022F00102C3F8B8204FF08B
:108800000062DA604FF00072DA60D3F8B83003F03B
:10881000C003402B16D0104BC3F8C0000F4AC3F85A
:10882000C4200D4BD3F8BC206FF30F021143C3F8E3
:10883000BC10084A01211170D3F8B8200A43C3F8CC
:10884000B8207047044BC3F8C400044AC3F8C020E2
:10885000E7E700BF841800200064024028100140B0
:10886000014B00221A7070478418002038B5044666
:108870000D46032818BF012806D0013C032C2ED832
:10888000DFE804F00D456F9001210220FFF7A8FEFC
:1088900001224FF48051594803F005FEEDE7002214
:1088A0004FF48041554803F0FEFD0022544B9B6875
:1088B00013F0020F04D1B2F5FA7F01D80132F5E7C7
:1088C0004F4B9D8100224E4B9B6813F0010F04D14A
:1088D000B2F5FA7F01D80132F5E7494BDB68012296
:1088E0004FF48041454803F0DEFD01224021454818
:1088F00003F0D9FD01224FF48051434803F0D3FD2A
:1089000001224FF48071414803F0CDFD38BD404B4A
:108910001B6813F0400F04D13D4A136843F0400335
:10892000136000224021374803F0BDFD0022384B80
:108930009B6813F0020F04D1B2F5FA7F01D801321F
:10894000F5E7334B9D810022314B9B6813F0010FFB
:1089500004D1B2F5FA7F01D80132F5E72C4BDB6880
:10896000BDE700224FF48051274803F09CFD002210
:10897000234B9B6813F0020F04D1B2F5FA7F01D8A4
:108980000132F5E71E4B9D8100221D4B9B6813F0C1
:10899000010F04D1B2F5FA7F01D80132F5E7184B87
:1089A000DB689CE71A4B1B6813F0400F04D1184A90
:1089B000136843F04003136000224FF480711348A2
:1089C00003F071FD0022124B9B6813F0020F04D1DB
:1089D000B2F5FA7F01D80132F5E70D4B9D810022F7
:1089E0000B4B9B6813F0010F04D1B2F5FA7F01D84D
:1089F0000132F5E7064BDB6871E700BF0004024077
:108A00000038004000000240000C0240001002400C
:108A10000054014010B5044600224FF480418248C2
:108A200003F041FD00224FF40071804803F03BFD4C
:108A3000002300E00133B3F5FA7FFBD301224FF4AA
:108A40008041794803F02FFD01224FF400717748EF
:108A500003F029FD002300E00133B3F5FA7FFBD3D7
:108A6000631E032B00F2DD80DFE803F002396EA500
:108A70006D4C01224FF40061204603F014FD0022EA
:108A80004FF48061204603F00EFD002300E0013327
:108A9000B3F5FA7FFBD3664A136843F040031360D3
:108AA0000023634A926812F0010F04D1B3F57A7F74
:108AB00001D80133F5E75E490A6822F040020A60F6
:108AC00000E00133B3F5FA7FFBD301224FF480615C
:108AD000554803F0E8FC564BD86880B210BD534CA3
:108AE00001224FF48061204603F0DDFC002240218A
:108AF000204603F0D8FC002300E00133B3F5FA7FF1
:108B0000FBD34C4A136843F0400313600023494AE7
:108B1000926812F0010F04D1B3F57A7F01D80133C6
:108B2000F5E744490A6822F040020A6000E0013398
:108B3000B3F5FA7FFBD3012240213C4803F0B3FC9C
:108B40003C4BD86880B2C9E7374C01224FF48061B2
:108B5000204603F0A8FC00224FF40061204603F0F9
:108B6000A2FC002300E00133B3F5FA7FFBD3304AC7
:108B7000136843F04003136000232D4A926812F0FB
:108B8000010F04D1B3F57A7F01D80133F5E7284905
:108B90000A6822F040020A6000E00133B3F5FA7F70
:108BA000FBD301224FF400611F4803F07CFC204BF3
:108BB000D86880B292E71D4C01224021204603F084
:108BC00072FC00224FF48061204603F06CFC00230D
:108BD00000E00133B3F5FA7FFBD3164A136843F084
:108BE000400313600023134A926812F0010F04D16E
:108BF000B3F57A7F01D80133F5E70E490A6822F010
:108C000040020A6000E00133B3F5FA7FFBD3012292
:108C10004FF48061054803F046FC064BD86880B2EB
:108C20005CE700205AE700BF001002400014024039
:108C3000003401400050014010B505282CD8DFE871
:108C400000F0030812171C26144802F021FA002035
:108C500010BD124C6421204602F0D4FA204602F0E6
:108C600032FB80B2F4E70D4802F0ACFA0020EFE7E7
:108C70000B4802F00DFA0020EAE7094C6421204677
:108C800002F0C0FA204602F01EFB80B2E0E7044882
:108C900002F098FA0020DBE70020D9E7DC0400208E
:108CA0009404002010B588B0002403940494059423
:108CB00006940794114B1A6C42F000521A641A6C15
:108CC00002F000520192019A1A6B42F001021A63FB
:108CD0001B6B03F001030293029B102303930323F6
:108CE000049303A9064803F0D5FA064B1968064A0F
:108CF0000A401A609C6008B010BD00BF00380240F6
:108D00000000024000740040FAEFFFFFB0F5805F02
:108D100001D340F6FF70074B986029B11A461B68D3
:108D200043F0010313607047024A136823F0010304
:108D3000136070470074004038B5044600210220DB
:108D4000FFF74EFC1E4D01224FF48051284603F0E0
:108D5000AAFB01224FF48041284603F0A4FB05F54D
:108D6000006501224FF48051284603F09CFB00224D
:108D70004FF40051284603F096FB0023114A9268F5
:108D800012F0020F05D15A1CB3F57A7F01D21346B7
:108D9000F4E70C4B9C8100230A4A926812F0010F01
:108DA00005D15A1CB3F57A7F01D21346F4E7054B7F
:108DB000DB6801224FF40051034803F074FB38BD17
:108DC0000004024000380040000C02402DE9F04150
:108DD0000546F9B94FF4005747F48078C2F30D0601
:108DE00046F48046C2F38D3242F480444046FFF799
:108DF000A3FF3046FFF7A0FF2046FFF79DFF4FF48B
:108E00004040FFF799FF05B947463846FFF794FF02
:108E1000BDE8F08142F20207DEE7000010B5064C23
:108E200001220421204603F03EFB012208212046B6
:108E300003F039FB10BD00BF001002402DE9F843DC
:108E4000BDF8209032B105460E461F46904650EAC6
:108E5000010303D1FFF7E2FFBDE8F883FFF7DEFF70
:108E600000240FE0002204210C4803F01CFB0DE05D
:108E7000384603F01FFCFFF7D1FF484603F01AFC09
:108E80000134A4B24445E7D2002DEBD1002EEFD03F
:108E900000220821014803F006FBE9E70010024028
:108EA00000B583B0012B05D90093FFF7C7FF03B0CE
:108EB0005DF804FB0223F7E730B583B004463F2892
:108EC00000D93F240A2003F0F5FB022500952B462C
:108ED000402201210020FFF7B1FF00952B462246DA
:108EE00000210120FFF7AAFF03B030BD024B002292
:108EF0001A705A809A8070478818002038B50C463E
:108F0000C0F30E0500210846FFF76AFB01224FF46B
:108F100080412C4803F0C7FA01224FF480512A48BF
:108F200003F0C1FA294B1B6813F0400F04D1274A04
:108F3000136843F04003136000224FF4805121482E
:108F400003F0B1FA0023214A926812F0020F05D112
:108F50005A1CB3F57A7F01D21346F4E71B4B9D816F
:108F600000231A4A926812F0010F05D15A1CB3F57A
:108F70007A7F01D21346F4E7144BDB680023134ACF
:108F8000926812F0020F05D15A1CB3F57A7F01D214
:108F90001346F4E70D4B9C8100230C4A926812F0B3
:108FA000010F05D15A1CB3F57A7F01D21346F4E7BD
:108FB000064BDB6801224FF48051024803F073FA3C
:108FC00038BD00BF00040240000C024000380040E1
:108FD00070B506460D46002408E036F81410054B1F
:108FE00033F81400FFF78AFF0134A4B2AC42F4D383
:108FF00070BD00BF0C17010800B583B001224FF40B
:1090000000610F4803F04FFA01211E20FFF776FFA1
:1090100001211D20FFF772FF0023019302E0019B55
:1090200001330193019BB3F57A7FF8D300224FF40B
:109030000061034803F037FA03B05DF804FB00BF9A
:10904000000C0240F8B50F461646012806D9054621
:10905000B0F5805F03D94FF4805500E00225B6F5E6
:10906000005F01D341F6FF7604211E20FFF746FF83
:10907000002431E0012138E001213CE0681A80B28F
:10908000012808D9013880B2611A02FB01F191FB75
:10909000F0F1591A0AE00120F6E7012D0FD9691EF7
:1090A00089B204FB02F292FBF1F2D11A11F5005FD2
:1090B00007DBB1F5005F05DB41F6FF7102E001213E
:1090C000EFE7124989B2890089B204F5C04080B245
:1090D000FFF714FF0134A4B2A54212D9334672003F
:1090E000002FDAD06908012DC4D98C42C6D20129DB
:1090F000C2D9013989B204FB02F292FBF1F2D11A12
:10910000D4E700211E20FFF7F9FEF8BD00E0FFFFC5
:1091100010B540F4004400210846FFF761FA01222F
:109120004FF480412C4803F0BEF901224FF48051E6
:109130002A4803F0B8F92A4B1B6813F0400F04D1FA
:10914000274A136843F04003136000224FF4805114
:10915000214803F0A8F90023214A926812F0020F77
:1091600005D15A1CB3F57A7F01D21346F4E71C4BA4
:109170009C8100231A4A926812F0010F05D15A1CF3
:10918000B3F57A7F01D21346F4E7154BDB68002371
:10919000134A926812F0020F05D15A1CB3F57A7F78
:1091A00001D21346F4E700230D4A93810C4A9268DA
:1091B00012F0010F05D15A1CB3F57A7F01D2134684
:1091C000F4E7074BDC68A4B201224FF48051024857
:1091D00003F069F9204610BD00040240000C024073
:1091E0000038004000B583B001224FF48051174889
:1091F00003F059F900224021154803F054F90023E7
:10920000019302E0019B01330193019BB3F57A7F47
:10921000F8D3012240210E4803F045F942210D48C0
:10922000FFF7D6FE00211E20FFF768FE01211D205A
:10923000FFF764FE01224FF40061074803F033F9A1
:10924000FFF754FE03B05DF804FB00BF00040240CA
:109250000008024088160108000C024008B50021F1
:109260001E20FFF74BFE01224FF40061014803F07E
:109270001AF908BD000C024070B5012806D9044651
:10928000B0F5805F03D94FF4805400E0022419B197
:109290000F2902D90F2100E001210D0205F47065AC
:1092A00045F01105264601F00F0104FB01F119B14B
:1092B000B1F5803F35D20E4642211B48FFF788FEAC
:1092C000FFF7CCFF43F230012720FFF717FE4FF4E2
:1092D00000713720FFF712FE40F201112B20FFF73B
:1092E0000DFE29462820FFF709FEB1B22920FFF71D
:1092F00005FE00211F20FFF701FE00215C20FFF783
:10930000FDFD00215D20FFF7F9FD611E89B2090115
:1093100089B25E20FFF7F2FD01211D20FFF7EEFD6F
:1093200070BD4FF6FF76C7E7041601082DE9F0413E
:109330000546884614461E46BDF81870FFF7D6FD50
:10934000B8F1000F04D04CB13F2C08D93F2406E0FF
:10935000FFF784FF1E20FFF7DBFE28E001240FB992
:109360004FF6FF7705F00305A400E4B2254336016C
:1093700006F0F00640F20114344343F21221272094
:10938000FFF7BCFD29463720FFF7B8FD214628200E
:10939000FFF7B4FD39462920FFF7B0FD00211F205B
:1093A000FFF7ACFDFFF728FE1E20FFF7B1FEBDE87A
:1093B000F0812DE9F04106460C4615461F46BDF8E2
:1093C0001880FFF793FD1CB1012C02D8022403E0A2
:1093D0001024B4F5805F04D835B10F2D05D90F25C1
:1093E00003E04FF48054F7E70125B8F5005F01D39F
:1093F00041F6FF7829462046FFF73EFF42463946B0
:109400002046FFF71FFE36B1FFF7F6FD1E20FFF7DF
:109410007FFEBDE8F081FFF721FFF7E7831E9BB2D7
:1094200040F6FE72934201D90020704710B5044601
:10943000FFF714FFFFF75AFD01212046FFF71CFF3D
:1094400004211E20FFF75AFD034B5C8000229A8006
:109450000120187010BD00BF8818002070B370B5CF
:109460000D4606461A4B1B7853B34B1E9BB20B2B73
:1094700028D8174A93880B445288934224D8002452
:10948000AC4215D236F8143003F5005292B2B2F560
:10949000804F1BD20E4A9088204480B2990089B236
:1094A00000F5C04080B2FFF729FD0134A4B2E7E720
:1094B000074A93882B449380012002E000207047E4
:1094C000002070BD0020FCE70020FAE70020F8E74C
:1094D0008818002008B5044B1B7813B9FFF706FD68
:1094E00008BDFFF7BBFEF9E78818002038B5054630
:1094F00008B1002303701A4B1B783BB1184B5B88F3
:10950000012B03D9164A9288934207D0FFF7E2FF56
:109510001E20FFF7FDFD0446204638BD00211E2019
:10952000FFF7ECFC00215D20FFF7E8FC0C4B5988AD
:10953000013989B2090189B25E20FFF7DFFC012100
:109540001D20FFF7DBFCFFF757FD1E20FFF7E0FDB6
:109550000446FFF7CBFC002DDED001232B70DBE7A8
:10956000881800202DE9F04F83B001900F46154672
:109570001C46BDF834B00020FFF7CAFD824601202A
:10958000FFF7C6FD81460220FFF7C2FD804660203E
:10959000FFF7BEFD9DF830301B0103F0F00340F2F1
:1095A00001161E431CB13F2C02D93F2400E00124C8
:1095B000BBF1000F01D14FF6FF7B05F00305A400BE
:1095C000E4B22543BAF1000F36D1012419F4F47F37
:1095D00000D0002418F40E6F00D0002410F03F0FCC
:1095E00000D0002427B1019B13F0010F00D100240B
:1095F0002720FFF78DFD43F21223984200D000246C
:109600002820FFF785FDB04200D000242920FFF775
:109610007FFD584500D000241F20FFF779FD00B1E1
:1096200000243720FFF774FDA84200D0002484F006
:10963000010003B0BDE8F08F0024C7E72DE9F04F2B
:1096400083B083460F4614461D460020FFF760FD99
:1096500082460120FFF75CFD81460220FFF758FD9E
:1096600080466020FFF754FD1CB1012C02D8022473
:1096700003E01024B4F5805F04D835B10F2D05D96F
:109680000F2503E04FF48054F7E701252E0206F47E
:10969000706646F01106019405F00F0504FB05F510
:1096A0001DB1B5F5803F4CD20195013CA4B2240117
:1096B000A4B2BAF1000F48D1012519F4F47F00D00B
:1096C000002518F40E6F00D0002510F03F0F00D0D9
:1096D00000251FB11BF0010F00D100252720FFF747
:1096E00017FD43F23003984200D000252820FFF7F1
:1096F0000FFDB04200D000252920FFF709FDBDF87D
:109700000430984200D000251F20FFF701FD00B172
:1097100000255D20FFF7FCFC00B100255E20FFF76F
:10972000F7FCA04200D000252B20FFF7F1FC40F20F
:109730000113984200D0002585F0010003B0BDE878
:10974000F08F4FF6FF730193AFE70025B5E70000F8
:109750000F4AD2F8FC3043F08073C2F8FC30A2F517
:109760005D4200235360116841F0010111605268AD
:1097700001E000BF01333F2BFBD9064B5B689342EE
:1097800003D00122044B1A7070470022FAE700BF91
:1097900000ED00E0001000E08E18002000B310B5CE
:1097A0000446104B1B78A3B10F4B59680F4B1A6836
:1097B0000F4BA3FB0232920C00FB02F20A4B5B68D8
:1097C0005B1A9342FAD30AE0012002F073FFA4F57A
:1097D0007A74B4F57A7FF7D8012002F06BFF10BDE0
:1097E000704700BF8E180020001000E0D401002058
:1097F00083DE1B4310B50A4C01224FF480612046E2
:1098000002F051FE0120FFF7C9FF00224FF48061F2
:10981000204602F048FE3220FFF7C0FF10BD00BF17
:109820000018024008B510F0010F15D14FF0704339
:1098300010F0020F01D043F4005310F0040F01D0D8
:1098400043F4804310F0080F01D043F40043034A6F
:109850009361FFF7CFFF08BD014BE9E70018024015
:10986000001000F010B502460C464FF40071054898
:1098700002F019FE2009FFF7D5FF04F00F00FFF7F3
:10988000D1FF10BD0018024008B501460120FFF7C6
:10989000E9FF08BD38B50546002404E02020FFF7A5
:1098A000F3FF0134E4B20F2C06D8002DF6D0285D6A
:1098B0000028F4D12020F2E738BD10B50446014657
:1098C0000020FFF7CFFF013CE4B2012C00D910BD0E
:1098D0004FF4FA60FFF762FFF9E708B540F0800047
:1098E000FFF7EBFF08BD000010B5FFF731FF1E4C7E
:1098F00000224FF40071204602F0D5FD00224FF403
:109900008061204602F0CFFD4FF07043A3614CF21E
:109910005030FFF743FF0320FFF784FF41F2883008
:10992000FFF73CFF0320FFF77DFF9620FFF736FF90
:109930000320FFF777FF9620FFF730FF0220FFF7A5
:1099400071FF3220FFF72AFF2820FFF7B6FF08201B
:10995000FFF7B3FF0120FFF7B0FF0620FFF7ADFFD1
:109960000C20FFF7AAFF10BD0018024038B50546CD
:109970000C460020FFF7B1FF2846FFF78BFF402081
:10998000FFF7ABFF2046FFF785FF38BD48B110B5A4
:1099900004461E220021F8F7A5F941F21113238095
:1099A00010BD704700B141837047E0B141808280B3
:1099B000C3801B0C0381BDF800304381BDF8043027
:1099C0008381BDF80830C381BDF80C300382BDF837
:1099D00010304382BDF814308382BDF81830C38242
:1099E000BDF81C300383704738B110B504460D2113
:1099F0000230FEF7CFFBA08310BD7047002918BFCF
:109A0000002815D000B584468E4600230CE05A008D
:109A10001CF813100EF813103CF813100132090A49
:109A20000EF802100133DBB20E2BF0D95DF804FB07
:109A30007047000030B5039C002918BF00285ED095
:109A400086468C46002C5DD009880088091A9CED5A
:109A5000017A01F6B73541F26E70854215D8DEED18
:109A6000027A06EE901AF8EEE66A67EEA67A2068A9
:109A7000181A06EE900AF8EE666A67EEA67A9FED6F
:109A8000236AC7EE866A37EE267ADEED016ADFEDDD
:109A9000207AB4EEE77AF1EE10FA09DCDFED1D7AF8
:109AA000B4EEE77AF1EE10FA04D59FED1A7A01E0F0
:109AB0009FED177A8CED017A07EE901AF8EEE77AAF
:109AC00067EEA67AFDEEE77A17EE900A00F5004001
:109AD000BDEEC77A17EE101A0844B0F57A7F06DBA0
:109AE0004DF6E051884204DD4DF6E05001E042F2CF
:109AF0006020022A01D080B230BD2360FBE74FF422
:109B00000040F9E74FF40040F6E700BF0000C8420C
:109B10000000FA460000FAC608B5FEF791FD08BD40
:109B200008B5FFF7F9FFA0B10B4B1B8823B1013338
:109B3000094A1380002008BD01220849084805F0A1
:109B4000B7FE0028F7D10123064A1370024A13809A
:109B5000F1E70320EFE700BF901800206015002018
:109B60002C0500209218002008B50D4B1B88A3B1CE
:109B7000013B9BB20A4A13800BB100200EE0012288
:109B80000849002005F094FE18B9074B00221A700E
:109B900004E0034B01221A8000E0002008BD00BF52
:109BA000901800206015002092180020F8B50029B8
:109BB00018BF002810D0144606460F46FFF7B0FF26
:109BC000054650B922463946304605F0A1FE054605
:109BD00018B1FFF7C9FF00E013252846F8BD10B5FE
:109BE00040B106F0EEF90446FFF7BEFF04B90446A3
:109BF000204610BD0024F7E7F0B5ADF5815D87B0D4
:109C00000C4617461D46002301930122014602A877
:109C1000FFF7CCFF064620B130460DF5815D07B059
:109C2000F0BD214602A806F0E1F9064678B102A887
:109C3000FFF7D5FF41F250036B441B68002BEBD0BC
:109C4000019B41F250026A4412681360E4E701ABE1
:109C50002A46394602A805F074FF0646E7E770B5C4
:109C600078B10C460646FFF75BFF054608B128466B
:109C700070BD2146304606F00CFB0546FFF774FF29
:109C8000F5E71325F3E700B587B06946FFF7E7FF6F
:109C9000B0FA80F0400907B05DF804FB38B578B140
:109CA0000546FFF73DFF044608B1204638BD28466B
:109CB00006F073FB082800D00446FFF755FFF4E7D1
:109CC0001324F2E738B588B10546FFF729FF0446AB
:109CD00008B1204638BD284606F0FDFA031FDBB266
:109CE000012B00D90446FFF73FFFF2E71324F0E70A
:109CF00010B5044600E00134237823B10C4AD25C4D
:109D000012F0080FF7D183B12046F7F759FF013859
:109D1000204402E0002300F80139844205D2037890
:109D2000034AD35C13F0080FF4D1204610BD00BFE6
:109D3000E90D010810B504464FF4C6720021F7F78B
:109D4000D1FF012384F8D13084F8D23084F809316E
:109D500084F80B31022284F80C214FF6FF72A4F82C
:109D60000E211022A4F8102184F8123141F6FF735D
:109D7000A4F814314FF47A73A4F8863110BD002989
:109D800018BF00280DD038B5134605463BB14C1E10
:109D900022461946F8F766F900232B5538BD0370A3
:109DA000FCE7704770B5002918BF00280CBF0124DC
:109DB000002427D005460E461349F8F7D1F9E0B143
:109DC00012492846F7F768FFB8B111492846F7F756
:109DD00063FF90B10F492846F8F7C2F948B10E4920
:109DE0002846F7F759FF20B10C492846F7F754FFEA
:109DF00030B900233370012402E0012030700446A2
:109E0000204670BD0024FBE73C100108401001080B
:109E1000481001084C1001085010010858100108A2
:109E200008B50021F7F77AFA08BD08B500221146F7
:109E3000F7F784FE08BD08B500221146F7F77EFE4D
:109E400080B208BD002918BF002800F0D28270B58A
:109E500082B0144606460D46002A00F0CD80C24965
:109E60002846F8F77DF9002800F0C180BF49284650
:109E7000F8F776F9002800F0C180BD492846F8F7C8
:109E80006FF9002800F0C680BA492846F8F768F94B
:109E9000002800F0CB80B8492846F8F761F900287F
:109EA00000F0CA80B5492846F8F75AF9002800F0B2
:109EB000C980B3492846F8F753F9002800F0C88054
:109EC000B0492846F8F74CF9002800F0C780AE49A1
:109ED0002846F8F745F9002800F0C680AB49284627
:109EE000F8F73EF9002800F0C580A9492846F8F7A0
:109EF00037F9002800F0C480A6492846F8F730F961
:109F0000002800F0C380A4492846F8F729F9002862
:109F100000F0C280A1492846F8F722F9002800F095
:109F2000C1809F492846F8F71BF9002800F0C0803F
:109F30009C492846F8F714F9002800F0BF809A4998
:109F40002846F8F70DF9002800F0BE80974928460A
:109F5000F8F706F9002800F0BD8095492846F8F783
:109F6000FFF8002800F0BC8092492846F8F7F8F87E
:109F7000002800F0BB8090492846F8F7F1F8002847
:109F800000F0BA808D492846F8F7EAF8002800F07A
:109F9000B9808B492846F8F7E3F8002800F0B8802C
:109FA00088492846F8F7DCF8002800F0B780864991
:109FB0002846F8F7D5F8002800F0B68083492846EF
:109FC000F8F7CEF8002800F0B58081492846F8F768
:109FD000C7F8002840F004817E492046F7F75CFE70
:109FE000002840F0AD80002386F8083104E02246C6
:109FF00011213046FFF7C3FE02B070BD0DF107011D
:10A000002046FFF7CFFE0028F6D09DF8073086F8EF
:10A01000D130F1E70DF107012046FFF7C3FE00281C
:10A02000EAD09DF8073086F8D230E5E72046FFF702
:10A0300002FF86F8D400DFE72046FFF7FCFE86F833
:10A04000D500D9E72046FFF7F6FE86F8D600D3E71D
:10A050002046FFF7F0FE86F8D700CDE72046FFF751
:10A06000EAFE86F8D800C7E72046FFF7E4FE86F848
:10A07000D900C1E72046FFF7DEFE86F8DA00BBE72D
:10A080002046FFF7D8FE86F8DB00B5E72046FFF74D
:10A09000D2FE86F8DC00AFE72046FFF7CCFE86F85C
:10A0A000DD00A9E72046FFF7C6FE86F8DE00A3E73D
:10A0B0002046FFF7C0FE86F8DF009DE72046FFF749
:10A0C000BAFE86F8E00097E72046FFF7B4FEA6F850
:10A0D000E20091E72046FFF7AEFEA6F8E4008BE72A
:10A0E0002046FFF7A8FEA6F8E80085E72046FFF720
:10A0F000A2FEA6F8F8007FE72046FFF79CFEA6F830
:10A10000F40079E72046FFF796FEA6F8040173E70E
:10A110002046FFF785FE86ED3B0A6DE72046FFF7F8
:10A120007FFE86ED3C0A67E72046FFF779FE86ED65
:10A130003F0A61E72046FFF773FE86ED400A5BE7C2
:10A1400025492046F7F7A8FD18B9012386F80831FC
:10A1500052E722492046F7F79FFD00287FF44CAFD5
:10A16000022386F8083147E75C1001086C100108EB
:10A17000781001088810010894100108A010010847
:10A18000AC100108B8100108C4100108D010010873
:10A19000DC100108E8100108F410010800110108A2
:10A1A0000C1101081C1101082C11010838110108BB
:10A1B00044110108581101086C1101087C110108B3
:10A1C0008C1101089C110108AC110108BC11010897
:10A1D000CC110108DC110108E0110108F01101089F
:10A1E00084492846F7F7BCFF00287BD082492846DF
:10A1F000F7F7B6FF00287BD080492846F7F7B0FF75
:10A2000000287BD07E492846F7F7AAFF00287BD09C
:10A210007C492846F7F7A4FF00287BD07A492846D6
:10A22000F7F79EFF00287BD078492846F7F798FF7C
:10A2300000287BD076492846F7F792FF00287BD08C
:10A2400074492846F7F78CFF00287BD072492846CE
:10A25000F7F786FF00287CD070492846F7F780FF83
:10A2600000287CD06E492846F7F77AFF00287CD07A
:10A270006C492846F7F774FF00287CD06A492846C5
:10A28000F7F76EFF00287CD068492846F7F768FF8B
:10A2900000287CD066492846F7F762FF00287CD06A
:10A2A00064492846F7F75CFF002800F0898062497E
:10A2B0002846F7F755FF002800F088805F492846B8
:10A2C000F7F74EFF002800F087805D492846F7F732
:10A2D00047FF00287FF490AE2046FFF7ACFD86F8DC
:10A2E0008B0189E62046FFF7A6FD86F8090183E683
:10A2F0002046FFF7A0FD86F80A017DE62046FFF71D
:10A300009AFD86F80B0177E62046FFF794FD86F864
:10A310000C0171E62046FFF78EFDA6F80E016BE6F4
:10A320002046FFF788FDA6F8100165E62046FFF7F6
:10A3300082FD86F812015FE62046FFF77CFDA6F855
:10A34000140159E62246602106F58B70FFF717FDD0
:10A3500052E62046FFF76FFD86F878014CE620466E
:10A36000FFF769FD86F8790146E62046FFF75DFDB7
:10A37000C6F87C0140E62046FFF75DFD86F88001C7
:10A380003AE62046FFF757FDA6F8820134E620465C
:10A39000FFF751FD86F884012EE62046FFF74BFDBE
:10A3A000012805D0022807D0FF2386F8853123E64F
:10A3B000002386F885311FE6012386F885311BE6E8
:10A3C0002046FFF738FDA6F8860115E62046FFF780
:10A3D00032FDA6F888010FE60DF107012046FFF7D0
:10A3E000E1FC00283FF408AE9DF8073086F88A317A
:10A3F00002E67047FC1101080C1201082012010846
:10A4000034120108481201085C1201087412010894
:10A410008C120108A0120108B0120108C012010834
:10A42000D0120108E8120108FC1201080C130108FF
:10A43000241301083C13010858130108781301087C
:10A4400088130108F0B5ADF2144D0E4603AB0021A0
:10A450000391009340F2FF3304AAFFF7CDFB0028DD
:10A4600042D1039B04AD0022EA540BE0002304F820
:10A47000013B00E0013423780D2BFBD00A2BF9D0EF
:10A480000DE025462B785BB318492846F7F7D8FF2F
:10A4900004460028EAD12846F7F792FB2C182846F4
:10A4A000FFF726FC05460378232B18BF002BE8D0C6
:10A4B0003B2BE6D03D21F5F7E7FE07460028E0D02C
:10A4C000002307F8013B2846FFF712FC05463846F3
:10A4D000FFF70EFC024629463046FFF7B3FCD0E7F3
:10A4E00001200DF2144DF0BD0020FAE7EC13010835
:10A4F0002DE9F04FADF2144D0023039331B107461F
:10A50000904689464E48FFF7BEFB20B900200DF269
:10A51000144DBDE8F08F03AB009340F2FF3304AA63
:10A5200000214748FFF768FB002840F08580039B27
:10A5300004AD0026EE5414E0002304F8013B00E0D3
:10A54000013423780D2BFBD00A2BF9D017E0DFF86C
:10A55000F8B09AF800301BB1BE423DD00136B6B219
:10A5600025462B78002B60D036492846F7F768FF40
:10A5700004460028E0D12846F7F722FB2C1828468D
:10A58000FFF7B6FB05460378232B18BF002BE7D057
:10A590003B2BE5D02C21F5F777FE82460028DFD053
:10A5A00000230AF8013B2C215046F5F76DFE834647
:10A5B00008B1002303702846FFF79AFB0546504672
:10A5C000FFF796FB8246BBF1000FC0D00BF10100F4
:10A5D000FFF78EFB8346BCE74846FFF7ABFB2A46F6
:10A5E00011214846FFF7CBFB5246602109F11100CB
:10A5F000FFF7C5FB5A46602109F17100FFF7BFFB69
:10A600005A46602109F58B70FFF7B9FB4946504661
:10A61000FFF718FF00283FF47AAFB8F1000F3FF4BE
:10A6200076AF0136A8F8006071E7B8F1000F05D0E9
:10A63000A8F8006000206AE7002068E7002066E7CD
:10A640002C100108EC130108BC14010810B582B0ED
:10A650000C460023ADF806300DF1060201461846FF
:10A66000FFF746FF10B10CB10023238002B010BDEC
:10A67000F0B583B00023ADF80630994218BF984278
:10A6800003D10025284603B0F0BD06460F460488D6
:10A690000134A4B20DF106022046FFF729FF05465A
:10A6A00070B9BDF80630002BECD0002239461046B8
:10A6B000FFF71EFF0028E5D0002232800546E1E7C3
:10A6C0003480DFE7014B83F83C0170479438002069
:10A6D0000A4B1B5C13F0070F0CD12D2814BF00236D
:10A6E0000123202808D03BB95F2801D00020704703
:10A6F000012070470120704701207047E90D0108D3
:10A70000034B0022DA701A7583F87420704700BF7B
:10A710009418002008B54FF4055200210148F7F7BE
:10A72000E1FA08BD941800202DE9F041002818BF77
:10A73000102994BF0127002732D9144680460AB950
:10A740002FE00134237823B1174AD35C13F0080FAC
:10A75000F7D12046F7F734FA204400E0013884426C
:10A7600006D210F8013C104AD35C13F0080FF5D163
:10A77000051B6B1E0F2B14D80026AE4206D2A05D1F
:10A78000FFF7A6FF074660B10136F6E72A462146E5
:10A790004046F7F7CDFB002308F80530012700E01D
:10A7A00000273846BDE8F081E90D010810B50C46D8
:10A7B000F7F7A4FEA04234BF002401240028D8BF2C
:10A7C00044F001040CB9002010BD0720FFF77AFF08
:10A7D000FAE7000030B587B00546012410E00320F9
:10A7E000FFF770FF034639E00320FFF76BFF0346D6
:10A7F00034E01E4B002283F874202BE00134A4B215
:10A8000042F20F739C422CD82346194A6021194802
:10A81000FFF7CCFF034608BB69461648FFF71FFA4F
:10A820000028EBD0031FDBB2012BD8D8002DE0D0DD
:10A830002346114A60211148FFF7B8FF034668B963
:10A8400069460E48FFF70BFA0028D7D0031FDBB28A
:10A85000012BC9D80020FFF735FF0346184607B083
:10A8600030BD0720FFF72EFF0346F7E794180020BE
:10A87000A4130108A8180020BC130108081900201F
:10A8800010B50B4B9B781BB9094B5B783BB910BDDE
:10A890000848FFF7A4F9064B00229A70F4E7064C2B
:10A8A0002046FFF79CF9002304F8DB3CEFE700BFEC
:10A8B00094180020A02900207019002008B5084B2A
:10A8C00093F874301BB9064B1B7D23B908BD0548AE
:10A8D000FFF7F8F9F7E70448FFF7F4F9F6E700BFE8
:10A8E0009418002008190020A818002008B5FFF7C8
:10A8F000C7FFFFF7E3FF074B00221A70A3F8D4202D
:10A90000A3F8D620A3F8D820A3F8DA20FFF7F8FEA2
:10A9100008BD00BF9418002008B51C48FFF7BEF919
:10A9200008BB1B4BB3F8D6301BB11A48FFF7B6F97A
:10A93000E8B919490A2201F1C800FFF737F9D0B97F
:10A94000134B01225A70B3F8D63043B10A2213498F
:10A950001348FFF72BF990B90D4B01229A70002094
:10A96000FFF7B0FE08BD0620FFF7ACFEFAE70620B1
:10A97000FFF7A8FEF6E70820FFF7A4FEF2E7FFF7CF
:10A98000B5FF0820FFF79EFEECE700BFD0130108DB
:10A9900094180020DC130108A818002008190020D2
:10A9A000A029002070B582B01C46BDF818500023C5
:10A9B0000193994218BF984218D00E46B5FA85F314
:10A9C0005B099CB193B90B882B44934213D801AB1C
:10A9D0002A46214605F0A1F910B9019B9D4210D0ED
:10A9E000FFF784FF0920FFF76DFE02E00120FFF76B
:10A9F00069FE02B070BDFFF779FF0B20FFF762FE22
:10AA0000F7E733882B4433800020FFF75BFEF0E745
:10AA100030B5ADF5885D81B000230393224B03F17F
:10AA20007102019203F111020092204AC0210DF53A
:10AA30008250F7F763FD431EBE2B17D8044612223F
:10AA40001B4904A8FFF7B2F8B8B9079904A805F0A4
:10AA5000CDFA0546A8B104A8FFF7C1F815B9039BC4
:10AA60009C421DD00A20FFF72DFE02E00A20FFF7CE
:10AA700029FE0DF5885D01B030BD0A20FFF722FEEA
:10AA8000F7E703AB22460DF5825104A805F045F91E
:10AA900005460028DFD104A805F047FA0546DAE7A5
:10AAA0000020FFF70FFEE4E797180020E4130108E9
:10AAB0002C10010808B5FFF72DFE08BD014B1878D2
:10AAC000704700BF94180020014B93F83C01704779
:10AAD0009438002070B505460C461646FFF7EEFF89
:10AAE00078B9FFF717FEFFF717F870B12CB12A46B7
:10AAF00011211A48FFF718FE58B90220FFF7E2FDAE
:10AB000070BD0420FFF7DEFDFAE70320FFF7DAFD52
:10AB1000F6E7134BA3F8D440A3F8D66001221A70CD
:10AB20003046FFF757FE38B10D4B00221A7003F57F
:10AB3000005393F83C01E3E7FFF7EEFE18B900205D
:10AB4000FFF7C0FDDCE7064C00232370FFF7D8FDBC
:10AB500004F5005494F83C01D2E700BF9718002098
:10AB60009418002000B583B01B4B1B7893B1002ACA
:10AB700018BF002912D0162A10D8012816D0022892
:10AB800002D1154B9B78E3B9FFF7B0FE0C20FFF71D
:10AB900099FD08E00520FFF795FD04E0FFF7A6FE0C
:10ABA0000120FFF78FFD03B05DF804FB0A48009217
:10ABB0000B46B0F8D42000F1D801DC30FFF7F2FEEC
:10ABC000F1E7054800920B46B0F8D62000F1DA0113
:10ABD0000248FFF7E7FEE6E794180020A0290020CE
:10ABE00010B5284B1B7833B3264BD3F8D820D3F8B5
:10ABF000D4309A4223D1234B5B7833BB214B9B78D3
:10AC00001BB1214805F091F950BBFFF739FEFFF762
:10AC1000FFFE58BB1B4B00241C70A3F8D440A3F8C4
:10AC2000D640A3F8D840A3F8DA40FFF769FD2046E4
:10AC3000FFF748FD10BD0520FFF744FDFAE7FFF7D9
:10AC400055FE0B20FFF73EFDF4E7104805F06DF9C7
:10AC50000028D3D0FFF74AFE0920FFF733FDE9E7CC
:10AC6000FFF744FE0920FFF72DFDE3E7FFF726FE7F
:10AC7000044C00232370FFF743FD04F5005494F8BF
:10AC80003C01D7E794180020A0290020701900206B
:10AC900008B5054B1B7823B9044B002283F83C21EF
:10ACA00008BDFFF723FEF7E7941800209438002032
:10ACB000014B01221A707047DC390020002302E0AA
:10ACC0002022C25401330F2BFAD90023037431B16F
:10ACD0000F2B04D8CA5C12B1C2540133F8E7704795
:10ACE000012803D0032803D1024870470248704767
:10ACF00002487047F8130108F01301080014010816
:10AD000088B108B50346084A12783AB9074A12785A
:10AD1000012A01D0064902E0064900E0024918462E
:10AD2000FFF7CCFF08BD7047E0390020DF39002075
:10AD3000081401081414010808B330B589B0054699
:10AD40000F4B1C787CB90F4B1878FFF7C9FF0346EF
:10AD50000D4A112103A8F7F7D1FB03A92846FFF7F5
:10AD6000ADFF09B030BD074B1878FFF7B9FF0346B8
:10AD70000094064A112103A8F7F7C0FBEDE77047DE
:10AD8000DE390020DF390020241401082C140108CA
:10AD90000A4B1B7803B9704700B58BB005A8FFF7C5
:10ADA000AFFF6846FFF7C8FF694605A8FEF7DEFD5E
:10ADB000034B00221A700BB05DF804FBDD39002054
:10ADC000DC39002010B50E4B00241C605C609C60D8
:10ADD000DC601C740B4B1C700B4B1C70FDF72AFBCA
:10ADE000FDF73AFC094B187058705C60FEF77CFD6B
:10ADF0000123074A1370074A1370FFF7C9FF10BDFC
:10AE0000E0390020DF390020DE390020D43900206D
:10AE1000DD390020DC39002010B586B00023019315
:10AE20000293039304938DF8143020B1014610224D
:10AE300001A8F7F717F9112201A90948F7F746F910
:10AE400008B906B010BD064C0DF1040CBCE80F00AB
:10AE50000FC4DCF800302370FFF72AFFF1E700BFD2
:10AE6000E039002002280AD008B5054B1B78834240
:10AE700000D108BD024B1870FFF71AFFF9E77047C1
:10AE8000DF39002008B5054B1B78834200D108BD8F
:10AE9000024B1870FFF70CFFF9E700BFDE39002006
:10AEA00038B5154B1C780CB9204638BD0546FDF762
:10AEB000D3FB124A127882420AD0104A10705560B1
:10AEC00000240F4B1B78002BEED0FFF761FFEBE760
:10AED0000A4B5868281A022807D95B789A4206D08C
:10AEE000064B5A702AB90024EBE70024E9E7002456
:10AEF000E7E70124E5E700BFDD390020D439002071
:10AF0000DC3900204A4B5A6822F440325A605A68B1
:10AF100041680A435A600268536823F4807353609F
:10AF200002685368016943EA012353600268536869
:10AF300023F0407353600268536881680B43536089
:10AF40000268936823F40063936002689368C168A1
:10AF50000B439360826A374B9A4257D002689368DA
:10AF600023F07063936002689368816A0B43936077
:10AF70000268936823F04053936002689368C16A43
:10AF80000B4393600268936823F0020393600268A6
:10AF90009368816943EA4103936090F82030002B65
:10AFA0003FD00268536843F40063536002685368FB
:10AFB00023F46043536001684B68426A013A43EAF4
:10AFC00042334B600268D36A23F47003D362016892
:10AFD000CB6AC269013A43EA0253CB6202689368C2
:10AFE00023F4007393600268936890F8301043EA8A
:10AFF000412393600268936823F48063936002683E
:10B000009368416943EA81239360704702689368BB
:10B0100023F0706393600268936823F04053936059
:10B02000B0E70268536823F400635360CAE700BFC7
:10B03000002301400100000F28B310B50446036C43
:10B0400043B1236C13F0100F0BD00120002384F8C0
:10B050003C3010BDFBF74AFC0023636484F83C30AD
:10B06000EFE7226C094B134043F0020323642046B0
:10B07000FFF748FF00206064236C23F0030343F0D4
:10B0800001032364E2E70120704700BFFDEEFFFFEC
:10B0900082B00023019390F83C30012B7ED0012335
:10B0A00080F83C3003689A6812F0010F13D19A6857
:10B0B00042F001029A603D4B1B683D4AA2FB03230C
:10B0C0009B0C03EB4303019302E0019B013B0193C3
:10B0D000019B002BF9D103689A6812F0010F52D03E
:10B0E000016C344A0A4042F4807202645A6812F4D5
:10B0F000806F05D0026C22F4405242F48052026408
:10B10000026C12F4805F19D0426C22F00602426495
:10B11000002280F83C206FF022021A60264B5B6808
:10B1200013F01F0F0DD103689A6812F0405F37D1FA
:10B130009A6842F080429A6000202DE0002242642A
:10B14000E6E703681D4A93420AD01B4B5B6813F085
:10B15000100F27D103681A4A93420AD000201BE03F
:10B160009A6812F0405FF0D19A6842F080429A608B
:10B17000EBE79A6812F0405F16D19A6842F080427D
:10B180009A60002008E0036C43F010030364436CF2
:10B1900043F001034364002002B070470220FBE744
:10B1A0000020F9E70020F7E70020F5E7D4010020B0
:10B1B00083DE1B43FEF8FFFF002301400020014017
:10B1C0000022014090F83C30012B17D0012380F879
:10B1D0003C300268936823F00103936003689B6826
:10B1E00013F0010F05D1026C054B134043F001032E
:10B1F0000364002380F83C301846704702207047F3
:10B20000FEEEFFFF70B504460D4603689A6812F41F
:10B21000806F03D09B6813F4807F19D101F044FA4A
:10B22000064623681A6812F0020F20D1B5F1FF3FDD
:10B23000F7D0B5B923681B6813F0020FF1D1236C66
:10B2400043F004032364002384F83C30032033E0FC
:10B25000036C43F020030364002380F83C3001209A
:10B260002AE001F021FA801BA842DAD9E2E76FF068
:10B2700012021A60236C43F40073236423689A68F3
:10B2800012F0405F17D1A269BAB9DA6A12F4700FEE
:10B2900003D09B6813F4806F11D1236C23F4807367
:10B2A0002364236C13F4805F0BD1236C43F0010300
:10B2B0002364002000E0002070BD0020FCE7002097
:10B2C000FAE70020F8E70368D86C704770477047CA
:10B2D000704770B5044603681E685D68C5F3401288
:10B2E00012EA56022CD0026C12F0100F03D1026C3D
:10B2F00042F4007202649A6812F0405F19D1A269A8
:10B30000BAB9DA6A12F4700F03D09A6812F4806F37
:10B310000FD15A6822F020025A60236C23F4807304
:10B320002364236C13F4805F03D1236C43F0010387
:10B3300023642046FFF7CAFF23686FF012021A60E9
:10B34000C5F3C01313EA960335D0236C13F0100F26
:10B3500003D1236C43F40053236423689A6812F4E6
:10B36000401F21D19A6B12F4401F03D09A6812F447
:10B37000806F19D15A6812F4806F15D19A6812F053
:10B38000405F11D1A2697AB95A6822F080025A60EE
:10B39000236C23F480532364236C13F4807F03D144
:10B3A000236C43F001032364204600F01FF9236857
:10B3B0006FF00C021A60C5F380131E4204D023689C
:10B3C0001B6813F0010F05D1C5F3806515EA56150A
:10B3D0000CD170BD236C43F4803323642046FFF707
:10B3E00076FF23686FF001021A60EDE7636C43F0AB
:10B3F0000203636423686FF020051D602046FFF799
:10B4000067FF23681D60E4E730B482B00022019238
:10B4100090F83C20012A00F0DC800346012280F8ED
:10B420003C200A68B2F1004F18BF092A22D90468EB
:10B43000E06892B202EB42021E3A4FF0070C0CFA9F
:10B4400002F220EA0202E2600A68634882420AD0FD
:10B450001D68E8688C6892B202EB42021E3A944082
:10B460002043E8601CE01868C2688C6842EA046205
:10B47000C26015E00468206992B202EB42024FF00C
:10B48000070C0CFA02F220EA020222611C68206911
:10B490000A8802EB42028D6805FA02F20243226139
:10B4A0004A68062A29D81C68606B02EB8202053ABA
:10B4B0004FF01F0C0CFA02F220EA020262631C68D1
:10B4C000606B4A6802EB8202053AB1F800C00CFAE0
:10B4D00002F2024362631868404A90423DD0186805
:10B4E0003E4A904243D018683C4A90424CD00020DB
:10B4F00083F83C0002B030BC70470C2A16D81D6897
:10B50000286B02EB8202233A1F2404FA02F220EA9B
:10B5100002022A631D68286B4A6802EB8202233A02
:10B520000C8804FA02F202432A63D4E71D68E86A31
:10B5300002EB8202413A1F2404FA02F220EA0202DC
:10B54000EA621D68E86A4A6802EB8202413A0C88A6
:10B5500004FA02F20243EA62BDE70A68B2F1004F60
:10B56000BDD11F48426822F440024260B7E70A6832
:10B57000122AB8D11A4A506820F40000506050686E
:10B5800040F480005060AEE70A681348112A18BFE3
:10B590008242ACD1124A506820F48000506050685A
:10B5A00040F40000506009680B4A91429FD10D4A57
:10B5B00012680D49A1FB0212920C02EB82025200AA
:10B5C000019202E0019A013A0192019A002AF9D10E
:10B5D0008DE702208EE700BF12000010002001401E
:10B5E00000230140D401002083DE1B43704700008C
:10B5F000002800F0068270B582B00446036813F09C
:10B60000010F29D0954B9B6803F00C03042B1AD033
:10B61000924B9B6803F00C03082B0FD06368B3F5C3
:10B62000803F40D0002B54D18C4B1A6822F48032DA
:10B630001A601A6822F480221A6039E0874B5B682E
:10B6400013F4800FEAD0854B1B6813F4003F03D03E
:10B650006368002B00F0D781236813F0020F74D0C9
:10B660007E4B9B6813F00C0F5ED07C4B9B6803F005
:10B670000C03082B53D0E368002B00F08980774A35
:10B68000136843F00103136001F00EF80546734B95
:10B690001B6813F0020F72D101F006F8401B02285C
:10B6A000F5D90320B4E16D4A136843F48033136085
:10B6B00063682BB300F0F8FF0546684B1B6813F472
:10B6C000003FC9D100F0F0FF401B6428F5D90320EA
:10B6D0009EE1B3F5A02F09D0604B1A6822F48032A6
:10B6E0001A601A6822F480221A60E1E75B4B1A683C
:10B6F00042F480221A601A6842F480321A60D7E756
:10B7000000F0D2FF0546554B1B6813F4003FA3D051
:10B7100000F0CAFF401B6428F5D9032078E14F4BA5
:10B720005B6813F4800FA6D14C4B1B6813F0020F1B
:10B7300003D0E368012B40F06881484A136823F086
:10B74000F803216943EAC1031360236813F0080F6B
:10B7500046D0636983B3414A536F43F00103536793
:10B7600000F0A2FF05463D4B5B6F13F0020F37D18F
:10B7700000F09AFF401B0228F5D9032048E1374A20
:10B78000136823F0F803216943EAC1031360DCE77F
:10B79000324A136823F00103136000F085FF054669
:10B7A0002E4B1B6813F0020FCFD000F07DFF401B23
:10B7B0000228F5D903202BE1284A536F23F0010317
:10B7C000536700F071FF0546244B5B6F13F0020FC7
:10B7D00006D000F069FF401B0228F5D9032017E1CD
:10B7E000236813F0040F7DD01C4B1B6C13F0805F9B
:10B7F0001ED11A4B1A6C42F080521A641B6C03F073
:10B8000080530193019B0125154B1B6813F4807F26
:10B8100010D0A368012B25D0002B3BD10F4B1A6F02
:10B8200022F001021A671A6F22F004021A671EE062
:10B830000025E9E70A4A136843F48073136000F0B7
:10B8400033FF0646064B1B6813F4807FE1D100F0FE
:10B850002BFF801B6428F5D90320D9E00038024073
:10B8600000700040724A136F43F001031367A3682E
:10B8700033B300F019FF06466D4B1B6F13F0020F38
:10B880002FD100F011FF801B41F288339842F3D989
:10B890000320BDE0052B09D0654B1A6F22F0010291
:10B8A0001A671A6F22F004021A67E0E7604B1A6FFA
:10B8B00042F004021A671A6F42F001021A67D6E7D3
:10B8C00000F0F2FE06465A4B1B6F13F0020F08D031
:10B8D00000F0EAFE801B41F288339842F3D903203E
:10B8E00096E0FDB9A369002B00F09180504A926860
:10B8F00002F00C02082A59D0022B19D04C4A1368C6
:10B9000023F08073136000F0CFFE0446484B1B68A1
:10B9100013F0007F48D000F0C7FE001B0228F5D9C5
:10B92000032075E0424A136C23F080531364D9E777
:10B930003F4A136823F08073136000F0B5FE05469C
:10B940003B4B1B6813F0007F06D000F0ADFE401BA0
:10B950000228F5D903205BE0E369226A1343626A97
:10B9600043EA8213A26A5208013A43EA0243E26AB6
:10B9700043EA0263226B43EA02732D4A5360136861
:10B9800043F08073136000F08FFE0446284B1B6861
:10B9900013F0007F06D100F087FE001B0228F5D9C6
:10B9A000032035E0002033E0002031E0204A5268D7
:10B9B000012B2FD002F48003E1698B422CD102F0DD
:10B9C0003F03216A8B4229D1616A47F6C073134055
:10B9D000B3EB811F24D102F44031A36A5B08013B21
:10B9E000B1EB034F1ED102F07063E16AB3EB016F5C
:10B9F0001AD102F0E042236BB2EB037F16D1002094
:10BA000006E001207047012002E0012000E0002054
:10BA100002B070BD0120FBE70120F9E70120F7E744
:10BA20000120F5E70120F3E70120F1E70120EFE72E
:10BA30000038024008B5264B9B6803F00C03042B2A
:10BA400041D0082B41D1224B5A6802F03F025B687B
:10BA500013F4800F12D01E4B5968C1F388111D4892
:10BA60000023A1FB0001F9F7C1FC194B5B68C3F38C
:10BA7000014301335B00B0FBF3F008BD144B586881
:10BA8000C0F388104FEA401CBCEB000C6EEB0E0EAE
:10BA90004FEA8E1343EA9C634FEA8C11B1EB0C0121
:10BAA00063EB0E03DB0043EA5173C90011EB000C9A
:10BAB00043F10003990200234FEA8C2041EA9C5194
:10BAC000F9F794FCD1E70348D7E70348D5E700BF6F
:10BAD0000038024040787D010024F400002800F086
:10BAE000A08070B50D460446524B1B6803F00F034F
:10BAF0008B420BD24F4A136823F00F030B431360A2
:10BB0000136803F00F038B4240F08D80236813F01D
:10BB1000020F17D013F0040F04D0474A936843F480
:10BB2000E0539360236813F0080F04D0424A9368EF
:10BB300043F460439360404A936823F0F003A168A4
:10BB40000B439360236813F0010F31D06368012B1E
:10BB500020D0022B25D0384A126812F0020F64D090
:10BB600035498A6822F0030213438B6000F09CFD84
:10BB70000646314B9B6803F00C036268B3EB820FFF
:10BB800016D000F091FD801B41F288339842F0D925
:10BB9000032045E0284A126812F4003FE0D101205A
:10BBA0003EE0254A126812F0007FD9D1012037E02B
:10BBB000204B1B6803F00F03AB420AD91D4A1368E0
:10BBC00023F00F032B431360136803F00F03AB4202
:10BBD0002DD1236813F0040F06D0174A936823F47D
:10BBE000E053E1680B439360236813F0080F07D01C
:10BBF000114A936823F46043216943EAC1039360C7
:10BC0000FFF718FF0C4B9B68C3F303130B4AD35C7D
:10BC1000D8400B4B18600B4B186800F007FD002054
:10BC200070BD012070470120FAE70120F8E70120EC
:10BC3000F6E700BF003C02400038024098170108B8
:10BC4000D4010020D0010020014B1868704700BFCC
:10BC5000D401002008B5FFF7F7FF044B9B68C3F33E
:10BC60008223034AD35CD84008BD00BF003802409D
:10BC70009017010808B5FFF7E7FF044B9B68C3F373
:10BC80004233034AD35CD84008BD00BF00380240AD
:10BC900090170108F0B583B00446066816F0010657
:10BCA0000DD0B54B9A6822F400029A609A68416BF5
:10BCB0000A439A60436B002B00F0678100262568D9
:10BCC00015F4002511D0AC4AD2F88C3023F440137F
:10BCD000E16B0B43C2F88C30E36BB3F5801F00F0CF
:10BCE0005681002B00F055810025236813F4801F36
:10BCF0000FD0A14AD2F88C3023F44003216C0B43BF
:10BD0000C2F88C30236CB3F5800F00F0448103B986
:10BD10000125236813F0807F00D0012613F0200F47
:10BD200040F03B81236813F0100F0CD0924BD3F8F6
:10BD30008C2022F08072C3F88C20D3F88C20A16B69
:10BD40000A43C3F88C20236813F4804F08D08A4A32
:10BD5000D2F8903023F44033616E0B43C2F8903038
:10BD6000236813F4004F08D0834AD2F8903023F4AC
:10BD70004023A16E0B43C2F89030236813F4803F38
:10BD800008D07D4AD2F8903023F44013E16E0B4383
:10BD9000C2F89030236813F4003F08D0764AD2F8F6
:10BDA000903023F44003216F0B43C2F89030236896
:10BDB00013F0400F08D0704AD2F8903023F00303FC
:10BDC000616C0B43C2F89030236813F0800F08D0E9
:10BDD000694AD2F8903023F00C03A16C0B43C2F8EF
:10BDE0009030236813F4807F08D0634AD2F89030F3
:10BDF00023F03003E16C0B43C2F89030236813F456
:10BE0000007F08D05C4AD2F8903023F0C003216D47
:10BE10000B43C2F89030236813F4806F08D0564A61
:10BE2000D2F8903023F44073616D0B43C2F8903028
:10BE3000236813F4006F08D04F4AD2F8903023F4EF
:10BE40004063A16D0B43C2F89030236813F4805F08
:10BE500008D0494AD2F8903023F44053E16D0B43A7
:10BE6000C2F89030236813F4005F08D0424AD2F839
:10BE7000903023F44043216E0B43C2F89030236886
:10BE800013F4800F08D03C4AD2F8903023F080633E
:10BE9000A16F0B43C2F89030236813F4001F0DD03C
:10BEA000354AD2F8903023F00063E16F0B43C2F8BB
:10BEB0009030E36FB3F1006F00F0D580236813F08A
:10BEC000080F00D0012513F4802F08D02A4AD2F899
:10BED000903023F04073616F0B43C2F890302368B9
:10BEE00013F4000F09D0244AD2F8903023F0805385
:10BEF000D4F880100B43C2F89030236813F0806FA1
:10BF000009D01D4AD2F8903023F00053D4F88410A1
:10BF10000B43C2F89030236813F0006F09D0164A23
:10BF2000D2F88C3023F00073D4F888100B43C2F899
:10BF30008C30236813F0805F09D00F4AD2F88C3020
:10BF400023F08063D4F88C100B43C2F88C3026B9F0
:10BF5000236813F0007F00F00681074A136823F07E
:10BF60008063136000F0A0FB0646034B1B6813F0D0
:10BF7000006F7AD002E000BF0038024000F094FB6E
:10BF8000801B6428F1D90320F0E0012697E6012602
:10BF9000A7E60125A9E60126B9E67F4B1A6C42F017
:10BFA00080521A641B6C03F080530193019B7B4AFF
:10BFB000136843F48073136000F076FB0746774BF9
:10BFC0001B6813F4807F06D100F06EFBC01B642851
:10BFD000F5D90320CAE0704B1B6F13F4407315D0E2
:10BFE000226B02F440729A4210D06B4B1A6F22F40B
:10BFF0004072196F41F480311967196F21F4803153
:10C0000019671A671B6F13F0010F12D1236B03F42A
:10C010004072B2F5407F1DD05F4A936823F4F81355
:10C0200093605D490B6F226BC2F30B0213430B67E6
:10C0300078E600F039FB0746574B1B6F13F0020FF1
:10C04000E4D100F031FBC01B41F288339842F3D9B0
:10C0500003208BE05048826822F4F81250491940BE
:10C060000A438260DDE7012528E7236813F0010F0A
:10C0700013D0636B8BB9484AD2F88430D2F884105D
:10C08000606803F4403343EA801301F070610B43AE
:10C09000A16843EA0173C2F88430236813F4002FC7
:10C0A00003D0E26BB2F5801F06D013F4801F1ED0C0
:10C0B000236CB3F5800F1AD1374AD2F88430D2F806
:10C0C0008410606803F4403343EA8013E06843EA75
:10C0D000006301F0E0410B43C2F88430D2F88C30A9
:10C0E00023F01F03616A01390B43C2F88C302368C7
:10C0F00013F0807F11D0284AD2F88400D2F884103F
:10C10000666823691B0443EA861300F070600343EA
:10C1100001F0E0410B43C2F88430236813F0007F44
:10C120000DD0626823691B0443EA8213E26843EA84
:10C130000263A26843EA0273174AC2F88430164ABF
:10C14000136843F08063136000F0AEFA0646124BAA
:10C150001B6813F0006F06D100F0A6FA801B64285C
:10C16000F5D9032002E0012D02D0002003B0F0BD7C
:10C17000094A136823F08053136000F095FA0546CE
:10C18000054B1B6813F0005F0CD000F08DFA401BCC
:10C190006428F5D90320E9E7003802400070004028
:10C1A000FFFCFF0F236813F4002F01D0E26B22B1D4
:10C1B00013F4801F1DD0236CDBB9354AD2F88830C8
:10C1C000D2F88810606903F4403343EA8013A06911
:10C1D00043EA006301F0E0410B43C2F88830D2F833
:10C1E0008C3023F4F853A16A013943EA0123C2F8E1
:10C1F0008C30236813F4001F03D0E36FB3F1006F9A
:10C2000031D0236813F0080F19D0214AD2F88810D2
:10C21000D2F88830606903F4403343EA801301F0B8
:10C2200070610B43E16943EA0173C2F88830D2F8C8
:10C230008C3023F44033E16A0B43C2F88C30144A4B
:10C24000136843F08053136000F02EFA0446104B3D
:10C250001B6813F0005F19D100F026FA001B642858
:10C26000F5D9032082E70A4AD2F88800D2F888106C
:10C270006569236A1B0443EA851300F07060034379
:10C2800001F0E0410B43C2F88830BAE700206DE7C7
:10C290000038024000230F2B00F2F48070B582B00A
:10C2A00066E085684FEA430E032404FA0EF425EA9B
:10C2B0000405CC6804FA0EF42C438460446824EA34
:10C2C00002044A68C2F300129A40224342605DE0D1
:10C2D000DC08083450F8242003F00705AD004FF0C7
:10C2E0000F0E0EFA05FE22EA0E0E0A69AA4042EA75
:10C2F0000E0240F824205DE0092200E0002202FA4C
:10C300000EF22A430234604D45F824205F4A9468B7
:10C310006FEA0C0224EA0C054E6816F4801F01D067
:10C320004CEA0405594CA560E46802EA04054E682D
:10C3300016F4001F01D04CEA0405544CE560646813
:10C3400002EA04054E6816F4003F01D04CEA0405E9
:10C350004E4C6560246822404D6815F4803F01D042
:10C360004CEA0402494C226001330F2B00F2888012
:10C3700001229A400C6804EA020C32EA0404F3D168
:10C380004C6804F00304013C012C8AD94A6802F08D
:10C390000302032A09D0C4685D000322AA4024EAEC
:10C3A00002048A68AA402243C2604A6802F003027B
:10C3B000022A8DD004684FEA430E032202FA0EF2DD
:10C3C00024EA02044A6802F0030202FA0EF222434F
:10C3D00002604A6812F4403FC6D02D4A546C44F4BF
:10C3E00080445464526C02F480420192019A9C0889
:10C3F000A51C254A52F8255003F0030E4FEA8E0E75
:10C400000F2202FA0EF225EA0205224A90423FF478
:10C4100075AF02F58062904222D002F580629042B0
:10C4200020D002F5806290421ED002F580629042D8
:10C430001CD002F5806290421AD002F580629042D0
:10C4400018D002F58062904216D002F580629042C8
:10C4500014D002F5806290423FF44EAF0A224EE7BC
:10C4600001224CE702224AE7032248E7042246E77A
:10C47000052244E7062242E7072240E708223EE77A
:10C4800002B070BD704700BF00380140003C014061
:10C4900000380240000002400369194201D0012027
:10C4A0007047002070470AB18161704709048161BB
:10C4B0007047436901EA030221EA030141EA0241AC
:10C4C0008161704710B582B01B4B1A6C42F08052EC
:10C4D0001A641B6C03F080530193019B174A136885
:10C4E00043F48033136000F0DFF80446134B5B68BD
:10C4F00013F4803F08D100F0D7F8001BB0F57A7F25
:10C50000F4D9032002B010BD0C4A136843F4003381
:10C51000136000F0C9F80446084B5B6813F4003F51
:10C5200007D100F0C1F8001BB0F57A7FF4D90320E1
:10C53000E8E70020E6E700BF003802400070004056
:10C54000002804DB0901C9B2044B1954704700F0FC
:10C550000F000901C9B2024B1954704700E400E012
:10C5600014ED00E000B500F00700C0F1070CBCF1CD
:10C57000040F28BF4FF0040C031D062B0FD9C31E58
:10C580004FF0FF3E0EFA0CF021EA000199400EFA3E
:10C5900003FE22EA0E0241EA02005DF804FB0023DA
:10C5A000EEE700000649CB6823F4E0631B041B0C94
:10C5B000000200F4E0600343024A1A43CA60704775
:10C5C00000ED00E00000FA0510B50446054BD86800
:10C5D000C0F30220FFF7C6FF01462046FFF7B0FF79
:10C5E00010BD00BF00ED00E0002807DB00F01F02D7
:10C5F000400901239340024A42F82030704700BFAF
:10C6000000E100E00138B0F1807F0BD24FF0E02371
:10C610005861054AF02182F8231000209861072212
:10C620001A6170470120704700ED00E010B5044624
:10C630000E4B1A784FF47A73B3FBF2F30C4A10687E
:10C64000B0FBF3F0FFF7DEFF68B90F2C01D9012032
:10C650000AE0002221464FF0FF30FFF7B5FF054BFF
:10C660001C60002000E0012010BD00BFCE010020B2
:10C67000D4010020D001002008B50320FFF792FF6D
:10C680000020FFF7D3FFFAF719F9002008BD0000DA
:10C69000034A1168034B1B780B441360704700BFBB
:10C6A000F4390020CE010020014B1868704700BF0C
:10C6B000F439002038B50446FFF7F6FF0546B4F11B
:10C6C000FF3F02D0044B1B781C44FFF7EDFF401BDB
:10C6D000A042FAD338BD00BFCE010020034B9B68B7
:10C6E000C3F30313024AD35CD840704700380240BA
:10C6F00098170108034B9B68C3F38223024AD35C5B
:10C70000D84070470038024090170108034B9B68DF
:10C71000C3F34233024AD35CD8407047003802402A
:10C72000901701080D4B5B6803F480039BB90C481C
:10C730000A4B5A6802F03F02B0FBF2F05A68C2F3AB
:10C74000881202FB00F05B68C3F3014301335B0016
:10C75000B0FBF3F070470348EAE700BF003802403F
:10C760000024F40040787D0108B5074B9B6803F076
:10C770000C03042B04D0082B04D1FFF7D3FF08BD12
:10C780000248FCE70248FAE70038024040787D01A1
:10C790000024F40008B5032808D00C282ED0B0F5EA
:10C7A000406F53D030287AD0002008BD514BD3F8C9
:10C7B0009030034043EA00434F4A934208D0B3F11C
:10C7C000031F0CD0013A934211D1FFF7CDFFECE7E4
:10C7D000484B186810F00200E7D04848E5E7454BA1
:10C7E000186F10F00200E0D04FF40040DDE7FFF7D3
:10C7F000BBFFFFF773FFFFF789FFD6E73D4BD3F889
:10C800009030034043EA00433D4A934208D0B3F1DD
:10C810000C1F0CD0043A934211D1FFF7A5FFC4E7D7
:10C82000344B186810F00200BFD03448BDE7314BDC
:10C83000186F10F00200B8D04FF40040B5E7FFF7D2
:10C8400093FFFFF74BFFFFF755FFAEE7294BD3F8F8
:10C850009030034043EA00432A4A934209D0B3F19F
:10C860000C2F0DD0A2F58062934211D1FFF77CFF0F
:10C870009BE7204B186810F0020096D01F4894E701
:10C880001C4B186F10F002008FD04FF400408CE763
:10C89000FFF76AFFFFF722FFFFF738FF85E7154B29
:10C8A000D3F89030034043EA0043174A934208D03C
:10C8B000B3F1301F0DD0103A934213D1FFF754FF5C
:10C8C00073E70C4B186810F002003FF46EAF0B4892
:10C8D0006BE7084B186F10F002003FF466AF4FF49F
:10C8E000004062E7FFF740FFFFF7F8FEFFF702FFA7
:10C8F0005BE700BF00380240020003000024F400A0
:10C9000008000C000008000C2000300008B5C0280A
:10C910000AD0B0F5407F2FD0B0F5405F55D0B0F5CC
:10C92000404F7BD0002008BD524BD3F890300340DD
:10C9300043EA0043504A934208D0B3F1C01F0CD0E1
:10C94000403A934211D1FFF70FFFECE7494B1868CB
:10C9500010F00200E7D04948E5E7464B186F10F0A9
:10C960000200E0D04FF40040DDE7FFF7FDFEFFF7E7
:10C97000B5FEFFF7BFFED6E73E4BD3F8903003403D
:10C9800043EA00433E4A934209D0B3F1032F0DD04E
:10C99000A2F58072934211D1FFF7E6FEC3E7354B53
:10C9A000186810F00200BED03448BCE7314B186F55
:10C9B00010F00200B7D04FF40040B4E7FFF7D4FE08
:10C9C000FFF78CFEFFF796FEADE72A4BD3F89030C9
:10C9D000034043EA00432B4A934209D0B3F1302F7E
:10C9E0000DD0A2F58052934211D1FFF7BDFE9AE718
:10C9F000204B186810F0020095D0204893E71D4B9B
:10CA0000186F10F002008ED04FF400408BE7FFF754
:10CA1000ABFEFFF763FEFFF76DFE84E7154BD3F81F
:10CA20009030034043EA0043174A934209D0B3F1E0
:10CA3000C02F0ED0A2F58042934213D1FFF794FE8F
:10CA400071E70C4B186810F002003FF46CAF0B4814
:10CA500069E7084B186F10F002003FF464AF4FF421
:10CA6000004060E7FFF780FEFFF738FEFFF742FE69
:10CA700059E700BF003802408000C0000024F400E5
:10CA80000002000300200030008000C000B5836871
:10CA900091FAA1FCBCFA8CFC4FEA4C0C4FF0030E4F
:10CAA0000EFA0CFC23EA0C0391FAA1F1B1FA81F120
:10CAB00049008A40134383605DF804FB00B5C368F6
:10CAC00091FAA1FCBCFA8CFC4FEA4C0C4FF0030E1F
:10CAD0000EFA0CFC23EA0C0391FAA1F1B1FA81F1F0
:10CAE00049008A401343C3605DF804FB00B5036A44
:10CAF00091FAA1FCBCFA8CFC4FEA8C0C4FF00F0EA3
:10CB00000EFA0CFC23EA0C0391FAA1F1B1FA81F1BF
:10CB100089008A40134303625DF804FB00B5436A51
:10CB2000090A91FAA1FCBCFA8CFC4FEA8C0C4FF07C
:10CB30000F0E0EFA0CFC23EA0C0391FAA1F1B1FAE4
:10CB400081F189008A40134343625DF804FB00B51C
:10CB5000036891FAA1FCBCFA8CFC4FEA4C0C4FF034
:10CB6000030E0EFA0CFC23EA0C0391FAA1F1B1FAC0
:10CB700081F149008A40134303605DF804FBF8B576
:10CB800007460E460D6895FAA5F5B5FA85F519E044
:10CB9000B26821463846FFF779FF3268F1687B6852
:10CBA00023EA020301FB02F213437B6016E0726981
:10CBB00021463846FFF7B2FF726821463846FFF734
:10CBC000C6FF0135346834FA05F21BD00122AA40B1
:10CBD0001440F6D07368013B012BD9D93269214644
:10CBE0003846FFF76BFF7368022BE5D194FAA4F384
:10CBF000B3FA83F3072BDAD8726921463846FFF778
:10CC000075FFD9E70020F8BD0B4B1B680B4AA2FB50
:10CC100003235B0A41F2883202FB03F31A46013B0D
:10CC20003AB1426B12F0800FF8D0C5238363002025
:10CC300070474FF000407047D4010020D34D621080
:10CC400084B00DF1040C8CE80E000B461343039ADC
:10CC50001343049A1343059A1343069A13434168F6
:10CC6000034A0A4013434360002004B0704700BFEA
:10CC70000081FFFFD0F8800070470B68C0F880305B
:10CC8000002070470323036000207047006800F015
:10CC9000030070470B6883604B688A681343CA6857
:10CCA00013430A691343C2686FF30B021343C36053
:10CCB000002070470069C0B2704714304058704778
:10CCC0000B6843624B6883628B68CA6813430A69C6
:10CCD00013434A691343C26A22F0F7021343C36243
:10CCE0000020704710B586B00446002301930293DC
:10CCF000039304934FF48063059301A9FFF7CAFFE0
:10CD00002046FFF781FF06B010BD000038B504468D
:10CD10000D46504B1B685049A1FB03135B0A03FBF4
:10CD200002F21346013A002B5DD0636B13F0450FFE
:10CD3000F7D013F4006FF4D1636B13F0040F06D136
:10CD4000636B13F0010F05D00120A0634DE00420B8
:10CD5000A0634AE0C523A3632046FFF7ABFFA842C8
:10CD600001D0012041E000212046FFF7A6FF034645
:10CD70003A481840C8B3002B38DB13F0804F38D145
:10CD800013F0005F37D113F0805F36D113F0006FDE
:10CD900036D113F0806F36D113F0807F36D113F483
:10CDA000000F36D113F4800F36D113F4001F36D1A3
:10CDB00013F4801F36D113F4802F36D113F4003FC3
:10CDC00036D113F4803F36D113F4004F36D113F42B
:10CDD000804F36D113F4005F36D113F0080F36D0F0
:10CDE0004FF4000001E04FF0004038BD4FF00070FC
:10CDF000FBE74020F9E78020F7E74FF48070F4E785
:10CE00004FF40070F1E74FF48060EEE74FF40060FC
:10CE1000EBE74FF48050E8E74FF40050E5E74FF4BC
:10CE20008040E2E74FF40040DFE74FF40030DCE7FA
:10CE30004FF48020D9E74FF40020D6E74FF480105C
:10CE4000D3E74FF40010D0E74FF48000CDE74FF464
:10CE50008030CAE7D4010020D34D621008E0FFFD06
:10CE600030B587B004460191102502954023039305
:10CE7000002304934FF48063059301A9FFF70AFF91
:10CE800041F2883229462046FFF740FF07B030BD07
:10CE900030B587B0044601911125029540230393D4
:10CEA000002304934FF48063059301A9FFF7F2FE7A
:10CEB00041F2883229462046FFF728FF07B030BDEF
:10CEC00030B587B0044601911225029540230393A3
:10CED000002304934FF48063059301A9FFF7DAFE62
:10CEE00041F2883229462046FFF710FF07B030BDD7
:10CEF00030B587B00446019118250295402303936D
:10CF0000002304934FF48063059301A9FFF7C2FE49
:10CF100041F2883229462046FFF7F8FE07B030BDBF
:10CF200030B587B00446019119250295402303933B
:10CF3000002304934FF48063059301A9FFF7AAFE31
:10CF400041F2883229462046FFF7E0FE07B030BDA7
:10CF500030B587B00446002301930C25029540228A
:10CF6000039204934FF48063059301A9FFF792FEA7
:10CF7000034A29462046FFF7C9FE07B030BD00BF6F
:10CF800000E1F50530B587B004460192072502950A
:10CF900040230393002304934FF48063059301A976
:10CFA000FFF778FE41F2883229462046FFF7AEFEB1
:10CFB00007B030BD30B587B00446019137250295E2
:10CFC00040230393002304934FF48063059301A946
:10CFD000FFF760FE41F2883229462046FFF796FEB1
:10CFE00007B030BD30B587B0044601910D250295DC
:10CFF00040230393002304934FF48063059301A916
:10D00000FFF748FE41F2883229462046FFF77EFEB0
:10D0100007B030BD0146144B1B68144AA2FB032322
:10D020005B0A41F2883202FB03F31A46013BBAB1B4
:10D030004A6B12F0450FF8D012F4006FF5D14B6B2C
:10D0400013F0040F06D1486B10F0010005D1C52381
:10D050008B637047042088637047012088637047A2
:10D060004FF00040704700BFD4010020D34D621044
:10D0700010B586B004460023019302220292C0221A
:10D08000039204934FF48063059301A9FFF702FE16
:10D090002046FFF7BFFF06B010BD10B586B00446AE
:10D0A000019109230293C0230393002304934FF4B7
:10D0B0008063059301A9FFF7EDFD2046FFF7AAFF66
:10D0C00006B010BD0146104B1B68104AA2FB03239B
:10D0D0005B0A41F2883202FB03F31A46013B82B13C
:10D0E0004A6B12F0450FF8D012F4006FF5D1486B7F
:10D0F00010F0040002D1C5238B63704704208863BD
:10D1000070474FF000407047D4010020D34D6210AB
:10D1100010B586B004460A4B0B43019329230293B2
:10D1200040230393002304934FF48063059301A9E4
:10D13000FFF7B0FD2046FFF7C5FF06B010BD00BFEA
:10D1400000001080F8B505460E461746234B1B68B5
:10D15000234AA2FB03235B0A41F2883202FB03F35A
:10D160001A46013B8AB36C6B14F0450FF8D014F4E7
:10D17000006FF5D16B6B13F0040F06D16B6B13F0DE
:10D18000010F05D00120A86321E00420A8631EE060
:10D190002846FFF78FFDB04201D0012017E0C523DC
:10D1A000AB6300212846FFF788FD034610F460407A
:10D1B00008D013F4804F0BD113F4004F0BD04FF471
:10D1C000805004E01B0C3B8001E04FF00040F8BDB4
:10D1D0004FF40050FBE74FF48030F8E7D401002013
:10D1E000D34D621070B586B004460D4600230193FE
:10D1F000032602964022039204934FF48063059322
:10D2000001A9FFF747FD2A4631462046FFF79AFF5E
:10D2100006B070BD0146164B1B68164AA2FB0323DD
:10D220005B0A41F2883202FB03F31A46013BE2B18A
:10D230004A6B12F0450FF8D012F4006FF5D14B6B2A
:10D2400013F0040F0BD14B6B13F001030AD1486BA1
:10D2500010F040000BD040228A631846704704202B
:10D26000886370470120886370474FF00040704723
:10D27000D4010020D34D621010B586B004464FF49F
:10D28000D57301930823029340230393002304934F
:10D290004FF48063059301A9FFF7FCFC2046FFF7DC
:10D2A000B9FF06B010BD000070B582B0044600237F
:10D2B00001930068FFF716FD054610B1284602B03D
:10D2C00070BD2068FFF7D8FF38B90123A364A36CB1
:10D2D000012B0BD02E46284614E00023A3642068BF
:10D2E000FFF700FD0028F2D00546E7E7002120689F
:10D2F000FFF760FE0028EDD04FF08055DEE7019B80
:10D3000001330193019A4FF6FE739A4213D896B9EE
:10D3100000212068FFF74EFEE0B912492068FFF7B0
:10D32000F7FE0646C0B900212068FFF7C6FCC30F10
:10D33000E5D01E46E3E7019A4FF6FE739A420ED8F7
:10D3400010F0804302D001236364B7E700226264D7
:10D350001D46B3E70546B1E74FF08055AEE74FF005
:10D360008075ABE7000010C170B581B104460E4670
:10D37000016D09040068FFF735FE054608B128462F
:10D3800070BD00212068FFF798FC3060F7E74FF090
:10D390000065F4E72DE9F04F87B005460C461646C8
:10D3A0009B46DDF840A0FFF77FF9002C36D0814680
:10D3B00095F83470FFB2012F40F004810023AB6375
:10D3C00006EB0B03EA6D93422ED8032385F8343025
:10D3D0002B680022DA626B6C012B00D076024FF0D2
:10D3E000FF3300934FEA4B230193902302930223D0
:10D3F0000393002304930123059369462868FFF7EC
:10D400005FFCBBF1010F14D902232B63314628685E
:10D41000FFF756FDA0B9DDF8048038E0AB6B43F0B0
:10D420000063AB630127D2E0AB6B43F00073AB63E7
:10D43000CDE001232B6331462868FFF729FDE9E79A
:10D440002B68654A9A63AB6B0343AB63012385F892
:10D45000343000232B63BAE02868FFF70BFC207000
:10D46000C0F307236370C0F30743A370000EE0709E
:10D470000434A8F104080136072EEDD9FFF714F99A
:10D48000A0EB090050450FD2BAF1000F0CD028686C
:10D49000466B16F4957615D1436B13F4004FEDD01F
:10D4A000B8F1000FEAD0E7E72B684B4A9A63AB6B01
:10D4B00043F00043AB63012385F8343000232B6332
:10D4C000032784E0436B13F4807F05D0BBF1010F89
:10D4D00002D96B6C032B38D12B685A6B12F0080FF2
:10D4E00044D15A6B12F0020F4CD15A6B12F0200F3C
:10D4F00054D12868436B13F4001F5BD0B8F1000FC0
:10D5000058D0FFF7B7FB2070C0F307236370C0F358
:10D510000743A370000EE0700434A8F10408FFF77D
:10D52000C3F8A0EB0900504502D2BAF1000FE0D1D8
:10D530002B68294A9A63AB6B43F00043AB6301232A
:10D5400085F8343000232B6341E0FFF701FD0346EB
:10D550000028C1D02A6820499163AA6B1343AB63AA
:10D56000012385F8343000232B6330E01A4A9A6394
:10D57000AB6B43F00803AB63012385F83430002321
:10D580002B6324E0144A9A63AB6B43F00203AB6352
:10D59000012385F8343000232B6318E00E4A9A6388
:10D5A000AB6B43F02003AB63012385F834300023D9
:10D5B0002B630CE040F23A538363012385F8343047
:10D5C000002704E0AB6B43F00053AB630127384600
:10D5D00007B0BDE8F08F00BFFF0540002DE9F04F18
:10D5E0008BB005460C4616469B46DDF850A0FFF76B
:10D5F0005BF8002C37D0804695F83470FFB2012FCD
:10D6000040F0E1800023AB6306EB0B03EA6D93422D
:10D610002FD8032385F834302B680022DA626B6C34
:10D62000012B00D076024FF0FF3304934FEA4B23D7
:10D6300005939023069300230793089301230993EE
:10D6400004A92868FFF73CFBBBF1010F16D9202382
:10D650002B6331462868FFF763FC0190019BABB94F
:10D66000DDF8149040E0AB6B43F00063AB6301273F
:10D67000AEE0AB6B43F00073AB63A9E010232B6308
:10D6800031462868FFF734FC0190E7E72B68524ADF
:10D690009A63AB6B019A1343AB63012385F8343073
:10D6A00000232B6394E023780393627843EA0223F8
:10D6B0000393A27843EA02430393E27843EA0263C6
:10D6C00003930434A9F1040903A92868FFF7D5FAE4
:10D6D0000136072EE7D9FEF7E7FFA0EB080050451B
:10D6E0000FD2BAF1000F0CD02868466B16F48D7675
:10D6F00015D1436B13F4804FEDD0B9F1000FEAD090
:10D70000E7E72B68344A9A63AB6B019A1343AB6328
:10D71000012385F8343000232B63032758E0436B43
:10D7200013F4807F05D0BBF1010F02D96B6C032B82
:10D7300018D12B685A6B12F0080F24D15A6B12F0D3
:10D74000020F2CD15A6B12F0100F34D0224A9A6378
:10D75000AB6B43F01003AB63012385F83430002337
:10D760002B6335E0FFF7F4FB03460028E1D02A687D
:10D7700019499163AA6B1343AB63012385F83430D5
:10D7800000232B6324E0144A9A63AB6B43F0080335
:10D79000AB63012385F8343000232B6318E00E4A75
:10D7A0009A63AB6B43F00203AB63012385F834301B
:10D7B00000232B630CE040F23A529A63012385F870
:10D7C0003430002704E0AB6B43F00053AB63012718
:10D7D00038460BB0BDE8F08FFF0540000346426EAF
:10D7E000920F0A70426EC2F383624A7090F867200B
:10D7F00002F003028A7090F86620CA7090F86520E3
:10D800000A7190F864204A71826E120DCA80B0F8D5
:10D810006A2002F00F020A72826EC2F3C0324A72AC
:10D82000826EC2F380328A72826EC2F34032CA7252
:10D83000826EC2F300320A7300224A73426C002ADD
:10D8400040F08680806E40F6FC7202EA8002D86E5C
:10D8500042EA90720A61DA6EC2F3C2620A7593F804
:10D860006F2002F007024A75DA6EC2F342528A75DF
:10D87000DA6EC2F38242CA75DA6EC2F3C2320A7637
:10D880000A6901325A65087E00F0070002308240C2
:10D890005A6591F808C00CF00F0C012000FA0CF04A
:10D8A0009865400A00FB02F2DA654FF400721A66CE
:10D8B000DA6EC2F380324A76DA6EC2F3C6128A7624
:10D8C000DA6E02F07F02CA761A6FD20F0A771A6FE9
:10D8D000C2F341724A771A6FC2F382628A771A6F73
:10D8E000C2F38352CA771A6FC2F3405281F82020E4
:10D8F000002081F82100B3F8722002F0010281F8C3
:10D9000022201A6FC2F3C03281F823201A6FC2F3AB
:10D91000803281F824201A6FC2F3403281F825202A
:10D920001A6FC2F3003281F826201A6FC2F38122E7
:10D9300081F827201A6FC2F3012281F828201B6F7B
:10D94000C3F3460381F82930012381F82A30704758
:10D95000012A11D1826E120402F47C12B0F86E001A
:10D9600002430A610A69013292025A65DA654FF48C
:10D9700000729A651A669BE7026805499163826B9B
:10D9800042F080528263012083F83400704700BF68
:10D99000FF05400070B590B004460123ADF8123089
:10D9A0000068FFF773F900286CD0636C032B45D136
:10D9B000636C032B5DD1636C032B1DD0BDF812107B
:10D9C000216509042068FFF768FB054600285BD144
:10D9D00000212068FFF771F9606604212068FFF7D5
:10D9E0006CF9A06608212068FFF767F9E0660C2152
:10D9F0002068FFF762F9206704212068FFF75DF9CE
:10DA0000000DE06405A92046FFF7E8FE00283ED19E
:10DA1000226D120400232068FFF7B4FA054698BB74
:10DA2000234653F8106B93E807008DE80700043491
:10DA300094E80E003046FFF703F925E02068FFF771
:10DA400017FB054600BB00212068FFF736F9606729
:10DA500004212068FFF731F9A06708212068FFF74B
:10DA60002CF9E0670C212068FFF727F9C4F8800043
:10DA70009EE70DF112012068FFF7B4FB0546002870
:10DA800099D001E04FF08065284610B070BD4FF08E
:10DA90008055F9E730B58BB0044600230493059315
:10DAA000069307930893762309930AAB13E90700BB
:10DAB0008DE8070004AB0ECB2068FFF7C1F818B162
:10DAC000012528460BB030BD05462268536823F473
:10DAD000807353602068FFF7D5F82268536843F4D9
:10DAE000807353600220FEF7E5FD2046FFF7DCFB64
:10DAF00030B1012584F83450A36B0343A363E0E7FE
:10DB00002046FFF747FF30B1012584F83450A36B5E
:10DB10000343A363D5E74FF400712068FFF7A0F932
:10DB20000028CED0236804499963A36B0343A36301
:10DB3000012584F83450C4E7FF054000A8B110B5B2
:10DB4000044690F8343063B1032384F8343020461F
:10DB5000FFF7A0FF58B9A0632063012384F8343095
:10DB600010BD0377F8F74AFFEEE701207047012068
:10DB7000F6E7436C0B60836C4B60C36C8B60036D8A
:10DB8000CB60436D0B61836D4B61C36D8B61036E25
:10DB9000CB610020704710B582B00446002301938A
:10DBA00001A9FFF7E1FB10B1A36B0343A363019845
:10DBB000C0F3432002B010BD0346026812F0400FCC
:10DBC00036D110B402681D4810400A684C682243E0
:10DBD000CC6822430C6922434C6922438C6922435E
:10DBE000CC6922430C6A2243104318605868144AD7
:10DBF00002408868B1F816C040EA0C0002435A603F
:10DC00008A68B2F5006F03D25A6842F480525A60B3
:10DC10000A6AB2F5005F07D00020DA6922F40062D8
:10DC2000DA615DF8044B70478A8C1A610020F4E7D2
:10DC30000120DA6922F40062DA6170474000FFFFD8
:10DC4000FBF0FFFF70B4046A036A23F00103036270
:10DC500042688569124B2B400D681D4324F0020475
:10DC60008B6823430F4C104EB04218BFA0420CBF2C
:10DC70000124002405D123F00803CE681E4326F0BA
:10DC800004032CB122F440724C6914438A69224384
:10DC9000426085614A684263036270BC704700BF9E
:10DCA0008CFFFEFF000001400004014070B4036AD5
:10DCB000026A22F4807202624268C569144C2C40E8
:10DCC0000E68264323F400738C6843EA0423114C46
:10DCD000114DA84218BFA0420CBF0124002406D158
:10DCE00023F40063CD6843EA052323F480633CB149
:10DCF00022F440524C6942EA04128C6942EA04124E
:10DD00004260C6614A68C263036270BC704700BF6C
:10DD10008CFFFEFF000001400004014070B4036A64
:10DD2000026A22F4805202624468C5690D4A2A40A0
:10DD30000D6842EA052223F400538D6843EA053357
:10DD4000094E0A4DA84218BFB04204D124F48044C1
:10DD50004D6944EA85144460C2614A680264036202
:10DD600070BC7047FF8CFFFE0000014000040140C2
:10DD700070B4036A026A22F4803202624468426D1F
:10DD80000D4D15400A682A4323F400338D6843EA99
:10DD900005430A4E0A4DA84218BFB04204D124F4EC
:10DDA00080344D6944EA0524446042654A688265CE
:10DDB000036270BC704700BF8FFFFEFF0000014090
:10DDC0000004014070B4036A026A22F48012026205
:10DDD0004468456D0D4A2A400D6842EA052223F445
:10DDE00000138D6843EA0553094E0A4DA84218BF37
:10DDF000B04204D124F480244D6944EA852444606F
:10DE000042654A68C265036270BC7047FF8FFFFEBF
:10DE1000000001400004014010B4036A046A24F0C9
:10DE200001040462846924F0F00C4CEA021223F02D
:10DE30000A030B43826103625DF8044B704710B420
:10DE4000036A046A24F010040462846924F4704CA8
:10DE50004CEA023223F0A00343EA01138261036219
:10DE60005DF8044B7047836823F070030B4343F065
:10DE7000070383607047704730B503683F4A90429C
:10DE800014BF4FF0000E4FF0010EB0F1804F14BFE1
:10DE900072464EF00102AAB9394CA04214BF0024C8
:10DEA0000124384DA8420DD064B904F1804404F532
:10DEB0008234A04214BF0024012405F50065A84265
:10DEC00000D01CB123F070034C682343002A33D1E7
:10DED0002B4A904214BF002201222A4CA0422BD090
:10DEE00052BB02F1804202F58232904214BF0022FE
:10DEF000012204F50064A0421ED0EAB9224A9042F1
:10DF000014BF0022012204F59A34A04214D09AB919
:10DF10001E4A904214BF0022012204F50064A04270
:10DF20000AD04AB91A4A904214BF00220122A4F52D
:10DF30009634A04200D022B123F4407CCB6843EA5F
:10DF40000C0323F080034A69134303608A68C262AA
:10DF50000A6882620F4A904214BF73464EF0010372
:10DF60000BB10B69036301234361036913F0010FD4
:10DF700003D0036923F00103036130BD00000140B9
:10DF80000008004000040040004401400018004028
:10DF9000002000400004014060B310B5044690F832
:10DFA0003D3013B3022384F83D30214651F8040B71
:10DFB000FFF762FF012384F8483084F83E3084F88C
:10DFC0003F3084F8403084F8413084F8423084F89F
:10DFD000433084F8443084F8453084F8463084F87F
:10DFE000473084F83D30002010BD80F83C30F8F711
:10DFF00061FDD7E70120704760B310B5044690F883
:10E000003D3013B3022384F83D30214651F8040B10
:10E01000FFF732FF012384F8483084F83E3084F85B
:10E020003F3084F8403084F8413084F8423084F83E
:10E03000433084F8443084F8453084F8463084F81E
:10E04000473084F83D30002010BD80F83C30FFF7A9
:10E0500012FFD7E70120704770B4036A026A22F00A
:10E060001002026242688569144C2C400D6844EA33
:10E07000052523F020038C6843EA0413104C114E4D
:10E08000B04218BFA0420CBF0124002406D123F0E7
:10E090008003CE6843EA061323F040033CB122F428
:10E0A00040624C6942EA84028C6942EA840242601E
:10E0B00085614A688263036270BC7047FF8CFFFE13
:10E0C000000001400004014038B590F83C30012BBD
:10E0D00000F0958004460D46012380F83C30142A58
:10E0E00000F28880DFE802F00B8686861F8686862F
:10E0F00034868686488686865D86868671000068B8
:10E10000FFF7A0FD2268936943F00803936122683A
:10E11000936923F0040393612268936929690B438F
:10E120009361002067E00068FFF796FF226893691B
:10E1300043F4006393612268936923F480639361DD
:10E1400022689369296943EA01239361002052E020
:10E150000068FFF7ABFD2268D36943F00803D36181
:10E160002268D36923F00403D3612268D369296943
:10E170000B43D36100203EE00068FFF7CFFD22682B
:10E18000D36943F40063D3612268D36923F48063C5
:10E19000D3612268D369296943EA0123D36100204E
:10E1A00029E00068FFF7E4FD2268536D43F008039F
:10E1B00053652268536D23F0040353652268536D41
:10E1C00029690B435365002015E00068FFF7FAFD4D
:10E1D0002268536D43F4006353652268536D23F442
:10E1E000806353652268536D296943EA01235365AF
:10E1F000002000E00120002384F83C3038BD0220DC
:10E20000FCE710B4846824F47F4C42EA03220A43FA
:10E2100042EA0C0282605DF8044B704790F83C3093
:10E22000012B76D010B50446012380F83C30022340
:10E2300080F83D3002689068374B034093600B686C
:10E24000602B4CD023D8402B54D011D8202B03D096
:10E250000AD80BB1102B05D119462068FFF703FE31
:10E26000002028E0012026E0302BF5D0012022E01C
:10E27000502B0AD1CA6849682068FFF7CDFD5021AC
:10E280002068FFF7F0FD002015E0012013E0B3F552
:10E29000805F3AD0B3F5005F14D0702B37D1CB68D4
:10E2A0004A6889682068FFF7ACFF2268936843F0EA
:10E2B000770393600020012384F83D30002384F825
:10E2C0003C3010BDCB684A6889682068FFF799FF29
:10E2D0002268936843F4804393600020EBE7CA68A8
:10E2E00049682068FFF7ABFD60212068FFF7BBFDA0
:10E2F0000020E0E7CA6849682068FFF78DFD4021EB
:10E300002068FFF7B0FD0020D5E70020D3E701200B
:10E31000D1E70220704700BF8800FEFF01F01F0117
:10E320004FF0010C0CFA01FC036A23EA0C030362B0
:10E33000036A8A40134303627047000010B5044625
:10E3400010293CD8DFE801F0093B3B3B1F3B3B3B3E
:10E35000263B3B3B2D3B3B3B340090F83E30DBB251
:10E36000013B18BF0123002B40F08980102974D88D
:10E37000DFE801F02C7373736373737367737373E4
:10E380006B7373736F0090F83F30DBB2013B18BFC3
:10E390000123E8E790F84030DBB2013B18BF0123CE
:10E3A000E1E790F84130DBB2013B18BF0123DAE727
:10E3B00090F84230DBB2013B18BF0123D3E790F85D
:10E3C0004330DBB2013B18BF0123CCE7022384F8C2
:10E3D0003E3001222068FFF7A1FF23682A492B4A1B
:10E3E000934218BF8B4203D15A6C42F400425A64E4
:10E3F0002368254AB3F1804F18BF934231D0A2F56C
:10E400007C4293422DD002F58062934229D002F5DE
:10E410008062934225D002F57842934221D002F5E2
:10E42000705293421DD0A2F59432934219D01A68CB
:10E4300042F001021A60002022E0022384F83F30FB
:10E44000C7E7022384F84030C3E7022384F8413051
:10E45000BFE7022384F84230BBE7022384F843304D
:10E46000B7E799680A4A0A40062A18BFB2F5803F02
:10E4700007D01A6842F001021A60002000E0012073
:10E4800010BD0020FCE700BF000001400004014077
:10E490000700010090F83C30012B3CD030B402461C
:10E4A000012380F83C30CB6823F440738868034331
:10E4B00023F480634868034323F40063086803433C
:10E4C00023F480530869034323F40053486903434A
:10E4D00023F48043886A034323F47023886943EA62
:10E4E000004310680D4D0E4CA04218BFA8420CD13D
:10E4F00023F470034C6A43EA045323F08073CC691D
:10E50000234323F00073096A0B434364002082F81D
:10E510003C0030BC70470220704700BF0000014043
:10E520000004014030B503683B4A904214BF4FF0ED
:10E53000000E4FF0010EB0F1804F14BF72464EF046
:10E540000102AAB9354CA04214BF00240124344D65
:10E55000A8420DD064B904F1804404F58234A0428D
:10E5600014BF0024012405F50065A84200D01CB1A9
:10E5700023F070034C682343002A33D1274A90428A
:10E5800014BF00220122264CA0422BD052BB02F124
:10E59000804202F58232904214BF0022012204F52B
:10E5A0000064A0421ED0EAB91E4A904214BF002265
:10E5B000012204F59A34A04214D09AB91A4A904222
:10E5C00014BF0022012204F50064A0420AD04AB917
:10E5D000164A904214BF00220122A4F59634A042AC
:10E5E00000D022B123F4407CCB684CEA03030360E3
:10E5F0008A68C2620A8882620D4A904214BF7346DA
:10E600004EF001030BB10B690363436943F001034F
:10E610004361002030BD00BF000001400008004001
:10E620000004004000440140001800400020004069
:10E6300000040140B2F5004F06D001EB5301B1FBDD
:10E64000F3F189B2C16070475A0802EB4102B2FB94
:10E65000F3F34FF6F0721A40C3F342031343C3605F
:10E660007047000038B5036813F0010F62D104460B
:10E670000D460368314A1A404B68C9680B43296943
:10E680000B43A9690B431A430260AB68426822F44A
:10E690004052134343606B69826822F44072134313
:10E6A0008360274B984216D0264B98421BD0264BAE
:10E6B00098421CD0254B98421DD0254B98421ED025
:10E6C000244B984220D0244B984222D0234B98428E
:10E6D00024D001202FE00320FEF75CF860B32B6804
:10E6E0000BBB012027E00C20FEF754F8F6E73020A2
:10E6F000FEF750F8F2E7C020FEF708F9EEE74FF416
:10E700004070FEF703F9E9E74FF44060FEF742F886
:10E71000E4E74FF44050FEF7F9F8DFE74FF44040EC
:10E72000FEF7F4F8DAE7AA6901462046FFF782FF10
:10E73000002000E0012038BD0120FCE7F369FFEF75
:10E74000001001400044004000480040004C0040E0
:10E75000005000400014014000780040007C004060
:10E76000034AD2F8883043F47003C2F88830704707
:10E7700000ED00E008B5044B03EB800252685268DC
:10E780000344187A904708BD203A002008B5084B8A
:10E790001B5C53B9064B01221A5403EB80025268EA
:10E7A00012680344187A904708BD0020FCE700BFB8
:10E7B000203A002038B5044C04EB80056D68AD6844
:10E7C0000444207AA84738BD203A002038B5044CCC
:10E7D00004EB80056D68ED680444207AA84738BDD5
:10E7E000203A002010B5044B03EB800464682469D0
:10E7F0000344187AA04710BD203A002042780078E0
:10E8000040EA02207047C378827842EA03224378C4
:10E8100043EA0223007840EA032070470170090AA6
:10E82000417070470170C1F307234370C1F3074380
:10E830008370090EC1707047944632B10A78013175
:10E8400002700130BCF1010CF8D170470170013049
:10E85000013AFBD1704784469CF800000CF1010C92
:10E860000B780131C01A013A01D00028F4D070476A
:10E87000034600E00133187808B18842FAD17047A6
:10E8800010B44FF0000C634602E04FF0010C01336E
:10E89000012B15D81A01184CA258002AF5D004688B
:10E8A000A242F4D1144A02EB0312546882689442E3
:10E8B000EDD1114A02EB0312946842699442E6D109
:10E8C000022B0BD0B1B90C4A02EB03139B89B3F5B1
:10E8D000807F0DD000205DF8044B7047022914BFE3
:10E8E00063464CF001030BB10020F4E71220F2E77D
:10E8F0001020F0E71020EEE7F8390020002000E0BB
:10E900000130012804D80301034AD358002BF7D162
:10E91000023818BF01207047F839002070B4002376
:10E9200000E00133012B13D81A01234CA4580268CC
:10E930009442F6D1204A02EB031254688268944252
:10E94000EFD11D4A02EB0312946842699442E8D168
:10E95000022B08D0F9B1184A02EB031292894ABB84
:10E960004FF480721DE00023012B05D81A01124CD0
:10E97000A2580AB10133F7E7022B19D00E4D1C0142
:10E9800005EB031206682E5184685460406990605C
:10E9900000209081DEE7084A02EB031292890132DF
:10E9A00092B2054901EB03118A81581C70BC704773
:10E9B0000020FBE70020F9E7F839002001380128A2
:10E9C00015D80D4B03EB00139B89B3F5807F03D063
:10E9D00043B1013B9BB200E00023074A02EB001267
:10E9E000938133B903010020034AD05070470220BD
:10E9F00070470020704700BFF8390020002303E073
:10EA00005DF8044B70470133012B11D81A010949F5
:10EA10008A588242F7D110B41A0100248C50013375
:10EA2000012BEDD81A0103498A588242F7D1F3E746
:10EA3000704700BFF839002002398369023B8B42DE
:10EA400004D94389C06A01FB030070470020704766
:10EA50000268C36A04339089B1FBF0F15289B1FBBB
:10EA6000F2F101E0091A0833186818B18142F9D2AD
:10EA700058680844704770B506460D4601F11A0003
:10EA8000FFF7BCFE3378032B00D070BD044605F1C0
:10EA90001400FFF7B3FE44EA0040F6E770B50646FF
:10EAA0000C46154691B204F11A00FFF7B7FE337811
:10EAB000032B00D070BD290C04F11400FFF7AEFE4B
:10EAC000F8E738B500234B72C36973B305460C46AB
:10EAD0000022134606E0BCF1090F0FD0A1184B72BB
:10EAE000013263460A2B0ED803F1010C296ACB5C74
:10EAF000202BF6D0052BEED1E523ECE7A1182E2034
:10EB000048720132EAE72244002353722B6ADB7A0F
:10EB10002372286A1C30FFF776FE2060286A1630C0
:10EB2000FFF771FEE080000CA08038BD2DE9F84FA2
:10EB300081468A46D1F8008000F1240B0B22202167
:10EB40005846FFF783FE00252B46082729E00136AB
:10EB500018F806302F2BFAD05C2BF8D04644CAF8B0
:10EB60000060002D44D099F82430E52B35D0202CBE
:10EB700037D8042389F82F30002035E014F0800FB7
:10EB800027D121461B48FFF773FE78BBA4F1610330
:10EB9000DBB2192B01D8203CE4B20BF8054001355B
:10EBA00033465E1C18F80340202CD7D95C2C18BFC4
:10EBB0002F2CCDD02E2C18BFAF42DFD82E3C18BF43
:10EBC00001240B2F08BF44F0010464B908250B276A
:10EBD000E6E7803C084B1C5DD3E7052389F8243029
:10EBE000C5E70023C6E70620BDE8F88F0620FBE74F
:10EBF0000620F9E738140108A81701080146006843
:10EC000008B1024603E04FF0FF307047013213783D
:10EC1000202B01D93A2BF9D13A2B01D00020704793
:10EC2000034613F8010B3038092898BF9A4203D1E4
:10EC300028B901320A6070474FF0FF3070474FF03B
:10EC4000FF30704738B50D46044698B103689BB154
:10EC50001A78A2B18188DA88914203D00920002471
:10EC60002C6038BD5878FFF785FD10F0010009D100
:10EC70002468F5E70920F3E71C460920F0E709209E
:10EC80000024EDE709200024EAE72DE9F041C578EA
:10EC900015B92846BDE8F0810446076B00F1340839
:10ECA00001233A4641464078FFF790FD0546A0B95A
:10ECB0000023E370636AFB1AE2699342E9D2A67803
:10ECC00008E0E3691F4401233A4641466078FFF7B4
:10ECD0007DFD013E012EF4D8DBE70125D9E770B5B3
:10ECE000036B8B4202D10026304670BD04460D46B0
:10ECF000FFF7CBFF06460028F6D101232A4604F190
:10ED000034016078FFF756FD10B101264FF0FF3552
:10ED10002563E9E738B504460023C3704FF0FF339D
:10ED20000363FFF7DCFF30BB054604F23220FFF738
:10ED300065FD4AF6552398421FD194F83430E92BEB
:10ED400007D0636B03F0FF130D4A934201D00225F5
:10ED500014E004F16A00FFF756FD20F07F40094BF4
:10ED600098420BD004F18600FFF74DFD064B984208
:10ED700004D0022502E0042500E00325284638BD22
:10ED8000EB00900046415400464154332DE9F04FCA
:10ED900087B00D46164600230B60FFF72FFF071EB6
:10EDA000C0F26781BE4B53F82740002C00F066810B
:10EDB0002C6006F0FE06237873B16078FFF7DAFC6A
:10EDC00010F0010508D1002E00F0548110F0040F5E
:10EDD00000F050810A254DE100232370F8B26070E5
:10EDE000FFF7D4FC10F0010F40F04A811EB110F083
:10EDF000040F40F0478104F10C0202216078FFF714
:10EE0000F1FC0546002840F03F81A289A2F500737D
:10EE10009BB2B3F5606F00F23981531E1A4201D0E4
:10EE2000012527E100212046FFF774FF022800F0AA
:10EE300088800026042800F02B81012800F22A8116
:10EE400004F13F00FFF7DAFCB4F80C80404540F0D5
:10EE5000238104F14A00FFF7D1FC074620B904F1F1
:10EE60005800FFF7D0FC0746E76194F84420A270F1
:10EE7000531EDBB2012B00F2118107FB02F300935A
:10EE800094F84190A4F80A90B9F1000F00F01081B5
:10EE900009F1FF3319EA030F40F00C8104F145003A
:10EEA000FFF7ACFC824620814FEA581BB0FBFBF316
:10EEB0000BFB13039BB2002B40F0FE8004F14700D4
:10EEC000FFF79CFC019020B904F15400FFF79BFC74
:10EED000019004F14200FFF791FC0146002800F088
:10EEE000ED80009BC318BAFBFBFB5B44019A9A427E
:10EEF000C0F0E680D21AB2FBF9F04A45C0F0E280D9
:10EF00004FF6F572904234D840F6F57290426AD9C5
:10EF10004FF0020B2FE0002006AB03EB860343F813
:10EF2000100C0136032E0ED804F13400330103F522
:10EF3000DF7318440379002BEDD00830FFF763FC32
:10EF4000EAE70026EEE700270AE031462046FFF711
:10EF5000E1FE01287FF66EAF0137032F3FF66AAF5F
:10EF600006AB03EB870353F8106C002EEDD10320A2
:10EF7000F2E74FF0030B00F10209C4F81890266283
:10EF80008A1962623344E362BBF1030F2ED0BAF1F7
:10EF9000000F00F09D80009B1A44A262BBF1020F9B
:10EFA00035D009EB490209F0010303EB5203434456
:10EFB000013BB3FBF8F3BB4200F28C804FF0FF3310
:10EFC0006361236180232371BBF1030F22D084F896
:10EFD00000B0344A138801339BB21380E38020468B
:10EFE000FFF70CFD46E04FF0010BC4E704F15E00B3
:10EFF000FFF704FC002867D1BAF1000F66D104F1D5
:10F000006000FFF700FCA0624FEA8903CFE74FEAF8
:10F010004903CCE704F16400FFF7F0FB0128D6D1E7
:10F02000711C2046FFF75BFE0028D0D1002323711E
:10F0300004F23220FFF7E2FB4AF655239842C6D18C
:10F0400004F13400FFF7DFFB174B9842BFD104F502
:10F050000670FFF7D8FB154B9842B8D104F507703E
:10F06000FFF7D1FB606104F50870FFF7CCFB20616E
:10F07000ADE70B25284607B0BDE8F08F0C25F9E772
:10F080000325F7E70A25F5E70125F3E70125F1E771
:10F090000125EFE70D25EDE70D25EBE70D25E9E768
:10F0A0001C3A0020183A00205252614172724161AC
:10F0B0000D25DFE70D25DDE70D25DBE70D25D9E77C
:10F0C0000D25D7E70D25D5E70D25D3E70D25D1E78C
:10F0D0000D25CFE70D25CDE72DE9F047012940F2B9
:10F0E0008E8004460D46174683698B4240F28B8022
:10F0F0000378022B49D0032B60D0012B40F0858090
:10F1000001EB5108416A8389B8FBF3F31944FFF717
:10F11000E6FD0646002873D104F1340A08F101091E
:10F12000A389B8FBF3F203FB128815F0010522D086
:10F130001AF8083003F00F0343EA0713DBB20AF8AA
:10F1400008300123E370616AA389B9FBF3F3194422
:10F150002046FFF7C4FD0646002851D1A389B9FB1C
:10F16000F3F203FB129945B1C7F307130AF809300C
:10F170000123E37044E0FBB2E1E71AF80930C7F37A
:10F18000032223F00F031343F0E7416A83895B08EE
:10F19000B5FBF3F31944FFF7A2FD064680BB04F16B
:10F1A00034006D00A389B5FBF3F203FB1255B9B22D
:10F1B0002844FFF733FB0123E37021E0416A838990
:10F1C0009B08B5FBF3F31944FFF789FD0646B8B970
:10F1D00027F0704704F13403AD00A289B5FBF2F1CA
:10F1E00002FB11551D442846FFF70DFB00F070414E
:10F1F00039432846FFF716FB0123E37000E002269F
:10F200003046BDE8F0870226FAE70226F8E7F8B5AF
:10F21000056801296AD90C46AB698B4268D92B78FD
:10F22000022B35D0032B49D0012B63D101EB5106C2
:10F23000696AAB89B6FBF3F319442846FFF74FFD23
:10F2400010B14FF0FF3052E0771CAB89B6FBF3F200
:10F2500003FB12662E4496F83460696AB7FBF3F339
:10F2600019442846FFF73BFD002845D1AB89B7FB81
:10F27000F3F203FB12772F4497F8343046EA032069
:10F2800014F0010F01D0000931E0C0F30B002EE0B3
:10F29000696AAB895B08B4FBF3F319442846FFF7AE
:10F2A0001EFD60BB05F134006400AB89B4FBF3F2D2
:10F2B00003FB12442044FFF7A1FA18E0696AAB8906
:10F2C0009B08B4FBF3F319442846FFF708FDC8B9BF
:10F2D00005F13400A400AB89B4FBF3F203FB124444
:10F2E0002044FFF790FA20F0704000E00120F8BDC4
:10F2F0000120FCE70120FAE74FF0FF30F7E74FF07D
:10F30000FF30F4E74FF0FF30F1E72DE9F041D0F89E
:10F310000080B1F5001F49D207460E4611F01F0FBD
:10F3200047D1416184681CBB98F80030022B01D999
:10F33000D8F82840E4B9B8F80830B3EB561F3AD9EA
:10F34000D8F82830FB61BC61FB69E3B3B8F80C2046
:10F35000B6FBF2F21344FB6108F13403B8F80C2059
:10F36000B6FBF2F102FB11610B443B6200201EE090
:10F37000B8F80A50B8F80C3003FB05F5AE420FD3CD
:10F3800021463846FFF743FF0446B0F1FF3F14D053
:10F39000012814D9D8F81830834212D9761BEDE72A
:10F3A00021464046FFF748FBF861CCE70220BDE864
:10F3B000F0810220FBE70220F9E70120F7E70220B5
:10F3C000F5E70220F3E70220F1E72DE9F0410546D9
:10F3D00006680F4651B9D6F81080B8F1000F12D068
:10F3E000B369434511D84FF001080EE0FFF70FFF56
:10F3F000034601284CD9B0F1FF3F4ED0B26982429A
:10F400004BD8B84601E04FF0010844460CE02146D5
:10F410002846FFF7FCFE034678B1B0F1FF3F18BF66
:10F4200001283AD0444537D00134B369A342EED81D
:10F43000B8F1010F2ED90224E9E74FF0FF3221463F
:10F440003046FFF749FE0246B0FA80F04009002F2F
:10F4500008BF002070B9A2B934617269B369023B78
:10F460009A4201D8013A7261337943F00103337152
:10F47000234612E0224639463046FFF72DFE02466B
:10F48000E9E7012A01D0012307E04FF0FF3304E050
:10F49000012302E0002300E000231846BDE8F081CC
:10F4A000F8B50C46056801292ED906461146AB6908
:10F4B000A3422BD94AB14FF0FF322846FFF70CFE8A
:10F4C000074610B123E0A24221D927462146304603
:10F4D000FFF79DFE0446E0B101281CD0B0F1FF3FCC
:10F4E0001BD0002239462846FFF7F6FD074670B9C3
:10F4F0006B69AA69911E8B42E5D201336B612B794E
:10F5000043F001032B71DEE7022700E002273846B3
:10F51000F8BD0027FBE70227F9E70127F7E738B531
:10F5200004460568C1692846FFF7D9FB20B9236A5C
:10F53000E5221A700123EB7038BD2DE9F843066807
:10F540004469C369002B74D005460F462034B4F5D6
:10F55000001F70D2B189B4FBF1F201FB12423AB93B
:10F560000133C3618169A1B93389B3EB541F0CD94D
:10F570006C6106F13403B289B4FBF2F102FB114471
:10F5800023442B620020BDE8F8830023C3610420DC
:10F59000F9E7B289B4FBF2F27389013B12EA03087E
:10F5A000E6D1FFF734FE8146012846D9B0F1FF3F8E
:10F5B00045D0B369834234D88FB1A9692846FFF793
:10F5C00004FF814600283CD001283CD0B0F1FF3F29
:10F5D0003BD03046FFF759FB28B10120D3E7002389
:10F5E000EB610420CFE7B289002106F13400FFF778
:10F5F0002DF949463046FFF71FFA30637389984565
:10F600000BD20123F3703046FFF73FFBF8B908F146
:10F610000108336B01333363F0E7336BA3EB08036B
:10F620003363C5F8189049463046FFF705FAE8619C
:10F630009EE70420A7E70420A5E70220A3E7012016
:10F64000A1E707209FE702209DE701209BE701201B
:10F6500099E770B5044606680021FFF756FE054697
:10F6600040B1284670BD00212046FFF766FF0546E1
:10F670000028F6D1E1693046FFF731FB0546002846
:10F68000EFD1206A03787BB1C37A03F03F03A37103
:10F69000C37A13F0080FE6D10B2204F12401FFF71F
:10F6A000DAF80028DFD1DCE70425DAE730B583B0EB
:10F6B00004460191056801E001330193019B1A782A
:10F6C0002F2AF9D05C2AF7D00022A2601B781F2BCA
:10F6D00021D901A92046FFF729FA034618BB204685
:10F6E000FFF7B7FF94F82F200346F8B912F0040F84
:10F6F00019D1A37913F0100F1FD005F134016369FC
:10F70000AA89B3FBF2F002FB103319442846FFF735
:10F71000B2F9A060DDE7802384F82F30114620463F
:10F72000FFF7F3FD0346184603B030BD0428FAD1B5
:10F7300012F0040FF7D10523F5E70523F3E7F8B539
:10F7400004460E4607680021FFF7DFFD0246B8B900
:10F75000002506E0002501212046FFF7EEFE0246C7
:10F7600070B9E1693846FFF7BAFA024640B9236A30
:10F770001B78002B18BFE52BECD10135B542EAD13F
:10F78000042A01D01046F8BD0722FBE770B50446F5
:10F7900006680121FFF7D3FF054608B1284670BD72
:10F7A000E1693046FFF79BFA05460028F6D1202292
:10F7B0000021206AFFF74AF80B2204F12401206A95
:10F7C000FFF73AF80123F370E8E7F8B504460E4670
:10F7D0000568042705E000212046FFF7AEFE074636
:10F7E000E8B9E169D9B12846FFF779FA0746B0B917
:10F7F000236A1A7892B1DB7A03F03F03A371E52AFA
:10F8000018BF2E2AE7D00F2BE5D023F02003082BBA
:10F8100014BF00230123B342DDD100E004270FB160
:10F820000023E3613846F8BD70B50446FFF72DFAB2
:10F83000054648B92378032B08D00022114660788A
:10F84000FEF7D0FF00B10125284670BD2379012BBA
:10F85000F3D104F13406A28900213046FEF7F6FF09
:10F860004AF6552104F23220FEF7D8FF0E49304601
:10F87000FEF7D8FF0D4904F50670FEF7D3FF616966
:10F8800004F50770FEF7CEFF216904F50870FEF756
:10F89000C9FF226A01322263012331466078FEF7F4
:10F8A00095FF00232371C8E7525261417272416192
:10F8B00070B584B0019000911646039103A8FFF73C
:10F8C0009DF9041E20DB114B53F8245025B1284626
:10F8D000FFF794F800232B70019B0BB100221A70E4
:10F8E000019B0A4A42F82430721E18BF0122002BE5
:10F8F00008BF42F0010212B1002004B070BD01A99E
:10F900006846FFF743FAF8E70B20F6E71C3A0020B9
:10F910002DE9F04391B00191002800F010811446C8
:10F92000064602F03F073A4603A901A8FFF72EFA60
:10F93000054628B100233360284611B0BDE8F083A6
:10F94000039B0493019904A8FFF7B0FE054660B934
:10F950009DF93F30002B52DB14F03E0F14BF012104
:10F96000002104A8FEF78CFF054614F01C0F5CD0A4
:10F97000002D50D0042D44D047F00807002DD9D1D8
:10F9800017F0080F61D0F6F7C9FE044601460C983F
:10F990000E30FEF747FF21460C981630FEF742FF67
:10F9A0000C9B2022DA72DDF80C80DDF8309049469D
:10F9B0004046FFF760F80446002249464046FFF7FC
:10F9C0006DF800210C981C30FEF72CFF039B0122E0
:10F9D000DA70002C39D0039BD3F830800022214606
:10F9E00004A8FFF75DFD05460028A3D14146039812
:10F9F000FFF775F90546013C039B1C6125E00625D0
:10FA0000B3E7FEF77BFF08B91225B5E704A8FFF7B7
:10FA1000BDFE0546B0E79DF8163013F0110F13D167
:10FA200014F0040FAAD0082584E7002D82D19DF898
:10FA3000163013F0100F7ED114F0020F05D013F022
:10FA4000010F02D0072575E70725002D7FF472AF5F
:10FA500017F0080F01D047F04007039B1B6B736240
:10FA60000C9BB362012F94BF0021012104A8FEF773
:10FA700055FF306108B902255CE7039CDDF8308052
:10FA800041462046FEF7F7FFB06008F11C00FEF784
:10FA9000BAFEF0600021F1623460E388B38037750C
:10FAA00071753162B16106F130084FF48052404601
:10FAB000FEF7CCFE17F0200F39D0F468002C36D0BA
:10FAC000B461039B5F899B8903FB07F7B16801E081
:10FAD0000225E41BBC4294BF002301235DB953B14E
:10FAE0003046FFF794FB01460128F1D9B0F1FF3F02
:10FAF000EFD10125EDE7F161002D7FF41BAF039FEE
:10FB0000B7F80C90B4FBF9F309FB13437BB138460B
:10FB1000FEF792FF08B902250CE7B4FBF9F20244A4
:10FB20003262012341467878FEF744FE28B9002D61
:10FB30003FF402AFFEE60425FCE60125FAE60925BE
:10FB4000FAE62DE9F04F85B004460F461546984673
:10FB50000023C8F8003003A9FFF774F801900028CB
:10FB600040F0B980637D0193002B40F0B480237D89
:10FB700013F0010F00F0CE80E668A369F61AAE42DA
:10FB800067D32E4665E0E36A1BB12046FEF760FFAF
:10FB900073E0E1692046FFF73AFB6EE04FF0020A9E
:10FBA00084F815A0CDF804A095E04FF0010A84F880
:10FBB00015A0CDF804A08EE04FF0020A84F815A03D
:10FBC000CDF804A087E094F91430002B04DB039BEC
:10FBD0009D890AFB05F532E0236AA3EB090353452F
:10FBE000F5D2039A928904F1300102FB0370FEF70B
:10FBF00023FEECE7226A4A450DD094F91430002B1D
:10FC00006DDB01234A4604F1300103984078FEF78A
:10FC1000D1FD002877D1C4F82090039B9D89A3696A
:10FC2000B3FBF5F205FB1233ED1AAE4200D23546B6
:10FC300004F130012A4619443846FEF7FDFD2F44F1
:10FC4000A3692B44A361D8F800302B44C8F80030D6
:10FC5000761B002E3FD0A169039A9589B1FBF5F37D
:10FC600005FB1313002BD8D1B1FBF5F55389013BEC
:10FC70001D4008D1002986D1A06801288ED9B0F195
:10FC8000FF3F92D0E061DDF80CB0E1695846FEF725
:10FC9000D3FE814600288FD0A944BBF80C30B6FBB8
:10FCA000F3FAB342A6D805EB0A03BBF80A20934245
:10FCB00001D9A2EB050A53464A4639469BF8010092
:10FCC000FEF778FD00283FF47EAF4FF0010A84F87C
:10FCD00015A0CDF804A0019805B0BDE8F08F012370
:10FCE00004F130019BF80100FEF770FD20B9237D7F
:10FCF00003F07F03237584E74FF0010A84F815A011
:10FD0000CDF804A0E7E74FF0010A84F815A0CDF87C
:10FD100004A0E0E707230193DDE72DE9F04F85B06C
:10FD200004460F46154698460023C8F8003003A93C
:10FD3000FEF788FF019000284AD1637D0193002BD4
:10FD400046D1237D13F0020F00F0EC80A369EB4253
:10FD5000C0F0B680DD43B3E0E36A002B3CD0204620
:10FD6000FEF776FE002800F0D880012839D0B0F1E7
:10FD7000FF3F3DD0E061A36803B9A06094F914305F
:10FD8000002B3CDBDDF80CB0E1695846FEF754FE71
:10FD90008146002848D0B144BBF80C30B5FBF3FADB
:10FDA000AB425FD806EB0A03BBF80A20934201D9A5
:10FDB000A2EB060A53464A4639469BF80100FEF775
:10FDC00005FDC0B34FF0010A84F815A0CDF804A0DA
:10FDD000019805B0BDE8F08FE1692046FFF7F5FA1C
:10FDE000C0E74FF0020A84F815A0CDF804A0EFE7B1
:10FDF0004FF0010A84F815A0CDF804A0E8E701232C
:10FE0000226A04F1300103984078FEF7DFFC20B944
:10FE1000237D03F07F032375B4E74FF0010A84F8D4
:10FE200015A0CDF804A0D3E74FF0020A84F815A07E
:10FE3000CDF804A0CCE7236AA3EB0903534504D310
:10FE4000039B9E890AFB06F62BE0039A928902FB2C
:10FE5000037104F13000FEF7EFFC237D03F07F0314
:10FE60002375EDE7236A4B4503D0A269E3689A4204
:10FE700042D3C4F82090039B9E89A369B3FBF6F29A
:10FE800006FB1233F61AB54200D22E4604F13000BA
:10FE9000324639461844FEF7CFFC237D63F07F03DA
:10FEA00023753744A3693344A361E268934238BFA2
:10FEB0001346E360D8F800303344C8F80030AD1B77
:10FEC0005DB3A169039A9689B1FBF6F306FB1313A0
:10FED000002BD0D1B1FBF6F65389013B1E407FF4D5
:10FEE0004DAF00297FF438AFA06800287FF43DAF04
:10FEF0002046FFF76AFA35E701234A4604F130014C
:10FF00009BF80100FEF756FC0028B2D04FF0010A22
:10FF100084F815A0CDF804A05AE7237D43F04003F0
:10FF2000237555E70723019352E770B582B0044665
:10FF300001A9FEF787FE70B9237D13F0400F0AD0A8
:10FF400013F0800F09D1F6F7E9FB0546616A0198C5
:10FF5000FEF7C5FE78B102B070BD0123226A04F13C
:10FF6000300101984078FEF731FC40BB237D03F05F
:10FF70007F032375E7E7A66AF37A43F02003F37261
:10FF8000A26831462068FEF789FDE16806F11C0091
:10FF9000FEF748FC294606F11600FEF743FC002157
:10FFA00006F11200FEF73AFC019B0122DA7001987B
:10FFB000FFF73AFC237D23F040032375CBE70120B4
:10FFC000C9E710B582B00446FFF7AFFF08B102B031
:10FFD00010BD01A92046FEF735FE0028F7D12069A3
:10FFE000FEF7ECFC0028F2D12060F0E72DE9F04F9D
:10FFF00083B004460D4601A9FEF724FE064678B9F3
:020000040801F1
:10000000667D6EB9E36A002B00F08E80B5F1FF3F8C
:100010000AD0E768AF4200D32F46A761002F3FD137
:10002000304603B0BDE8F08F984658F804BBD4F8CA
:1000300008A0BAF1000F27D04FF0020909F1020918
:100040005146002701370D462046FFF7E0F80146EC
:10005000012813D9B0F1FF3F13D001358542F1D00B
:10006000CB4505D3434643F8087BC8F804A098461F
:10007000019B9B698B4209D98A46DFE70226667598
:10008000CEE701266675CBE74FF00209E36AC3F8B5
:100090000090D94500F2FB800023C8F80030BFE78C
:1000A0007D1E29462046FEF7D3FC0146E061DDF8BF
:1000B00004804046FEF7C0FC00B3B8F80C30B5FB36
:1000C000F3F5B8F80A20013A15400544B7FBF3F2FE
:1000D00003FB1277002FA3D0226AAA42A0D094F982
:1000E0001430002B0DDB01232A4604F13001019866
:1000F0004078FEF75FFBA0B9256291E7022666759E
:100100008EE7012304F1300198F80100FEF75EFB51
:1001100020B9237D03F07F032375E4E7012666758C
:100120007EE7012666757BE7E368AB4204D2227D59
:1001300012F0020F00D11D46A3690022A261E5B1B1
:10014000019AB2F80A80928902FB08F873B16A1E1C
:10015000B2FBF8F2013BB3FBF8F18A4206D3C8F1D7
:1001600000021340A361EF1AE56904E0A06850B3F0
:10017000E0612F460546002D45D1A369E268934210
:1001800004D9E360227D42F0400222750198828901
:10019000B3FBF2F102FB1133002B3FF441AF226AB3
:1001A000AA423FF43DAF94F91430002B5DDB0123EC
:1001B0002A4604F1300101984078FEF7FBFA002846
:1001C00062D125622CE700212046FFF7FEF80128C6
:1001D00004D0B0F1FF3F04D0A060C9E702266675E5
:1001E0001EE7012666751BE729462046FFF70FF834
:1001F0000546B5F1FF3F2DD0012D2ED9019B9B69FE
:10020000AB422AD9E561474510D9A7EB0807A36996
:100210004344A361237D13F0020FE5D02946204615
:10022000FFF7D3F805460028E3D10746A3693B440E
:10023000A3610198B0F80C80B7FBF8F308FB1373C7
:100240008BB12946FEF7F8FB054648B1B7FBF8F736
:100250003D4492E701266675E2E602266675DFE612
:1002600002266675DCE61D4687E7012304F13001AE
:100270004078FEF7ABFA20B9237D03F07F032375A6
:1002800095E701266675CBE601266675C8E6112658
:10029000C6E630B58FB001900C46002202A901A835
:1002A000FEF774FD054610B128460FB030BD019928
:1002B00002A8FFF7FBF905460028F5D19DF9373074
:1002C000002B06DB002CEFD0214602A8FEF7F9FB3D
:1002D000EAE70625E8E7F0B59DB00190022203A900
:1002E00001A8FEF753FD039B1093044610B120466E
:1002F0001DB0F0BD019910A8FFF7D8F904460028F9
:10030000F5D1022110A8FEF7BBFA04460028EED171
:100310009DF96F30002B3CDB9DF8465015F0010F26
:1003200039D1039F18993846FEF7A5FB064615F00C
:10033000100F13D1002CDAD110A8FFF7F0F8044603
:10034000B0FA80F04009002E08BF0020D0B9002C80
:10035000CDD10398FFF768FA0446C8E704970690E2
:10036000002104A8FEF7D1FF04460028BFD10021D8
:1003700004A8FFF72AFA044610B10428DAD1DBE713
:100380000724D7E70022314610A8FFF789F8044672
:10039000DDE70624ABE70724A9E72DE9F04F91B08C
:1003A0000190022203A901A8FEF7F0FC039B04932D
:1003B000044618B1204611B0BDE8F08F019904A899
:1003C000FFF774F9002800F09780042801D0044654
:1003D000F0E7002104A8FEF7F8FF039A53899189FA
:1003E00001FB03F30793814618B1012802D10224CF
:1003F00003E00724B9F1FF3F55D0002C4ED0F6F7AB
:100400008DF98246002C56D1039E49463046FEF7B0
:1004100013FB054606F13408B28900214046FEF779
:1004200015FA0B2220214046FEF710FA4FF02E0B52
:1004300086F834B0102386F83F30514606F14A0062
:10044000FEF7F0F94A4641460398FEF727FB06F10E
:100450005407202241463846FEF7EEF986F855B09B
:10046000069A03980378032B1FD03946FEF716FB34
:10047000039B5E89F6B16F1C039B1D630122DA703A
:100480000398FEF702FC0446A0B9039B9A89002159
:100490004046FEF7DBF9013E3D46EBE71046FEF72E
:1004A000F4FB0446ABE70124A9E7836A9342DCD15D
:1004B0000022DAE72CB10022494604A8FEF7F0FF3B
:1004C00078E704A8FFF762F904460028F3D10C9CF2
:1004D000514604F11600FEF7A5F94A462146039855
:1004E000FEF7DCFA1023E372039B0122DA70039813
:1004F000FFF79AF904465DE708245BE7134B5B7A44
:1005000013BB10B5044603F0FF00104B93F809C06D
:100510005FFA8CFC4FF0000E03F80CE093F809C072
:1005200003EB8C0CCCF804405C7A1C4422725A7A9F
:10053000541CE4B25C7230320A703A234B702F23A1
:100540008B7081F803E010BD01207047203A002035
:1005500008B50022FFF7D2FF08BD000010B5034622
:100560000C4A0D490D48006840B10C48006803442E
:10057000521A934206D8094A136010BD0748084C26
:100580000460F2E7F1F700FC0C2303604FF0FF304A
:10059000F3E700BF00000820004000002C3A0020D4
:1005A000303A00200120704708B5F1F7EDFB162323
:1005B00003604FF0FF3008BD08B54FF0FF31FFF783
:1005C000F3FFFEE770B50C461646002506E0AFF3D4
:1005D0000080214601F8010B01350C46B542F6DBDF
:1005E000304670BD70B50C461646002504E014F880
:1005F000010BAFF300800135B542F8DB304670BD2A
:100600004FF0FF3070474FF400534B6000207047AD
:100610000120704700207047026852E8003F23F431
:10062000907342E800310029F6D1026802F1080314
:1006300053E8003F23F00103083242E8003100296B
:10064000F3D1036E012B06D02023C0F880300023A5
:10065000036683667047026852E8003F23F0100388
:1006600042E800310029F6D1EEE7000010B504465B
:1006700083680269134342691343C26913430168E3
:100680000868914A02401A430A602268536823F4BA
:100690004053E1680B435360A269236A1A432168FF
:1006A0008B6823F4306313438B602368874A93423B
:1006B00018D0874A93423AD0864A93424FD0864A0E
:1006C00093425ED0854A93426DD0854A93427FD053
:1006D000844A934200F09180834A934200F0A280C2
:1006E00010230BE0814BD3F8903003F00303032B6E
:1006F0001BD8DFE803F00216AB180123E069B0F560
:10070000004F00F0D780082B00F23881DFE813F0AB
:1007100014012701120136012A0136013601360182
:100720002D010423EAE70823E8E71023E6E76F4BEF
:10073000D3F8903003F00C030C2B0ED8DFE803F055
:10074000070D0D0D090D0D0D880D0D0D0B0000236E
:10075000D4E70423D2E70823D0E71023CEE7634B86
:10076000D3F8903003F03003202B73D005D8002B42
:1007700072D0102B72D10423C0E7302B70D1082324
:10078000BCE75A4BD3F8903003F0C003802B69D0FC
:1007900005D8002B68D0402B68D10423AEE7C02BCE
:1007A00066D10823AAE7514BD3F8903003F4407385
:1007B000B3F5007F5ED006D8002B5DD0B3F5807F07
:1007C0005CD104239AE7B3F5407F59D1082395E71C
:1007D000464BD3F8903003F44063B3F5006F51D02B
:1007E00006D8002B50D0B3F5806F4FD1042385E796
:1007F000B3F5406F4CD1082380E73C4BD3F89030E1
:1008000003F44053B3F5005F44D006D8002B43D027
:10081000B3F5805F42D1042370E7B3F5405F3FD169
:1008200008236BE7314BD3F8903003F44043B3F522
:10083000004F37D005D8BBB3B3F5804F36D1042372
:100840005CE7B3F5404F33D1082357E7022355E760
:10085000022353E7022351E700234FE710234DE71C
:1008600010234BE7022349E7002347E7102345E71E
:10087000102343E7022341E700233FE710233DE72E
:1008800010233BE7022339E7012337E7102335E73D
:10089000102333E7022331E700232FE710232DE74E
:1008A00010232BE7022329E7002327E7102325E75E
:1008B000102323E7082B5BD8DFE803F01A343A5AF9
:1008C000375A5A5A1E0000BFF369FFEF001001406B
:1008D0000044004000480040004C004000500040F0
:1008E0000014014000780040007C004000380240C5
:1008F000FBF7B0F900283DD06268530803EB4003D2
:10090000B3FBF2F3A3F110014FF6EF72914233D82B
:100910009AB222F00F02C3F3420313432268D3605A
:10092000002030E0FBF7A6F9E4E7FBF783F8E1E706
:100930001748E1E7164802E0FBF78CF900B363685B
:1009400000EB5300B0FBF3F0A0F110024FF6EF7391
:100950009A4217D8236880B2D860002013E0FBF7D2
:1009600089F9EBE7FBF766F8E8E74FF40040E6E7C4
:10097000012008E0002006E0012004E0012002E060
:10098000002000E001200023A366E36610BD00BF45
:100990000024F400436A13F0080F06D0026853687D
:1009A00023F40043416B0B435360436A13F0010F80
:1009B00006D00268536823F40033816A0B43536006
:1009C000436A13F0020F06D00268536823F48033A1
:1009D000C16A0B435360436A13F0040F06D00268E8
:1009E000536823F48023016B0B435360436A13F075
:1009F000100F06D00268936823F48053816B0B4379
:100A00009360436A13F0200F06D00268936823F4C2
:100A10000053C16B0B439360436A13F0400F0AD03D
:100A20000268536823F48013016C0B435360036C1A
:100A3000B3F5801F0BD0436A13F0800F06D0026815
:100A4000536823F40023816C0B43536070470268A2
:100A5000536823F4C003416C0B435360EBE72DE96B
:100A6000F84305460E4617469946DDF820802B6868
:100A7000DC6936EA04040CBF01240024BC423AD1EC
:100A8000B8F1FF3FF3D0FBF70FFEA0EB09004045A4
:100A900034D8B8F1000F33D02B681A6812F0040F65
:100AA000E5D0B6F1400218BF0122802EDFD0002A27
:100AB000DDD0DA6912F0080F11D1DA6912F4006F93
:100AC000D5D04FF400621A622846FFF7A5FD202317
:100AD000C5F88430002385F8783003200CE0082422
:100AE0001C622846FFF798FDC5F88440002385F86E
:100AF0007830012000E00020BDE8F8830320FBE708
:100B00000320F9E730B583B004460023C0F88430F1
:100B1000FBF7CAFD05462268126812F0080F0FD1D4
:100B200023681B6813F0040F26D12023E367C4F861
:100B3000803000202066606684F8780003B030BD05
:100B40006FF07E430093034600224FF400112046CD
:100B5000FFF785FF0028E3D0226852E8003F23F02A
:100B6000800342E800310029F6D12023E367002307
:100B700084F878300320E1E76FF07E4300932B4642
:100B800000224FF480012046FFF769FF0028CCD0F7
:100B9000226852E8003F23F4907342E800310029B4
:100BA000F6D1226802F1080353E8003F23F0010365
:100BB000083242E800310029F3D12023C4F8803004
:100BC000002384F878300320B8E768B310B50446F2
:100BD000C36F03B32423E3672268136823F0010380
:100BE0001360636AE3B92046FFF740FD012811D086
:100BF0002268536823F4904353602268936823F07B
:100C00002A0393602268136843F0010313602046AF
:100C1000FFF778FF10BD80F87830F6F71FF8D9E7B6
:100C20002046FFF7B7FEDEE701207047DFF834D03B
:100C3000FDF796FD0C480D490D4A002302E0D458FB
:100C4000C4500433C4188C42F9D30A4A0A4C002316
:100C500001E013600432A242FBD3F0F77BFFF5F70B
:100C600025FC70470000082000000020D80100206B
:100C700038180108D8010020303A0020FEE70000B3
:100C8000F8B500BFF8BC08BC9E467047F8B500BF79
:080C9000F8BC08BC9E46704749
:100C980035000000CEFBFFFFCB0300000100000081
:100CA8000000000034000000CEFBFFFFCB03000073
:100CB8000100000000000000BC89D897B2D29C3C1B
:100CC80033A7A8D523F649393DA7F444FD0FA5322B
:100CD8009D978CCF08BA5B25436FAC6428066811D2
:100CE80000000000000000000000000000000000FC
:100CF80000000000000000000000000000000000EC
:100D080000000000000000000000000000000000DB
:100D180010111213141516171819000000000000FE
:100D2800001A1B1C1D1E1F00000000000000000010
:100D380000000000000000000000000000000000AB
:100D4800001A1B1C1D1E1F000000000000000000F0
:100D5800000000000000000000000000000000008B
:100D6800000000000000000000000000000000007B
:100D7800000000000000000000000000000000006B
:100D8800000000000000000000000000000000005B
:100D9800000000000000000000000000000000004B
:100DA800000000000000000000000000000000003B
:100DB800000000000000000000000000000000002B
:100DC800000000000000000000000000000000001B
:100DD800000000000000000000000000000000000B
:100DE80000202020202020202020282828282820F3
:100DF80020202020202020202020202020202020EB
:100E08002088101010101010101010101010101052
:100E18001004040404040404040404101010101042
:100E2800101041414141414101010101010101010C
:100E3800010101010101010101010101101010105E
:100E480010104242424242420202020202020202DE
:100E58000202020202020202020202021010101032
:100E6800200000000000000000000000000000005A
:100E7800000000000000000000000000000000006A
:100E8800000000000000000000000000000000005A
:100E9800000000000000000000000000000000004A
:100EA800000000000000000000000000000000003A
:100EB800000000000000000000000000000000002A
:100EC800000000000000000000000000000000001A
:100ED800000000000000000000000000000000000A
:100EE80000000000000000000500000019000000DC
:100EF8007D00000000000000000000000000F03F3E
:100F080000000000000024400000000000005940DC
:100F18000000000000408F40000000000088C3402F
:100F280000000000006AF8400000000080842E41A4
:100F380000000000D01263410000000084D79741F0
:100F48000000000065CDCD41000000205FA00242F6
:100F5800000000E876483742000000A2941A6D426B
:100F6800000040E59C30A2420000901EC4BCD6425E
:100F780000003426F56B0C430080E03779C3414309
:100F880000A0D8855734764300C84E676DC1AB437F
:100F9800003D9160E458E143408CB5781DAF15449D
:100FA80050EFE2D6E41A4B4492D54D06CFF0804478
:100FB800F64AE1C7022DB544B49DD9794378EA448D
:100FC800BC89D897B2D29C3C33A7A8D523F6493917
:100FD8003DA7F444FD0FA5329D978CCF08BA5B2539
:100FE800436FAC642806C80A0080E03779C34143E0
:100FF800176E05B5B5B89346F5F93FE9034F384D77
:10100800321D30F94877825A3CBF737FDD4F157522
:10101800196600084D6600086166000885660008C4
:10102800A966000870726F66696C65732E637376C3
:1010380000000000310000007472756500000000B7
:10104800796573003000000066616C73650000000C
:101058006E6F000070726F66696C655F6E616D65BA
:10106800000000006175746F5F72756E000000000B
:10107800626F6F745F656E61626C6564000000008A
:10108800776F726B5F656E61626C6500753576317E
:101098005F656E61626C6500753576325F656E619D
:1010A800626C65006C64315F656E61626C6500003E
:1010B8006C64325F656E61626C65000072656631F2
:1010C8005F656E61626C6500726566325F656E6150
:1010D800626C6500746563315F656E61626C6500A2
:1010E800746563325F656E61626C65007473315F4D
:1010F800656E61626C6500007473325F656E616273
:101108006C650000706964315F66726F6D5F686F4F
:1011180073740000706964325F66726F6D5F686F28
:101128007374000061766572616765730000000082
:101138006D6573736167655F696400006C617365F1
:1011480072315F7461726765745F74656D700000F9
:101158006C61736572325F7461726765745F746520
:101168006D7000006C61736572315F6375727265D2
:101178006E7400006C61736572325F6375727265BC
:101188006E7400006C61736572315F7069645F70C2
:10119800000000006C61736572315F7069645F699B
:1011A800000000006C61736572325F7069645F7083
:1011B800000000006C61736572325F7069645F697A
:1011C8000000000077617665666F726D5F6D6F6411
:1011D800650000007361770067656E65726174650C
:1011E800645F7372616D0000637573746F6D5F7314
:1011F80072616D0077617665666F726D5F656E61AD
:10120800626C650077617665666F726D5F7472698E
:10121800616E676C6500000077617665666F726D58
:101228005F7361775F73746570000000776176653E
:10123800666F726D5F7061745F6261736500000054
:1012480077617665666F726D5F7061745F706572E5
:10125800696F640077617665666F726D5F73616D43
:10126800706C655F636F756E7400000077617665FA
:10127800666F726D5F686F6C645F6379636C6573CA
:101288000000000077617665666F726D5F616D7052
:101298006C6974756465000077617665666F726D58
:1012A8005F736F75726365006164393833335F65E6
:1012B8006E61626C650000006164393833335F74B5
:1012C8007269616E676C65006164393833335F66D3
:1012D80072657175656E63795F776F72640000007F
:1012E80073746D33325F6461635F656E61626C65F0
:1012F8000000000073746D33325F6461635F636F75
:10130800646500007465635F6D6F64756C61746912
:101318006F6E5F656E61626C650000007465635F87
:101328006D6F64756C6174696F6E5F6C6173657203
:10133800000000007465635F6D6F64756C617469AB
:101348006F6E5F6672657175656E63795F687A0046
:101358007465635F6D6F64756C6174696F6E5F61EE
:101368006D706C69747564655F636F646500000017
:101378006473313830395F6170706C790000000037
:101388006473313830395F706F736974696F6E5F79
:1013980066726F6D5F6D696E0000000070726F6637
:1013A800696C65732F50524F46253034752E494E5F
:1013B8004900000077617665732F574156452530FF
:1013C80034752E435356000070726F66696C6573EE
:1013D80000000000776176657300000025732C25F6
:1013E800732C25730D0A0000574F524B0000000064
:1013F8004552524F5200000049444C45000000003D
:101408004E6F2070726F66696C6500004D616E7575
:10141800616C20636F6E74726F6C00002573204FCF
:101428004B000000257320455252202530325800C9
:10143800222A2B2C3A3B3C3D3E3F5B5D7C7F0000E3
:101448002E0000006E660000696E69747900000065
:10145800616E000042616C6C6F6320737563636535
:1014680065646564000000002E2E2F2E2E2F2E2E70
:101478002F2E2E2F2E2E2F2E2E2F6E65776C696213
:101488002F6C6962632F7374646C69622F6764746C
:101498006F612D6765746865782E630043000000EE
:1014A800504F5349580000002C2066756E637469CC
:1014B8006F6E3A2000000000617373657274696F83
:1014C8006E2022257322206661696C65643A206665
:1014D800696C6520222573222C206C696E65202595
:1014E80064257325730A00005245454E54206D61EA
:1014F8006C6C6F6320737563636565646564000075
:101508002E2E2F2E2E2F2E2E2F2E2E2F2E2E2F2EEE
:101518002E2F6E65776C69622F6C6962632F737406
:10152800646C69622F6D707265632E630000000041
:10153800232D302B20000000686C4C006566674541
:101548004647000030313233343536373839414276
:1015580043444546000000003031323334353637D5
:101568003839616263646566000000000000F9189C
:10157800FC301D47825A6D6A41768A7DFF7F8A7DDD
:1015880041766D6A825A1D47FC30F918000007E75A
:1015980004CFE3B87EA59395BF89768201807682D1
:1015A800BF8993957EA5E3B804CF07E711111E0EF6
:1015B8000D0122220200FF0244440200FF03666676
:1015C8000200FF0477771E0E0D0588880A040306BB
:1015D80099990A040307AAAA0A040308BBBB0A04C8
:1015E8000309CCCC0A04030ADDDD1E0E0D0BEEEE5A
:1015F8001E0E0D0CF0F00A04030D00000000000E92
:101608000000000000000000000000400000000092
:1016180000000000001F0000000000000E00000095
:10162800000000000000000030301101FFFF000042
:10163800010103000000000000000000000000009D
:101648000000000000400000000200000000000050
:101658000000000000000000000000000000000082
:101668000000000000000000000000000000000072
:1016780000000000A00F0000F03F00010100010081
:101688000000000000000000000000000000004012
:101698000000000000000000001F00000000000023
:1016A8000E000000000000000000000012322101BE
:1016B800FFFF00000101030000000000000000001F
:1016C8000000000000000000004000000606991914
:1016D800009A000000000000000000000000000068
:1016E800A00F000000000000000000000000000043
:1016F8000000000000000000000000000000FF16CD
:1017080001000100000001000200030004000500C0
:1017180006000700080009000A000B000C000D0075
:101728000E001F00200022002300240025002600B0
:101738002700280029002A002B002C002D002E004D
:101748002F003000310032003300340035003600FD
:1017580037003E003F004000410042004300440083
:1017680045004700500051005200530054005500F6
:1017780056005700580059005A005B005C005D0095
:101788005E005F001E001D0000000000010203044F
:101798000000000000000000010203040607080919
:1017A80043554541414141434545454949494141E1
:1017B8004592924F4F4F5555594F554F9C4F9E9FAD
:1017C80041494F55A5A5A6A7A8A9AAABACADAEAFF0
:1017D800B0B1B2B3B4414141B8B9BABBBCBDBEBFE8
:1017E800C0C1C2C3C4C54141C8C9CACBCCCDCECF84
:1017F800D1D145454549494949D9DADBDCDD49DFDD
:101808004FE14F4F4F4FE6E8E85555555959EEEF20
:10181800F0F1F2F3F4F5F6F7F8F9FAFBFCFDFEFF48
:081828009803FF7F010000009E
:041830006902000841
:041834004102000865
:101838000400002000000000F40100205C020020E9
:10184800C4020020000000000000000000000000AA
:101858000000000000000000000000000000000080
:101868000000000000000000000000000000000070
:101878000000000000000000000000000000000060
:10188800430000000000000000000000000000000D
:101898000000000000000000000000000000000040
:1018A80043000000000000000000000000000000ED
:1018B8000000000000000000000000000000000020
:1018C80043000000000000000000000000000000CD
:1018D8000000000000000000000000000000000000
:1018E80043000000000000000000000000000000AD
:1018F80000000000000000000000000000000000E0
:10190800430000000000000000000000000000008C
:1019180000000000000000000000000000000000BF
:10192800430000000000000000000000000000006C
:10193800000000000000000000000000000000009F
:10194800430000000000000000000000000000004C
:10195800000000000000000000000000000000007F
:10196800151F00080937000800000000E80D0108ED
:1019780048140108BC140108BC140108BC1401086F
:10198800BC140108BC140108BC140108BC140108EB
:10199800BC140108BC140108FFFFFFFFFFFFFFFF95
:1019A800FFFFFFFFFFFF00000100415343494900CB
:1019B800000000000000000000000000000000001F
:1019C80000000000000000000000415343494900A6
:1019D80000000000000000000000000000000000FF
:1019E80000000000000000000000000000000000EF
:1019F80003000000F40100200101020101010100BF
:081A0800100000000024F400AE
:0400000508010C2DB5
:00000001FF
